:100000000C94EF300C94E9330C9414340C943F347A
:100010000C946A340C9495340C94C0340C94EB34E6
:100020000C9416350C9420310C9420310C94203112
:100030000C9420310C9420310C9420310C942031FC
:100040000C9420310C94E4E00C9420310C94203179
:100050000C9420310C9420310C9476CF0C942231E6
:100060000C9420310C9451A70C94FDA70C942031D2
:100070000C9420310C9420310C9420310C942031BC
:100080000C9420310C9420310C9420310C942031AC
:100090000C9420310C9420310C9420310C9420319C
:1000A0000C9420310C9420310C9420310C9420318C
:1000B0000C9420310C9420310C9420310C9420317C
:1000C0000C9420310C9420310C9420310C9420316C
:1000D0000C9420310C9420310C9420310C9420315C
:1000E0000C9420315F326432693273327D32F632E1
:1000F00087328F329732A132AB32B532C432CE3230
:10010000F632D832E232EC321A331D330C3310336C
:1001100016335433213325332B332F3333333933D1
:100120003D334133543347334B334F33086BE86A25
:10013000EE6AEB6AF16AF46AF76A036BFA6A146BA7
:10014000FD6A006B8CA48AA4AEA4ABA4A9A4E0A40D
:10015000DDA4DBA439A507A504A502A584A78AA769
:100160009BA7A6A7AEA7C3A7B2A7C3A7B6A7BAA7C0
:10017000C3A7C0A700B605B60AB612B617B61CB616
:1001800021B626B643B643B62BB643B630B635B61F
:100190003EB65EB663B668B670B675B67AB67FB66A
:1001A00084B6A1B6A1B689B6A1B68EB693B69CB6F2
:1001B000BCB6C1B6C6B6CEB6D3B6D8B6DDB6E2B614
:1001C000FFB6FFB6E7B6FFB6ECB6F1B6FAB61AB7A9
:1001D0001FB724B72CB731B736B73BB740B75DB7B9
:1001E0005DB745B75DB74AB74FB758B724B829B818
:1001F00034B83FB84AB855B860B86BB8A0B8A0B822
:10020000A0B8A0B876B8BFB8CBB8DCB8EDB8FEB827
:100210000FB920B931B969B969B969B969B93FB9D3
:1002200088B994B9A5B9B6B9C7B9D8B9E9B9FAB90D
:1002300032BA32BA32BA32BA08BA51BA5ABA69BA0A
:1002400074BA7FBA8ABA95BA9FBACEBACEBACEBAC3
:10025000CEBAA7BA10BB16BB27BB33BB3FBB56BB3E
:1002600066BB49BC76BB49BC86BB49BC97BBA3BB3C
:10027000B8BBC4BBF6BB07BC16BC22BC2EBC3DBC85
:1002800070BC79BC8DBC9CBCABBCC5BCD8BCEDBD46
:10029000EBBCEDBDFEBCEDBD12BD24BD3CBD56BDED
:1002A0008BBD9FBDB1BDC0BDCFBDE1BD14BE1DBEE8
:1002B00031BE40BE4FBE69BE7CBE91BF8FBE91BFF6
:1002C000A2BE91BFB6BEC8BEE0BEFABE2FBF43BF3E
:1002D00055BF64BF73BF85BFB8BFBEBFCDBFD7BF5B
:1002E000DFBFF4BF02C0DFC010C0DFC01EC0DFC070
:1002F0002DC03CC04DC064C099C0A8C0B7C0BFC02D
:10030000C7C0D6C0084AD73B3BCE016E84BCBFFDF8
:10031000C12F3D6C74319ABD56833DDA3D00C77FD5
:1003200011BED9E4BB4C3E916BAAAABE000000806E
:100330003F05A84CCDB2D44EB93836A9020C50B9FD
:10034000918688083CA6AAAA2ABE000000803F0029
:100350000D9491660D94DA1E0D94B6440D94866B3F
:100360004E414E494E495459494E46CDCCCC3D0A9A
:10037000D7233C17B7D13877CC2B329595E6241F7D
:10038000B14F0A000020410000C84200401C462036
:10039000BCBE4CCA1B0E5AAEC59D7400000A0B02AF
:1003A000090C0D0E08070304010000000000000006
:1003B000000000000000000000000000000000003D
:1003C00000000000000000121110000000000000FA
:1003D000000000000000000000000000000000001D
:1003E0000001021020200808102040102040800248
:1003F000010201080402010102040810204080806B
:1004000040201008040201800402018040201008EE
:1004100004020108040201010204081020408001C6
:100420000204081020408005050505070508080896
:1004300008020202020A0A08080404040401010175
:10044000010101010103030303030303030407077D
:10045000070C0C0C0C0C0C0C0C020202020606061B
:1004600006060606060B0B0B0B0B0B0B0B000020F6
:10047000002300260029002C002F0032000001007C
:100480000003010601090100002200250028002BBD
:10049000002E003100340002010000050108010BAC
:1004A0000100002100240027002A002D0030003325
:1004B0000001010000040107010A0101060D00FE10
:1004C00009016602D620FFFE0BFE0AFE0D00602227
:1004D0001969808080808080800080183363A0A0AC
:1004E000A00357675050F850F850500259692078CF
:1004F000A0A0702828F02002596948A85010204078
:1005000050A89002586840A0A040A0989068281376
:1005100063808080113B6B204040808080808040E1
:100520004020113B6B804040202020202040408014
:1005300006556520A870A8200455652020F82020C5
:10054000113363604080065161F811336340E0402D
:100550000259690808101020404080800259692023
:1005600050888888888850200259692060A02020FF
:10057000202020F80259697088880810204080F8EF
:10058000025969F80810207008088870025969102B
:100590001030505090F81010025969F88080B0C89F
:1005A0000808887002596970888080F0888888708F
:1005B000025969F808101020204040400259697023
:1005C00088888870888888700259697088888878D7
:1005D0000808887011386840E040000040E0401191
:1005E000386840E0400000604080025969081020EF
:1005F000408040201008045464F80000F802596953
:1006000080402010081020408002596970888808B6
:10061000102020002002596970888898A8A8B0800E
:10062000780259692050888888F888888802596932
:10063000F048484870484848F002596970888080FE
:100640008080808870025969F04848484848484886
:10065000F0025969F8808080F0808080F802596942
:10066000F8808080F0808080800259697088808066
:10067000809888887002596988888888F88888886E
:1006800088123969E040404040404040E0025969EA
:10069000381010101010109060025969888890A0CE
:1006A000C0A0908888025969808080808080808086
:1006B000F80259698888D8A8A88888888802596962
:1006C00088C8C8A8A89898888802596970888888B6
:1006D0008888888870025969F0888888F0808080CE
:1006E00080015A6A70888888888888A870080259AA
:1006F00069F0888888F0A09088880259697088809D
:10070000807008088870025969F820202020202075
:1007100020200259698888888888888888700259CA
:1007200069888888885050502020025969888888B4
:1007300088A8A8A8A850025969888850502050500D
:10074000888802596988885050202020202002592A
:1007500069F808101020404080F8113B6BE0808061
:1007600080808080808080E00259698080404020C5
:1007700010100808113B6BE02020202020202020B2
:1007800020E0085363205088015161F82A226280DA
:10079000400256667008788898680259698080809F
:1007A000F088888888F00256667088808088700299
:1007B0005969080808788888888878025666708899
:1007C000F880887002596930484040F0404040400D
:1007D0000058687088888878088870025969808015
:1007E00080B0C8888888881238684000C04040407F
:1007F00040E0004A6A100030101010109090600223
:10080000596980808090A0C0A09088123969C0404A
:10081000404040404040E0025666D0A8A8A8A888C2
:10082000025666B0C88888888802566670888888AC
:100830008870005868F0888888F080808000586848
:100840007888888878080808025666B0C880808052
:10085000800256667088601088700258684040F0C8
:10086000404040483002566688888888986802561A
:10087000668888885050200256668888A8A8A850A4
:1008800002566688502020508800586888888898CA
:1008900068088870025666F810204080F8015B6B8B
:1008A0001820202020C020202020182219698080B4
:1008B00080808080808080015B6BC0202020201899
:1008C00020202020C008536348A890FFFFFFFFFFAF
:1008D000FFFFFFFFFFFFFFFFFFFFFFFFFFFFFFFF28
:1008E000FFFFFFFFFFFFFFFFFFFFFFFF0D00602285
:1008F0001969800080808080808080035868207023
:10090000A8A0A0A8702002596930484040E04040AB
:1009100048B00356668870505070880259698888BC
:100920005050F820F82020221969808080800080B3
:10093000808080124A6A6090806090906010906021
:100940001A3262A0A00359697088A8D8C8D8A888AC
:1009500070045767700878887800F8035666285046
:10096000A0A05028045363F80808163161E0035929
:10097000697088E8D8D8E8D888700A5161F81744B7
:1009800064609090600357672020F8202000F807EB
:10099000356540A02040E007356540A04020C02AD2
:1009A000226240800058688888888898E8808002A1
:1009B000596978E8E8E8E868282828262161C020F5
:1009C0002262408007356540C04040E004576770B0
:1009D0008888887000F8035666A050282850A00226
:1009E0005A6A40C04040E00818283808025A6A4055
:1009F000C04040E01028081038025A6A40A0402049
:100A0000A048182838080259692000202040808812
:100A10008870025A6A40200020508888F88888022E
:100A20005A6A10200020508888F88888025A6A3054
:100A3000480020508888F88888025A6A2850002088
:100A4000508888F88888025A6A5050002050888858
:100A5000F88888025A6A20502020508888F88888B0
:100A600002596958A0A0A0B0E0A0A0B8005B6B70CC
:100A700088808080808088702040025A6A402000F0
:100A8000F88080F08080F8025A6A102000F8808098
:100A9000F08080F8025A6A304800F88080F0808048
:100AA000F8025A6A505000F88080F08080F8123ABC
:100AB0006A804000E04040404040E0123A6A2040F6
:100AC00000E04040404040E0124A6A609000E04050
:100AD00040404040E0123A6AA0A000E04040404060
:100AE00040E0025969F0484848E8484848F0025A4E
:100AF0006A2850008888C8A8988888025A6A4020C6
:100B00000070888888888870025A6A10200070886F
:100B10008888888870025A6A304800708888888877
:100B20008870025A6A285000708888888888700205
:100B30005A6A505000708888888888700355658884
:100B400050205088015B6B08709898A8A8A8C8C866
:100B50007080025A6A4020008888888888887002DD
:100B60005A6A10200088888888888870025A6A30FB
:100B7000480088888888888870025A6A505000889F
:100B8000888888888870025A6A10200088885020D7
:100B900020202002596980F0888888F080808002B7
:100BA0005969609090A0A0908888B002596940204F
:100BB00000700878889868025969102000700878D9
:100BC00088986802596930480070087888986802E7
:100BD00059692850007008788898680259695050FF
:100BE00000700878889868025A6A304830007008A7
:100BF00078889868025666702870A0A850005868D7
:100C00007088808088702040025969402000708878
:100C1000F88088700259691020007088F880887008
:100C20000259693048007088F8808870025969500C
:100C300050007088F8808870123969804000C04088
:100C4000404040E0123969204000C040404040E050
:100C5000124969609000C040404040E0123969A0EC
:100C6000A000C040404040E0025A6A50206010702E
:100C70008888888870025969285000B0C888888898
:100C800088025969402000708888888870025969F4
:100C90001020007088888888700259693048007078
:100CA00088888888700259692850007088888888E8
:100CB000700259695050007088888888700357679F
:100CC000202000F8002020015868087098A8A8C8C3
:100CD0007080025969402000888888889868025985
:100CE000691020008888888898680259693048000F
:100CF0008888888898680259695050008888888850
:100D00009868005B6B102000888888986808887055
:100D1000005A6A8080B0C88888C8B08080005B6B49
:100D2000505000888888986808887001050700FE80
:100D30000500FB01F220FFFE05FE05FE0200400259
:100D400015258080800080053242A0A002556550A4
:100D5000F850F8500146562070C030E0200255652A
:100D60009010204048025565608068906805122206
:100D700080800225354080808040022535804040BB
:100D80004080043343A040A003334340E0400122AD
:100D9000324080043141E002112180025565081083
:100DA0002040800245556090909060022535C040FB
:100DB000404040024555E0106080F0024555E0108B
:100DC0006010E00245552060A0F020024555F080FB
:100DD000E010E00245556080E09060024555F0105B
:100DE00020404002455560906090600245556090FB
:100DF0007010600313238000800214248000808020
:100E00000235452040804020033343E000E00235B6
:100E1000458040204080024555E01060004002556A
:100E2000657088B8A870024555609090F0900245B2
:100E300055E090E090E0023545608080806002459A
:100E400055E0909090E0023545E080E080E002358A
:100E500045E080E080800245557080B0907002458A
:100E6000559090F09090023545E0404040E00245BA
:100E700055301010906002455590A0C0A0900235EA
:100E80004580808080E002556588D8A88888024522
:100E90005590D0B09090024555609090906002457A
:100EA00055E09090E080014656609090906010026E
:100EB0004555E09090E09002455570806010E0024A
:100EC0003545E0404040400245559090909060028A
:100ED00045559090A0A04002556588A8A8A850024A
:100EE000455590906090900245559090701060022A
:100EF0003545E0204080E0022535C0808080C0027A
:100F000055658040201008022535C0404040C0058E
:100F1000324240A0024151F0052232804002445446
:100F20007090907002455580E09090E002344460EB
:100F3000808060024555107090907002445460B0FB
:100F4000C0600235452040E0404000465670909019
:100F500070106002455580E0909090021525800049
:100F60008080800027374000404040408002455547
:100F70008090A0E0900215258080808080025464DB
:100F8000F0A8A8A8024454E09090900244546090C5
:100F90009060004656E09090E08080004656709049
:100FA00090701010023444A0C0808002445470C07D
:100FB00030E002354540E04040200244549090909B
:100FC000700244549090A040025464A8A85050026B
:100FD0003444A04040A000465690909070106002AB
:100FE0004454F02040F002354560408040600215D6
:100FF000258080808080023545C0402040C0054269
:101000005250A0FFFFFFFFFFFFFFFFFFFFFFFFFFAB
:10101000FFFFFFFFFFFFFFFFFFFFFFFFFFFFFFFFE0
:10102000FFFFFFFF020040FFFFFFFFFFFFFFFFFF8B
:10103000FFFFFFFFFFFFFFFFFFFFFFFFFFFFFFFFC0
:10104000FFFFFFFFFFFFFFFFFFFFFFFFFFFFFFFFB0
:10105000FFFFFFFFFFFFFFFFFFFFFFFFFFFFFFFFA0
:10106000FFFFFFFFFFFFFFFFFFFFFFFFFFFFFFFF90
:10107000FFFFFFFFFFFFFFFFFFFFFFFFFFFFFFFF80
:10108000FFFFFFFFFFFF01050800FF0601210235FA
:1010900020FFFF07FF06FF090050221656808080C0
:1010A000800080153353A0A0A00257575050F8502D
:1010B000F850500257572070A070287020133555F3
:1010C00080A040A02002475740A0A040A0A05025EB
:1010D00013538080801226564080808080401226E4
:1010E000568040404040800245559060F06090023C
:1010F00055552020F8202011335360408004415181
:10110000F011335340E040024656101020408080DA
:1011100012365640A0A0A0A04012365640C0404013
:1011200040E00246566090106080F0024656F02083
:10113000601090600246562060A0F02020024656C3
:10114000F080E01090600246566080E0909060026F
:101150004656F01020204040024656609060909025
:1011600060024656609090701060122555C0C00015
:10117000C0C0113656606000604080123656204074
:1011800080804020034353F000F012365680402008
:1011900020408012365640A0204000400158583070
:1011A0004898A8A8904030024656609090F09090E1
:1011B000024656E090E09090E002465660908080B3
:1011C0009060024656E090909090E0024656F08083
:1011D000E08080F0024656F080E080808002465633
:1011E000609080B090600246569090F0909090127F
:1011F0003656E040404040E002465670202020A095
:101200004002465690A0C0A0A09002465680808022
:101210008080F002465690F0F090909002465690F2
:10122000D0F0B0B090024656609090909060024628
:1012300056E09090E08080014757609090D0B06079
:1012400010024656E09090E0909002465660904022
:10125000209060123656E040404040400246569092
:1012600090909090600246569090909060600246F8
:1012700056909090F0F0900246569090606090905A
:10128000025656888850202020024656F0102040F2
:1012900080F0123656E080808080E00246568080E2
:1012A00040201010123656E020202020E016325246
:1012B00040A0014151F016225280400244547090E7
:1012C00090700246568080E09090E0123454608026
:1012D000806002465610107090907002445460B0C6
:1012E000C060024656205040E040400145556090A5
:1012F0007010600246568080E09090901236564002
:1013000000C04040E01137572000202020A04002BC
:101310004656808090E09090123656C04040404043
:10132000E0025454D0A8A8A8024454E0909090023F
:10133000445460909060014555E090E08080014504
:10134000557090701010024454A0D0808012345414
:1013500060C020C00246564040E040502002445445
:1013600090909070123454A0A0A04002545488A8C9
:10137000A850024454906060900145559090709040
:1013800060024454F02040F0024757304020C02013
:101390004030221656808080808080024757C020CF
:1013A00040304020C006425250A0FFFFFFFFFFFF29
:1013B000FFFFFFFFFFFFFFFFFFFFFFFFFFFFFFFF3D
:1013C000FFFFFFFFFFFFFFFFFFFFFF090050221697
:1013D000568000808080800146562070A0A070203A
:1013E0000246562050E04050A0025555887050707B
:1013F000880256568850F820F8202217578080809F
:10140000008080800247577080E0907010E01731B4
:1014100051A002565670A8C8C8A87014355560A0CF
:101420006000E003435350A050123353E0202014D7
:101430003151E002565670E8D8E8D870173151E0C3
:1014400015335340A04012355540E04000E01435BC
:101450005540A02040E0143555C020C020C01622C1
:10146000524080014555909090E08002565678E8B1
:10147000E8682828241151801122524080143555E3
:1014800040C04040E014355540A04000E0034353C5
:10149000A050A0024757808080A060F020024757EC
:1014A0008080A0D010207002475780408060A0F05C
:1014B0002012365640004080A0400247574020602E
:1014C00090F0909002475720406090F09090024733
:1014D0005760906090F0909002475750A06090F055
:1014E000909002475790006090F0909002475760AC
:1014F000906090F0909002465670A0A0F0A0B001CD
:101500004757609080809060400247574020F080AD
:10151000E080F00247572040F080E080F00247571B
:101520006090F080E080F00247579000F080E0800B
:10153000F01237578040E0404040E01237572040DB
:10154000E0404040E012375740A0E0404040E01209
:101550003757A000E0404040E00256567048E84847
:10156000487002475750A090D0B090900247574023
:10157000206090909060024757204060909090606B
:101580000247576090609090906002475750A0606B
:101590009090906002475790006090909060123356
:1015A00053A040A002465670B0B0D0D0E0024757DA
:1015B00040209090909060024757204090909090EB
:1015C000600247576090909090906002475790005B
:1015D0009090909060025757102088502020200251
:1015E000465680E09090E0800246566090A0A09021
:1015F000A00247574020007090907002475720404B
:1016000000709090700247572050007090907002C8
:10161000475750A00070909070024656500070904E
:10162000907002475760906070909070025454F030
:1016300068B078113555608080604002475740207F
:101640000060B0C06002475720400060B0C0600238
:10165000475760900060B0C060024656500060B0CE
:10166000C060123757804000C04040E0123757201A
:101670004000C04040E012375740A000C04040E06A
:10168000123656A000C04040E0024757A040A010CC
:1016900070906002475750A000E09090900247572A
:1016A000402000609090600247572040006090907A
:1016B000600247576090006090906002475750A0CA
:1016C00000609090600246569000609090601235E5
:1016D000554000E0004002445470B0D0E00247574B
:1016E00040200090909070024757204000909090CA
:1016F000700247576090009090907002465690009C
:101700009090907001485820400090907090600137
:1017100047578080E090E08080014757900090908C
:1017200070906025753A2530327500253032753A53
:101730002530327500202020200025202000252083
:1017400000253164002532640025336400253464AB
:101750000025356400253664000000007E0060002E
:10176000600060F87ECC60CC60CC60F860CC00CCCF
:1017700000CC00CC00000000000000FE7F0E7026B0
:1017800064724E7A5E324C8241324C7A5E724E26E0
:10179000640E70FE7F000000000000FE7F0E70C629
:1017A00063C24382411A58BA5D1A588241C243C685
:1017B000630E70FE7F00000000000088088808109B
:1017C0001120222022101188088808101100000022
:1017D000000000000000000000000020221011881E
:1017E000088808101120222022101188080000000B
:1017F00000000000000000000000000000000000E9
:10180000000000000000000000000000000000FEDA
:101810007FFE7F06600000000000000000F00FF86F
:101820001FF81FF81FF00FF00FF81FF81FF81FE048
:1018300007C0038001000000003048483045727244
:101840003A207574663820666F6E74206E6F74204F
:10185000696E697469616C697A65642E004572729B
:101860003A207574663820666F6E74206E6F74202F
:10187000696E697469616C697A65642E004572727B
:101880003A207574663820666F6E74206E6F74200F
:10189000696E697469616C697A65642E00506C6563
:1018A000617365207265736574005052494E5445EA
:1018B000522048414C544544007F80FFC0FFC0FF88
:1018C000C07F807F80FFC0FFC0FFC03F001E000CB4
:1018D00000FFFFFF0E000E000E000E000E000E00B7
:1018E0000E000E007FC03F801F000E0004000400A9
:1018F0000E001F003F807FC00E000E000E000E0085
:101900000E000E000E000E0000FE0003FF80078395
:10191000C00E01C00E00E01C00E07F00E03E00E0D1
:101920001C00E00800E00000E00001C00E01C00F54
:10193000078007FF0001FC0003F8000FFE001E0FE8
:1019400000380700380380700380700FE07007C014
:101950007003807001007000003800003807001E1E
:101960000F000FFE0003F80000060C00FE07022621
:1019700003BC017FFE08FE08FE05080806000040C3
:10198000F0C88888987810050808060000C0F88814
:1019900088888888F80505050600012030F8302081
:1019A0000508080600002070F820202020E0050926
:1019B000090600FF2070A8A8B888887020050606D0
:1019C000060001E08CEA8C8A0A0509090600FFF886
:1019D000A88888888888A8F8050A0A0600FE20508A
:1019E00050505088A8A8887003030306000340A045
:1019F00040FFFFFFFFFFFFFFFFFFFFFFFFFFFFFFB6
:101A0000FFFFFFFFFFFFFF0000000605FF010707C4
:101A100006020080808080800080030303060105A9
:101A2000A0A0A005060606000050F85050F850058A
:101A300009090600FF2070A8A07028A870200507DB
:101A400007060000C8C81020409898050707060040
:101A50000040A0A040A89068010303060205808012
:101A6000800309090601FF2040408080804040201B
:101A70000309090601FF80404020202040408005E6
:101A8000070706000020A8702070A820050505069D
:101A900000012020F820200203030601FFC040803F
:101AA000050101060003F8020202060100C0C0059C
:101AB00007070600000810102040408005070706B1
:101AC0000000708898A8C8887003070706010040C6
:101AD000C040404040E0050707060000708808103D
:101AE0002040F8050707060000F808103008887045
:101AF00005070706000010305090F8101005070782
:101B0000060000F880F00808887005070706000046
:101B1000304080F0888870050707060000F808103C
:101B2000102020200507070600007088887088882C
:101B300070050707060000708888780810600205A5
:101B400005060100C0C000C0C00206060601FFC0B5
:101B5000C000C040800305050601012040804020F0
:101B6000050303060002F800F803050506010180DD
:101B700040204080050707060000708810202000E4
:101B8000200507070600007088B8A8B88070050710
:101B900007060000708888F888888805070706000F
:101BA00000F04848704848F00507070600007088B4
:101BB0008080808870050707060000F04848484884
:101BC00048F0050707060000F88080F08080F805DF
:101BD0000707060000F88080F08080800507070670
:101BE00000007088808098887005070706000088CC
:101BF0008888F8888888030707060100E04040408D
:101C00004040E005070706000038101010109060F3
:101C10000507070600008890A0C0A0908805070768
:101C2000060000808080808080F80507070600009D
:101C300088D8A8888888880507070600008888C88B
:101C4000A898888805070706000070888888888813
:101C500070050707060000F08888F080808005077F
:101C60000706000070888888A890680507070600A6
:101C700000F08888F0A090880507070600007088AB
:101C80008070088870050707060000F820202020D3
:101C90002020050707060000888888888888700546
:101CA0000707060000888888885050200507070627
:101CB000000088888888A8A85005070706000088C3
:101CC0008850205088880507070600008888502023
:101CD000202020050707060000F80810204080F8A3
:101CE0000309090601FFE080808080808080E00594
:101CF000070706000080404020101008030909066D
:101D000001FFE020202020202020E0050303060022
:101D1000052050880501010600FEF80303030601B3
:101D200005804020050505060000700878887805C4
:101D300007070600008080F0888888F00505050602
:101D4000000070808088700507070600000808788A
:101D5000888888780505050600007088F080700581
:101D60000707060000304840E040404005070706EE
:101D700000FE7088888878087005070706000080D4
:101D800080F0888888880307070601004000C0406B
:101D90004040E00409090601FE1000301010101048
:101DA000906005070706000080808890E090880317
:101DB0000707060100C04040404040E00505050619
:101DC0000000D0A8A8A8A8050505060000B0C8888E
:101DD0008888050505060000708888887005070753
:101DE0000600FEF0888888F080800507070600FE60
:101DF00078888888780808050505060000B0C8803E
:101E0000808005050506000078807008F00507074A
:101E10000600002020F820202018050505060000F7
:101E200088888898680505050600008888885020FD
:101E30000505050600008888A8A8500505050600C8
:101E40000088502050880507070600FE88888850C3
:101E5000204080050505060000F8102040F8030921
:101E6000090601FF20404040804040402001090910
:101E70000602FF80808080808080808003090906C0
:101E800001FF8040404020404040800503030600A1
:101E90000248A890FF1FFFFFFFFFFFFF6000000048
:101EA0000001FF400000000000FF80000000000073
:101EB0007F83CF00000C303F87FF80000C301F86EF
:101EC0007980000C000F8C30C7838C30E78C30CFCA
:101ED000C7CC31F38C30DCECEC33B98C30D86C6C83
:101EE00033198C30D06C0C33198C30D86C0C3319FE
:101EF0008C30DC6C0E3B198C30CF7C079F198C30FA
:101F0000C77C038F19400000000000026000000041
:101F10000000061FFFFFFFFFFFF8000000000000A9
:101F200000000000000000000000000000000000B1
:101F3000000000000000000000000000000C000095
:101F400000000000000C0000000000000012000073
:101F5000000000000023000000000000002100003D
:101F600000000000004C800000000000005E8000C7
:101F700000000000009240000000000000A14000AE
:101F8000000000000121200000000000027F9000FE
:101F900000000000020010000000000007FFF80031
:101FA0000000000004000800000000000800040019
:101FB0000000000008000600000000001000020001
:101FC00000000000301E010000000000207F8100A2
:101FD0000000000041FFE0800000000043FCF080B2
:101FE00000000000873B7840000000018EDBFC60B1
:101FF000000000010FEBCC20000000021FEDB61026
:10200000000000021FDEB6100000000439CD7F087A
:102010000000000436E0FF08000000087EC0BB841A
:10202000000000187F005D86000000107FC0ED8278
:10203000000000203CC07301000000203B337F0102
:10204000000000701BE77E03800000C81DEEDE0468
:10205000C00000880FDEDC04400001240FDF3C09D3
:102060002000012607DBF8192000027203E7F013B5
:102070009000025101FFE02290000489007F80243B
:1020800048000904801E004824000BFE400000DFC9
:10209000F40010004000008002001FFFFFFFFFFF60
:1020A000FE00000000000000000000000000000032
:1020B000000000000000000000001022103C3C0E58
:1020C0001F001022100422110400102210082211F7
:1020D0000400102210083C110400102210102211DC
:1020E000040010221020221104001E1C1E3C3C0E75
:1020F00004000000000000000000000000000000DC
:1021000000000000000000000000000000000000CF
:1021100000000000000000000000000000000000BF
:1021200000000000000000000000000000000000AF
:10213000000000000000000000000000000000009F
:10214000000000000000000000000000000000008F
:10215000000000000000000000060900FE060189E2
:1021600002FE20FFFE07FE06FE000000060007013B
:1021700006060602008080808000800303030601BB
:1021800003A0A0A00507070600FF5050F850F85024
:10219000500509090600FE2070A8A07028A870202C
:1021A0000608080600FF40A8481020485408050704
:1021B000070600FF60909060989068010303060294
:1021C000038080800207070602FF408080808080B5
:1021D000400207070602FF8040404040408005055E
:1021E000050600008850F850880505050600002007
:1021F00020F820200204040602FEC04040800501B1
:1022000001060002F8020202060200C0C00406062F
:1022100006010010102040808004060606010060C0
:10222000909090906003060606010040C040404038
:10223000E00406060601006090102040F004060647
:10224000060100F020601010E005060606000010F0
:10225000305090F810040606060100F080E01010DF
:10226000E00406060601006080E090906004060627
:10227000060100F010102040400406060601006030
:1022800090609090600406060601006090907010C7
:1022900060020505060200C0C000C0C002070706B4
:1022A00002FEC0C000C040408005050506000018C1
:1022B00060806018050303060001F800F8050505B5
:1022C000060000C0300830C0040707060100609017
:1022D00010604000400506060600007090A8B0801F
:1022E00070050606060000205088F8888805060656
:1022F000060000F088F08888F004060606010060F9
:102300009080809060040606060100E09090909016
:10231000E0040606060100F080E08080F004060676
:10232000060100F080E0808080040606060100605F
:102330009080B090600406060601009090F09090A6
:1023400090030606060100E040404040E005060616
:102350000600003810101090600406060601009078
:10236000A0C0A090900406060601008080808080B6
:10237000F005060606000088D8A8A8888804060686
:1023800006010090D0B090909005060606000070FF
:102390008888888870040606060100E09090E08036
:1023A000800407070601FF609090D0B0601004061B
:1023B00006060100E09090E09090040606060100F9
:1023C000609040209060050606060000F82020205E
:1023D000202004060606010090909090906004066C
:1023E00006060100909090F0606005060606000069
:1023F0008888A8A8D88805060606000088502020EE
:102400005088050606060000888850202020040613
:1024100006060100F010204080F0030606060100C9
:10242000E080808080E00406060601008080402075
:102430001010030606060100E020202020E005031E
:10244000030600032050880501010600FEF8020281
:10245000020602048040040404060100709090709B
:102460000406060601008080E09090E00404040663
:102470000100708080700406060601001010709044
:10248000907004040406010060B0C07004060606E3
:102490000100205040E040400406060601FE609026
:1024A000907010600406060601008080E090909015
:1024B0000306060601004000C04040E0030808068D
:1024C00001FE200060202020A04004060606010036
:1024D0008080A0C0A090030606060100C0404040D6
:1024E00040E0050404060000D0A8A88804040406FF
:1024F0000100E09090900404040601006090906058
:102500000406060601FEE09090E0808004060606C0
:1025100001FE709090701010040404060100A0D019
:10252000808004040406010070C030E00406060642
:1025300001004040E0405020040404060100909057
:102540009070040404060100909060600504040685
:10255000000088A8A8500404040601009060609060
:102560000406060601FE9090907090600404040634
:102570000100F02040F003070706010020404080E2
:102580004040200107070602FF8080808080808015
:1025900003070706010080404020404080040202FB
:1025A00006010350A0FFFFFFFFFFFFFFFFFFFFFF3C
:1025B000FFFFFFFFFFFFFFFFFFFFFFFFFFFFFFFF2B
:1025C000FFFFFFFFFFFF00000006000701060606F1
:1025D00002008000808080800406060601FF2070D3
:1025E000A0A070200507070600FF304840F04040DB
:1025F000F8050505060000A8508850A8050606063F
:1026000000008850F820F8200107070602FF8080AC
:1026100080008080800407070601FF708060906062
:1026200010E0030101060105A00607070600007877
:102630008494A494847803050506010160A06000D9
:10264000E00505050600002850A0502804030306F5
:102650000100F01010040101060102F00607070650
:1026600000007884B4A4A48478040101060105F074
:102670000403030601026090600507070600FF20BF
:1026800020F8202000F803050506010140A02040A5
:10269000E0030505060101C0204020C00202020639
:1026A000020440800405050601FF9090B0D080052B
:1026B000060606000078E8E86828280101010602FD
:1026C00002800202020602FE4080030505060101A7
:1026D00040C04040E003050506010140A04000E085
:1026E000050505060000A0502850A00508080600B2
:1026F000FF40C04050703078100508080600FF40C9
:10270000C04050680810380508080600FFC0204087
:1027100030F03078100407070601002000206080A8
:10272000906005070706000040202050708888054B
:10273000070706000010202050708888050707064C
:1027400000002050205070888805070706000028E8
:102750005020507088880507070600005000205060
:102760007088880507070600002050205070888870
:1027700005060606000078A0F0A0A0B80408080628
:1027800001FE6090808090602040040707060100F1
:102790004020F080E080F00407070601002040F0B0
:1027A00080E080F00407070601002050F080E08000
:1027B000F00407070601005000F080E080F00307F6
:1027C000070601008040E0404040E00307070601A3
:1027D000002040E0404040E003070706010040A021
:1027E000E0404040E0030707060100A000E0404051
:1027F00040E00506060600007048E84848700407F7
:102800000706010050A090D0B09090040707060181
:10281000004020609090906004070706010020406F
:10282000609090906004070706010020506090902F
:10283000906004070706010050A06090909060042B
:10284000070706010050006090909060050505069E
:10285000000088502050880408080601FF1070B05E
:10286000B0D0D0E08004070706010040209090908F
:10287000906004070706010020409090909060044B
:10288000070706010020509090909060040707060B
:10289000010050009090909060050707060000101E
:1028A00020885020202004060606010080E0909039
:1028B000E0800406060601006090A0A090A0040736
:1028C0000706010040200070909070040707060181
:1028D000002040007090907004070706010020500F
:1028E000007090907004070706010050A0007090DF
:1028F0009070040606060100500070909070040766
:102900000706010020502070909070050404060016
:102910000070A8B0780406060601FE708080702062
:102920004004070706010040200060B0C0700407A3
:102930000706010020400060B0C0700407070601D0
:102940000020500060B0C070040606060100500070
:1029500060B0C070030707060100804000C040401F
:10296000E0030707060100204000C04040E00307E5
:102970000706010040A000C04040E0030606060133
:1029800000A000C04040E0040707060100306010CE
:102990007090906004070706010050A000E090903E
:1029A0009004070706010040200060909060040733
:1029B00007060100204000609090600407070601B0
:1029C000002050006090906004070706010050A0AE
:1029D0000060909060040606060100500060909030
:1029E000600505050600002000F800200404040628
:1029F000010070B0D0E004070706010040200090FD
:102A0000909070040707060100204000909090709D
:102A100004070706010020500090909070040606FD
:102A20000601005000909090700409090601FE20F4
:102A300040009090907090600408080601FE80802D
:102A4000E09090E080800408080601FE500090901D
:102A5000907090605072696E742066726F6D205332
:102A600044005072696E742066726F6D205344008A
:102A7000022E2E004D61696E00536D6F6F74686990
:102A80006E6700536D6F6F7468696E67005A005A05
:102A9000005900590058005800436F727265637402
:102AA000696F6E00436F7272656374696F6E004D7B
:102AB00061696E0046696C616D656E7400544D43CA
:102AC0002064726976657273004261636B6C617336
:102AD000680053746570732F6D6D004A65726B00EA
:102AE000416363656C65726174696F6E0056656CF5
:102AF0006F6369747900436F6E666967757261749C
:102B0000696F6E004573746570732F6D6D0045734A
:102B1000746570732F6D6D005A73746570732F6DCB
:102B20006D005A73746570732F6D6D005973746501
:102B300070732F6D6D005973746570732F6D6D0018
:102B40005873746570732F6D6D005873746570736E
:102B50002F6D6D00416476616E636564205365740A
:102B600074696E67730056652D6A65726B005665F1
:102B70002D6A65726B00567A2D6A65726B00567A03
:102B80002D6A65726B0056792D6A65726B005679F5
:102B90002D6A65726B0056782D6A65726B005678E7
:102BA0002D6A65726B00416476616E6365642053C3
:102BB000657474696E677300416D617820450041EA
:102BC0006D6178204500416D6178205A00416D614A
:102BD00078205A00416D6178205900416D6178205C
:102BE0005900416D6178205800416D61782058008E
:102BF000412D74726176656C00412D747261766549
:102C00006C00412D7265747261637400412D7265B0
:102C1000747261637400416363656C004163636552
:102C20006C00416476616E636564205365747469F9
:102C30006E6773005654726176206D696E0056544B
:102C4000726176206D696E00566D696E00566D6911
:102C50006E00566D6178204500566D617820450004
:102C6000566D6178205A00566D6178205A00566D75
:102C70006178205900566D6178205900566D617851
:102C8000205800566D6178205800416476616E636B
:102C900065642053657474696E6773004C6F61647A
:102CA000206D6D004C6F6164206D6D00556E6C6F12
:102CB0006164206D6D00556E6C6F6164206D6D00F8
:102CC000416476616E6365204B00416476616E639A
:102CD00065204B00416476616E63656420536574C2
:102CE00074696E67730044697361626C6520737404
:102CF000657070657273004D3834004175746F2DC6
:102D000063616C696272617465004C6576656C2004
:102D1000582041786973004D313137204C65766514
:102D20006C696E67205820417869730A4732380A07
:102D3000473020583136302046393939390A473042
:102D4000205A352046363030300A4739310A4D3264
:102D500031312053300A4D3430300A4D393036206D
:102D60005A3630300A4730205A2D3135204635301A
:102D7000300A4730205A3520463530300A4739303E
:102D80000A4D3430300A4D393036205A3936300A3F
:102D90004D3231312053310A4732380A4D31313703
:102DA000204C6576656C696E6720646F6E652E0ACF
:102DB000004175746F20686F6D6500473238004DB3
:102DC0006F76652061786973004D61696E004578A2
:102DD00074727564657220004175746F20686F6D40
:102DE0006500473238004D6F7665205A004D6F768A
:102DF000652059004D6F76652058004D6F76656DE2
:102E0000656E7400457874727564657220004D6F4C
:102E1000766520302E316D6D004D6F766520316DF9
:102E20006D004D6F76652031306D6D004D6F7665AC
:102E3000206178697300486F74656E6420746F6FE9
:102E400020636F6C6400457874727564657220004D
:102E50004D6F7665205A004D6F76652059004D6F95
:102E600076652058004D6F7665205A004D6F766567
:102E70002059004D6F7665205800576169742066AF
:102E80006F720066696C616D656E74207075726733
:102E9000650000506C6561736520776169742E0070
:102EA000507265737320627574746F6E00746F2056
:102EB000726573756D65207072696E740057616913
:102EC0007420666F720066696C616D656E74206C4B
:102ED0006F616400496E736572742066696C616D20
:102EE000656E7400616E6420707265737320627524
:102EF00074746F6E00746F20636F6E74696E7565A5
:102F000000507265737320627574746F6E00746F15
:102F10002068656174206E6F7A7A6C65004E6F7AF6
:102F20007A6C652068656174696E6700506C6561D4
:102F3000736520776169742E2E2E005761697420A5
:102F4000666F720066696C616D656E7420756E6C7B
:102F50006F6164005761697420666F720066696C06
:102F6000616D656E74206368616E676500746F20C3
:102F70007374617274005061726B696E672E2E2ECD
:102F8000004368616E67696E672046696C616D65B4
:102F90006E7400554E4C4F41442046494C414D45BE
:102FA0004E54004C4F41442046494C414D454E54EF
:102FB0000020204E6F7A7A6C653A20002000456E22
:102FC000642066696C616D656E74206368616E670C
:102FD00065005075726765206D6F7265000043680B
:102FE000616E67652066696C616D656E7400556E13
:102FF0006C6F61642066696C616D656E74004C6F06
:1030000061642066696C616D656E74004D363030A8
:1030100020423020542564004D373032203B256457
:10302000004D37303220542564004D373031205464
:103030002564005072656865617420437573746F10
:103040006D005072656865617420437573746F6DAF
:10305000005072656865617420414253005072658A
:103060006865617420504C41004261636B004E6F93
:103070002053442063617264005072696E7420664C
:10308000726F6D2053440041626F757420507269F5
:103090006E746572004368616E67652066696C6175
:1030A0006D656E74004368616E67652066696C616A
:1030B0006D656E74004D36303020423000436F6EC7
:1030C00066696775726174696F6E0054656D7065CD
:1030D000726174757265004D6F76656D656E740012
:1030E000526573756D65207072696E740054756EEB
:1030F000650053746F70207072696E740050617552
:103100007365207072696E7400496E666F20736318
:103110007265656E005072696E74657220537461D9
:103120007473004669726D776172652056657273BB
:10313000696F6E004D61696E0053746F702070721C
:10314000696E74004D61696E005072696E74206121
:10315000626F72746564004D3234004D3235205018
:103160000A4D32340050726F6265205A204F6666F5
:10317000736574004261627973746570205900420E
:1031800061627973746570205800466C6F770046F1
:103190006C6F770046616E207370656564004661F0
:1031A0006E2073706565640042656400426564006A
:1031B0004E6F7A7A6C65004E6F7A7A6C6500537048
:1031C000656564005370656564004D61696E004219
:1031D0006162797374657020590042616279737419
:1031E00065702058002569730025696D2025697375
:1031F000002569682025696D2025697300256964AB
:10320000202569682025696D202569730025697965
:1032100020256964202569682025696D202569734A
:10322000003E2000457874727564656420746F7484
:10323000616C3A00256C642E25696D003E20004CBF
:103240006F6E67657374206A6F622074696D653A8A
:10325000003E2000546F74616C207072696E74209F
:1032600074696D653A00436F6D706C657465643A9E
:1032700020005072696E7420436F756E743A20009E
:10328000436F6F6C646F776E0046616E207370657C
:1032900065640046616E2073706565640042656414
:1032A00000426564004E6F7A7A6C65004E6F7A7AE0
:1032B0006C65004D61696E00526573746F726520B4
:1032C0006661696C73616665004C6F61642073654B
:1032D0007474696E67730053746F726520736574DC
:1032E00074696E67730050726F6265205A204F6672
:1032F0006673657400416476616E6365642053652E
:103300007474696E6773004D61696E0050726F620C
:1033100065205A204F66667365740053746570703B
:10332000696E67206D6F64650053656E736F726CB4
:1033300065737320686F6D696E67004879627269A2
:1033400064207468726573686F6C64004472697697
:1033500065722063757272656E7400436F6E74726D
:103360006F6C004530004F6666004F6E00453000C0
:103370005A004F6666004F6E005A0059004F66664D
:10338000004F6E00590058004F6666004F6E00589F
:1033900000544D43206472697665727300537465FE
:1033A000616C746843686F7020656E61626C6564FF
:1033B000005900590058005800544D432064726968
:1033C00076657273004530004530005A005A005946
:1033D00000590058005800544D43206472697665C6
:1033E0007273004530004530005A005A00590059A8
:1033F0000058005800544D4320647269766572731A
:10340000004D696E6920322072656164792E00502A
:1034100072696E74696E672E2E2E005072696E741A
:103420002070617573656400436172642072656D1C
:103430006F766564004361726420696E73657274AF
:103440006564004D33310043616E6E6F7420656EAC
:10345000746572207375626469723A20002E0A00E6
:103460006F70656E206661696C65642C2046696CBE
:10347000653A20006175746F25632E67006572726E
:103480006F722077726974696E6720746F20666945
:103490006C650A004E6F74205344207072696E741C
:1034A000696E670A005344207072696E74696E67B2
:1034B000206279746520002E0A0044656C65746989
:1034C0006F6E206661696C65642C2046696C653A94
:1034D000200046696C652064656C657465643A001B
:1034E00057726974696E6720746F2066696C653AFB
:1034F00020002E0A006F70656E206661696C65643D
:103500002C2046696C653A20002E0A006F70656EAB
:10351000206661696C65642C2046696C653A200000
:1035200046696C652073656C65637465640A002088
:1035300053697A653A200046696C65206F70656E44
:1035400065643A20002066696C653A200066726501
:10355000736800646F696E67004E6F772000454E98
:103560004420535542524F5554494E450A0022209B
:10357000706F73002220706172656E743A2200537E
:103580005542524F5554494E452043414C4C2074AE
:1035900061726765743A2200747279696E6720748B
:1035A0006F2063616C6C207375622D67636F646557
:1035B0002066696C6573207769746820746F6F206A
:1035C0006D616E79206C6576656C732E204D415867
:1035D000206C6576656C2069733A310A004D32348F
:1035E000004D323320257300534420636172642000
:1035F0006F6B0A006F70656E526F6F742066616941
:103600006C65640A00766F6C756D652E696E697401
:10361000206661696C65640A00534420696E6974B0
:10362000206661696C0A00286E6F2066696C6529E6
:103630000043616E6E6F74206F70656E20737562EB
:1036400064697220007C3C3E5E2B3D3F2F5B5D3BFE
:103650002C2A225C004F4646004F4E006563686F7F
:103660003A004572726F723A004572726F7220773B
:10367000726974696E6720746F20454550524F4DD2
:10368000210A00507265737320627574746F6E2026
:10369000286F72204D3130382920746F20686561A1
:1036A00074206E6F7A7A6C650A00507265737320AD
:1036B000627574746F6E20286F72204D3130382916
:1036C00020746F20726573756D650A00496E7365AD
:1036D00072742066696C616D656E7420616E642021
:1036E000707265737320627574746F6E20286F72C8
:1036F000204D313038290A004D3630303A20546F91
:103700006F20636F6C6400486F74656E6420746F23
:103710006F20636F6C640A00486F74656E64207478
:103720006F6F20636F6C640A00496E73657274205A
:1037300066696C616D656E7420616E64207072657F
:10374000737320627574746F6E20286F72204D3110
:103750003038290A004C4F570048494748004F4B22
:10376000004572726F723A20416C6C200020636FCA
:103770006E6E656374696F6E2E2E2E200054657315
:1037800074696E6720004C4F570048494748004F06
:103790004B004572726F723A20416C6C20002063BE
:1037A0006F6E6E656374696F6E2E2E2E20005465E9
:1037B0007374696E6720004C4F57004849474800B2
:1037C0004F4B004572726F723A20416C6C200020A2
:1037D000636F6E6E656374696F6E2E2E2E200054BB
:1037E000657374696E6720004C4F5700484947481D
:1037F000004F4B004572726F723A20416C6C200092
:1038000020636F6E6E656374696F6E2E2E2E2000BE
:1038100054657374696E672000544D4320434F4EC6
:103820004E454354494F4E204552524F5200445248
:10383000565F535441545553090050574D5F5343FD
:10384000414C45090050574D434F4E460900434FE8
:103850004F4C434F4E46090043484F50434F4E464E
:103860000900544849474809090054434F4F4C54F4
:1038700048525309005450574D544852530900546C
:103880005354455009090054504F574552444F571F
:103890004E0900494F494E09090047535441540904
:1038A000090049484F4C445F4952554E090047436F
:1038B0004F4E4609090009000920426164207265E3
:1038C00073706F6E73652100092042616420726518
:1038D00073706F6E73652100092042616420726508
:1038E00073706F6E736521000920426164207265F8
:1038F00073706F6E73652100303D2E3332350031A9
:103900003D2E31380066616C736500747275650018
:1039100066616C73650074727565006D6178002F67
:103920003331002F3331002F33310066616C736502
:10393000007472756500303D2E33323500313D2EF6
:1039400031380066616C736500747275650066617C
:103950006C73650074727565006D6178002F33318A
:10396000002F3331002F33310066616C73650074B2
:1039700072756500303D2E33323500313D2E3138C1
:103980000066616C736500747275650066616C73C6
:10399000650074727565006D6178002F3331002FFA
:1039A0003331002F33310066616C736500747275BA
:1039B000650066616C7365007472756500303D2E3C
:1039C00033323500313D2E31380066616C7365004D
:1039D000747275650066616C73650074727565005C
:1039E0006D6178002F3331002F3331002F333100D8
:1039F00066616C7365007472756500447269766502
:103A000072207265676973746572733A0A006F7425
:103A100009006F74707709007332676109007332AF
:103A2000676209006F6C6109006F6C620900737452
:103A3000737409006673616374697665090073675E
:103A40005F726573756C7409007374616C6C677573
:103A50006172640900445256535441545553005303
:103A600074616C6C67756172642074687273002D88
:103A7000737461727409006879737465726573692F
:103A8000730A2D656E640900626C616E6B20746947
:103A90006D65006F66662074696D6509004F54207E
:103AA0007072657761726E206861730A6265656E17
:103AB00020747269676765726564004F5420707284
:103AC000657761726E005B6D6D2F735D09007077B5
:103AD0006D0A7468726573686F6C6409007473743E
:103AE000657009006D7374657073090073746561A6
:103AF0006C746843686F70007673656E7365090057
:103B000050574D207363616C6500435320616374AB
:103B100075616C0900486F6C642063757272656E24
:103B2000740052756E2063757272656E74004D413B
:103B3000582063757272656E7400524D5320637520
:103B40007272656E74005365742063757272656E6F
:103B50007400456E61626C656409000900617869F2
:103B6000733A70776D5F7363616C652F6375727202
:103B7000656E745F7363616C652F6D6563685F6C00
:103B80006F61647C666C6167737C7761726E636F72
:103B9000756E740A006D41290A00206472697665A9
:103BA00072206F76657274656D706572617475727E
:103BB00065207761726E696E67212028003A2000C7
:103BC0002063757272656E742064656372656173DB
:103BD000656420746F20006D41290A0020647269B9
:103BE000766572206F76657274656D70657261744A
:103BF000757265207761726E696E67212028003AC0
:103C000020002063757272656E742064656372654E
:103C10006173656420746F20006D41290A0020647F
:103C20007269766572206F76657274656D70657203
:103C30006174757265207761726E696E67212028E4
:103C4000003A20002063757272656E7420646563AB
:103C500072656173656420746F200025756420258A
:103C60003032753A25303275006D41290A002064E2
:103C70007269766572206F76657274656D706572B3
:103C80006174757265207761726E696E6721202894
:103C9000003A20002063757272656E74206465635B
:103CA00072656173656420746F2000447269766583
:103CB00072206572726F7200636F696C2073686F37
:103CC000727420636972637569740A006F76657235
:103CD00074656D70657261747572650A0020647236
:103CE00069766572206572726F72206465746563AF
:103CF0007465643A2030780063616E63656C0072AD
:103D00006573756D656400726573756D65007061CE
:103D10007573656400706F7765726F6666002F2F2C
:103D2000616374696F6E3A0020573A0020573A0079
:103D3000457874727564657220436F6F6C696E6745
:103D40002E2E2E0045787472756465722048656168
:103D500074696E672E2E2E00202F002042403A00FC
:103D600020403A00546865726D616C2052756E6136
:103D700077617900453120544845524D414C2052DD
:103D8000554E415741590042656400202D20496E2F
:103D900076616C6964206578747275646572206EF2
:103DA000756D62657220210A0048656174696E67ED
:103DB000206661696C6564004265640048656174F1
:103DC000696E67206661696C6564004531204865ED
:103DD0006174696E67206661696C6564004D494E67
:103DE00054454D502074726967676572656400457B
:103DF00031204572723A204D494E54454D50004293
:103E00006564004D415854454D5020747269676790
:103E100065726564004531204572723A204D415803
:103E200054454D500042656400626564002C207367
:103E3000797374656D2073746F70706564212048A8
:103E400065617465725F49443A2000236465666960
:103E50006E652044454641554C545F004B6420003C
:103E60004B6920004B70200000626564005049449B
:103E7000204175746F74756E652066696E6973682C
:103E80006564212050757420746865206C617374BA
:103E9000204B702C204B6920616E64204B642063A2
:103EA0006F6E7374616E74732066726F6D206265DD
:103EB0006C6F7720696E746F20436F6E66696775EB
:103EC000726174696F6E2E680A0050494420417512
:103ED000746F74756E65206661696C656421207409
:103EE000696D656F75740A00546865726D616C2048
:103EF00052756E6177617900453120544845524DC5
:103F0000414C2052554E415741590042656400488A
:103F1000656174696E67206661696C65640045312E
:103F20002048656174696E67206661696C6564002C
:103F300042656400504944204175746F74756E6524
:103F4000206661696C6564212054656D70657261DD
:103F50007475726520746F6F20686967680A002045
:103F60004B643A2000204B693A2000204B703A20E5
:103F7000000A20436C617373696320504944200A2E
:103F8000002054753A2000204B753A2000206D61C6
:103F9000783A2000206D696E3A200020643A2000B3
:103FA00020626961733A2000504944204175746F62
:103FB00074756E652073746172740A0050494420F0
:103FC0004175746F74756E65206661696C656421F6
:103FD0002054656D706572617475726520746F6FC1
:103FE00020686967680A001000AD0330016A01505B
:103FF000022B0170030A019004F500B005E500D022
:1040000006D800F007CE001009C500300ABE0050E7
:104010000BB700700CB100900DAB00B00EA600D035
:104020000FA200F0109D001012990030139500505F
:1040300014920070158E0090168B00B0178700D078
:10404000188400F0198100101B7E00301C7B00508A
:104050001D7900701E7600901F7300B0207000D094
:10406000216E00F0226B001024690030256600509C
:104070002663007027610090285E00B0295C00D0A4
:104080002A5900F02B5600102D5400302E510050AC
:104090002F4E0070304B0090314800B0324500D0B8
:1040A000334200F0343E0010363B003037370050CA
:1040B00038330070392E00903A2900B03B2300D0ED
:1040C0003C1B00F03D1100103F0100F03F000010CC
:1040D00000C90210012C014001220170011801B039
:1040E000010E01F00104015002FA00B002F00030AC
:1040F00003E600D003DC009004D2007005C800A0E5
:1041000006BE000008B400B009AA00D00BA00060F1
:104110000E960060118C000015820020197800C0F6
:104120001D6E00A0226400B0275A00902C500000A1
:10413000314600E0343C0010383200903A280060EC
:104140003C1E00A03D1400803E0A00203F00006F8E
:1041500070656E00545249474745524544003A2025
:10416000007A5F6D6178007A5F6D696E00795F6DCE
:10417000617800785F6D696E005265706F72746966
:104180006E6720656E6473746F70207374617475EC
:10419000730A00456E6473746F7073202563202565
:1041A0006320256320256300205A3A0020593A00F5
:1041B00020583A00656E6473746F70732068697478
:1041C0003A2000486F6D696E67206661696C6564AE
:1041D000000A53746174733A2046696C616D656EB0
:1041E0007420757365643A20002C204C6F6E6765EF
:1041F0007374206A6F623A2000546F74616C20748B
:10420000696D653A200053746174733A20002C2064
:104210004661696C65643A20002C2046696E6973BA
:104220006865643A20005072696E74733A200053D6
:10423000746174733A2000496E76616C696420651C
:10424000787472756465720A00205A3A0020593AEF
:104250000020436F756E7420583A00C23100001C74
:10426000260000F4190000D80F0000EB080000C081
:10427000040000750200004001000024F4D4305016
:10428000C38E20C2A24017828B7011127A910D81C9
:104290006CD90AA861E108C7586607615143061E38
:1042A0004B5D05C145A7041A411104093D980371EE
:1042B0003931034036DB0265339102D43054028039
:1042C0002E1D02632CEE01752AC501B028A0011035
:1042D0002781018F2564012B244B01E0223401AC9E
:1042E000211F018D200D01801FFC00841EED009711
:1042F0001DDF00B81CD200E61BC600201BBC0064FA
:104300001AB200B219A8000A19A0006A189900D1BF
:1043100017910040178B00B516840031167E00B34C
:104320001579003A157300C7146F0058146A00EE2F
:104330001366008813630025135E00C7125B006CD0
:1043400012570015125400C111510070114F002175
:10435000114B00D61049008D104700461044000252
:10436000104200C00F4000800F3E00420F3C00068C
:104370000F3B00CB0E3800930E37005C0E35002744
:104380000E3400F30D3200C10D3100900D3000608D
:104390000D2E00320D2D00050D2C00D90C2B00AE7A
:1043A0000C2900850C29005C0C2700350C27000E19
:1043B0000C2600E80B2400C40B2400A00B23007D76
:1043C0000B23005A0B2100390B2100180B2000F899
:1043D0000A1F00D90A1E00BB0A1E009D0A1D00808C
:1043E0000A1D00630A1C00470A1B002C0A1B00114F
:1043F0000A1A00F7091A00DD091900C4091900ABEF
:10440000091900920917007B091800630917004C6D
:1044100009160036091600200916000A091500F5CC
:10442000081500E0081400CC081400B8081400A413
:10443000081400900813007D0812006B0813005840
:104440000812004608120034081100230811001257
:1044500008110001081100F0071000E0071000D05B
:10446000071000C0071000B0070F00A1071000914F
:10447000070E0083070F0074070F0065070E005733
:10448000070E0049070E003B070D002E070E002007
:10449000070D0013070D0006070D00F9060C00EDCF
:1044A000060D00E0060C00D4060C00C8060C00BC8B
:1044B000060C00B0060C00A4060B0099060C008D3B
:1044C000060B0082060B0077060B006C060B0061E2
:1044D000060A0057060B004C060A0042060A00387E
:1044E000060A002E060A0024060A001A060A001010
:1044F00006090007060A00FD050900F4050900EB9E
:10450000050900E2050900D9050900D0050900C721
:10451000050900BE050900B5050800AD050800A5A0
:104520000509009C050800940508008C0508008416
:104530000508007C050800740508006C0507006587
:104540000508005D050700560508004E05070047F1
:104550000507004005080038050700310507002A57
:10456000050700230507001C050600160507000FB8
:104570000507000805060002050700FB040600F514
:10458000040700EE040600E8040600E2040700DB6E
:10459000040600D5040600CF040600C9040600C3C3
:1045A000040600BD040600B7040600B1040500AC13
:1045B000040600A6040600A00405009B040600955E
:1045C000040500900406008A0405008504050080A7
:1045D0000406007A04050075040500700405006BEC
:1045E00004050066040500610405005C040500572D
:1045F000040500520405004D04050048040500436D
:104600000405003E0404003A0405003504050030AA
:104610000404002C04050027040400230405001EE4
:104620000404001A04040016040500110404000D1B
:10463000040400090405000404040000040400FC50
:10464000030400F8030400F4030400F0030400EC86
:10465000030400E8030400E4030400E0030400DCB6
:10466000030400D8030400D4030400D0030400CCE6
:10467000030400C8030300C503030024F404D92085
:104680001BC40C5C0E9804C4095F0265077101F439
:1046900005F900FB04B30048048700C10369005812
:1046A00003550003034500BE023A00840231005363
:1046B000022A002902250004022000E4011C00C88F
:1046C000011900AF01170098011400840113007153
:1046D0000110006101100051010E0043010D003670
:1046E000010B002B010B0020010B00150109000C30
:1046F00001090003010800FB000800F3000800EBBB
:10470000000700E4000600DE000600D8000600D224
:10471000000600CC000500C7000500C2000500BD72
:10472000000400B9000400B5000400B1000400ADAD
:10473000000400A9000400A5000300A20003009FDC
:104740000004009B00030098000300950002009302
:10475000000300900003008D0002008B000300881E
:104760000002008600020084000300810002007F36
:104770000002007D0002007B000200790002007749
:104780000001007600020074000200720001007156
:104790000002006F0002006D0001006C0002006A60
:1047A0000001006900020067000100660001006569
:1047B000000100640002006200010061000100606D
:1047C0000001005F0002005D0001005C0001005B71
:1047D0000001005A00010059000100580001005773
:1047E0000001005600010055000100540001005373
:1047F0000000005300010052000100510001005070
:104800000001004F0001004E0000004E0001004D6D
:104810000001004C0001004B0000004B0001004A69
:104820000001004900010048000000480001004765
:104830000001004600000046000100450000004560
:104840000001004400010043000000430001004259
:104850000000004200010041000000410001004052
:104860000001003F0000003F0001003E0000003E4C
:104870000001003D0000003D0001003C0000003C44
:104880000000003C0001003B0000003B0001003A3A
:104890000000003A00010039000000390001003832
:1048A0000000003800000038000100370000003729
:1048B000000100360000003600000036000100351F
:1048C0000000003500000035000100340000003415
:1048D000000000340001003300000033000000330A
:1048E00000010032000000320000003200010031FF
:1048F00000000031000000310001003000000030F5
:10490000000000300001002F0000002F0000002FE9
:104910000000002F0001002E0000002E0000002EDD
:104920000001002D0000002D0000002D0000002DD2
:104930000001002C0000002C0000002C0000002CC6
:104940000001002B0000002B0000002B0000002BBA
:104950000001002A0000002A0000002A0000002AAE
:1049600000010029000000290000002900000029A2
:104970000000002900010028000000280000002895
:104980000000002800000028000100270000002788
:10499000000000270000002700000027000100267B
:1049A000000000260000002600000026000000266F
:1049B0000001002500000025000000250000002562
:1049C0000000002500000025000100240000002454
:1049D0000000002400000024000000240001002347
:1049E000000000230000002300000023000000233B
:1049F000000000230000002300010022000000222C
:104A0000000000220000002200000022000000221E
:104A10000001002100000021000000210000002111
:104A20000000002100000021000000210001002002
:104A300000000020000000200000002000000020F6
:104A40000000002000000020000000200001001FE6
:104A50000000001F0000001F0000001F0000001FDA
:104A60000000001F0000001F0001001E0000001ECB
:104A70000000001E0000001E00000020204D363007
:104A800033200020204D3931340020204D3931337E
:104A90000020204D393036003A0A0020286D6D295B
:104AA000002055004C0046696C616D656E74206C89
:104AB0006F61642F756E6C6F6164206C656E6774D6
:104AC00068733A0A0020204D393030204B004C6981
:104AD0006E65617220416476616E63653A0A0054C6
:104AE00030204500205A00205900205800447269A7
:104AF000766572207374657070696E67206D6F647F
:104B0000653A0A00205900205800544D4332313391
:104B100030205374616C6C477561726420746872E4
:104B20006573686F6C643A0A002054302045002099
:104B30005A00205900205800487962726964205454
:104B400068726573686F6C643A0A002054302045BF
:104B500000205A0020590020580053746570706579
:104B600072206472697665722063757272656E7404
:104B70003A0A0020204D383531205A005A2D507203
:104B80006F6265204F66667365740020440020499B
:104B90000020204D333034205000204400204900B4
:104BA00020204D333031205000504944207365742B
:104BB00074696E67733A0A0020460020420020485C
:104BC0000020204D3134352053004D6174657269E9
:104BD000616C2068656174757020706172616D65CB
:104BE000746572733A0A0020204D3432302053002D
:104BF0004175746F20426564204C6576656C696E02
:104C0000673A0A00204500205A0020590020580029
:104C100020540020530020204D3230352042002007
:104C2000453C6D61785F655F6A65726B3E00205838
:104C30003C6D61785F785F6A65726B3E20593C6DB0
:104C400061785F795F6A65726B3E205A3C6D61786E
:104C50005F7A5F6A65726B3E00416476616E636580
:104C6000643A20423C6D696E5F7365676D656E7472
:104C70005F74696D655F75733E20533C6D696E5F4F
:104C800066656564726174653E20543C6D696E5F53
:104C900074726176656C5F66656564726174653EA9
:104CA0000020540020520020204D3230342050008B
:104CB000416363656C65726174696F6E2028756EFF
:104CC0006974732F7332293A20503C7072696E7484
:104CD0005F616363656C3E20523C72657472616310
:104CE000745F616363656C3E20543C7472617665E9
:104CF0006C5F616363656C3E0A00204500205A00CA
:104D000020590020204D3230312058004D61786903
:104D10006D756D20416363656C65726174696F6E5A
:104D20002028756E6974732F7332293A0A00204562
:104D300000205A0020590020204D323033205800E6
:104D40004D6178696D756D20666565647261746525
:104D5000732028756E6974732F73293A0A0053748F
:104D60006570732070657220756E69743A0A002050
:104D7000204D3134392043203B20556E6974732017
:104D8000696E2043656C736975730A002020473291
:104D900031202020203B20556E69747320696E20DD
:104DA0006D6D0020204D3536392053310048617239
:104DB00064636F6465642044656661756C74205338
:104DC000657474696E6773204C6F616465640A0072
:104DD0002823000028230000C8000000E80300008A
:104DE00000009643000096430000964300002042D6
:104DF0000000C8420000C842000048430000D243FF
:104E0000290A002062797465733B20637263200075
:104E10002073746F7265642073657474696E677350
:104E200020726574726965766564202800202863A5
:104E3000616C63756C6174656429210A0020213DF1
:104E40002000454550524F4D20435243206D697319
:104E50006D61746368202D202873746F72656429F6
:104E600020002053697A653A2000496E6465783ADB
:104E70002000204D61726C696E3D563634290A005F
:104E8000454550524F4D2076657273696F6E206DA7
:104E900069736D617463682028454550524F4D3DDC
:104EA00000290A002062797465733B2063726320D5
:104EB0000053657474696E67732053746F72656410
:104EC0002028000A003B20454550524F4D20496E96
:104ED0006465783A20005570646174696E67207A61
:104EE0006F666673657420696E20454550524F4D5C
:104EF0003A2000454550524F4D20646174617369FA
:104F00007A65206572726F722E0A0050726F626944
:104F10006E67206661696C65640A0050726F626931
:104F20006E67206661696C6564005761726E696EB8
:104F3000673A20486F6D696E672042756D70204436
:104F4000697669736F72203C20310A0002020448BE
:104F50006F6D6520257325732573206669727374E0
:104F6000002066697273740A00486F6D6520002026
:104F7000746F6F206C6F6E672065787472757369DB
:104F80006F6E2070726576656E7465640A002063CA
:104F90006F6C6420657874727573696F6E207072BF
:104FA0006576656E7465640A0020453A00205A3AB9
:104FB0000020593A00583A00000048420000484298
:104FC00000002042FF01010000000000000000007E
:104FD000000040000030430000454300003743001C
:104FE0000040C0000040430000374300002D430054
:104FF00000404300003743000040C00000A0C00054
:1050000000000020746F6F206C6F6E6720657874ED
:10501000727573696F6E2070726576656E74656403
:105020000A0020636F6C6420657874727573696F11
:105030006E2070726576656E7465640A00627573C1
:10504000793A2070617573656420666F7220696EAD
:105050007075740A00627573793A207061757365B2
:105060006420666F7220757365720A0062757379C9
:105070003A2070726F63657373696E670A004D3111
:1050800031372050726F6265207375636365737387
:1050900066756C0A0020496E76616C6964206578DB
:1050A0007472756465722000205A3A200020593AC3
:1050B000200042656420583A200050726F626520DB
:1050C0005A204F66667365743A20003F5A206F7508
:1050D00074206F662072616E676520282D322074FF
:1050E0006F2035290A004D31343520533C696E64F8
:1050F00065783E206F7574206F662072616E6765FB
:105100002028302D31290A00436C69636B20746FAD
:1051100020726573756D652E2E2E00220A00556E65
:105120006B6E6F776E20636F6D6D616E643A2022D7
:1051300000454550524F4D204F4B0A004E6F206D99
:105140006F76652E004543484F00494E464F004557
:1051500052524F52530044525952554E00434F4DF4
:105160004D554E49434154494F4E006F66660045C8
:10517000514A514F5156515D5144454255473A00AD
:105180004C756C7A426F74204D696E692032204FE5
:1051900046462E00205A00205900580020204D611C
:1051A000783A2000205A00205900580020204D69EC
:1051B0006E3A2000536F667420656E6473746F706E
:1051C000733A20005072696E742074696D653A20DC
:1051D000004D3131332053002F2F20004361703AAE
:1051E000004348414D4245525F54454D5045524160
:1051F00054555245004D4F54494F4E5F4D4F444515
:105200005300544845524D414C5F50524F54454312
:1052100054494F4E004155544F5245504F52545FE0
:1052200053445F5354415455530050524F4D5054C2
:105230005F535550504F525400454D455247454ECF
:1052400043595F50415253455200434153455F4CCF
:10525000494748545F4252494748544E45535300CA
:10526000544F47474C455F4C494748545300534FB0
:105270004654574152455F504F5745520042554999
:105280004C445F50455243454E54004C4556454CA6
:10529000494E475F44415441005A5F50524F424586
:1052A000004155544F4C4556454C005052494E54C0
:1052B0005F4A4F420050524F4752455353004155A9
:1052C000544F5245504F52545F54454D5000564F25
:1052D0004C554D455452494300454550524F4D00A1
:1052E00042494E4152595F46494C455F5452414EE6
:1052F000534645520053455249414C5F584F4E5F0B
:10530000584F4646004649524D574152455F4E411F
:105310004D453A4D61726C696E20204649524D5799
:105320004152455F56455253494F4E3A322E302E28
:10533000302E3130352045585452554445525F5433
:105340005950453A536D616C6C4C617965722053CC
:105350004F555243455F434F44455F55524C3A6861
:10536000747470733A2F2F636F64652E616C65706F
:10537000686F626A656374732E636F6D2F6469660C
:10538000667573696F6E2F4D41524C494E205052D5
:105390004F544F434F4C5F56455253494F4E3A314D
:1053A0002E30204D414348494E455F545950453AAF
:1053B0004C756C7A426F74204D696E6920322045BD
:1053C000585452554445525F434F554E543A31203C
:1053D000555549443A65353530323431312D6434D0
:1053E00036642D343231642D626133612D61323087
:1053F0003132366437393330660A0020284E6F74F4
:1054000020796574206D656173757265642900206B
:105410002041766572616765206D6561737572659F
:1054200064206261636B6C61736820286D6D293A3A
:10543000002020536D6F6F7468696E6720286D6D52
:10544000293A202020202020202020202020202039
:10545000202020530020204261636B6C6173682020
:1054600044697374616E636520286D6D293A20204C
:105470002020202020200020202020202846312EFF
:1054800030203D2066756C6C2C2046302E30203D3F
:10549000206E6F6E65290A002020436F727265636B
:1054A00074696F6E20416D6F756E742F466164650F
:1054B0002D6F75743A2020202020460061637469A6
:1054C00076653A0A00696E004261636B6C617368CD
:1054D00020636F7272656374696F6E206973200058
:1054E000205A0020506F736974696F6E616C20459B
:1054F00072726F723A0A004E6F7A7A6C6520546944
:1055000070204F757465722044696D656E73696FA4
:105510006E733A0A002020546F703A200020204613
:10552000726F6E743A200020204C6566743A200039
:105530004261636B6C6173683A0A00205A004365EC
:105540006E7465723A0A00202046726F6E743A20BB
:105550000020204C6566743A20002020546F703A79
:10556000200053696465733A0A00426564204C6503
:1055700076656C696E6720004661696C65642074AD
:105580006F20656E61626C6520426564204C6576B3
:10559000656C696E670A00426564204C6576656CCF
:1055A00020436F7272656374696F6E204D6174720F
:1055B00069783A000A0A426564204C6576656C2079
:1055C000436F7272656374696F6E204D61747269A6
:1055D000783A00202B000A436F7272656374656429
:1055E00020426564204865696768742076732E20C0
:1055F00042656420546F706F6C6F67793A0A0020BF
:105600002B000A4265642048656967687420546FFE
:10561000706F6772617068793A0A2020202B2D2DF7
:105620002D204241434B202D2D2B0A2020207C2071
:10563000202020202020202020207C0A204C207C9C
:1056400020202020282B29202020207C20520A20C6
:1056500045207C20202020202020202020207C206D
:10566000490A2046207C20282D29204E20282B293D
:10567000207C20470A2054207C202020202020202D
:10568000202020207C20480A2020207C2020202050
:10569000282D29202020207C20540A2020207C2016
:1056A000202020202020202020207C0A2020204F85
:1056B0002D2D2046524F4E54202D2D2B0A202830C0
:1056C0002C30290A003474682070726F6265207073
:1056D0006F696E742C2064697374616E63652066F3
:1056E000726F6D20706C616E653A20002028445204
:1056F0005952554E2900473239204175746F204266
:105700006564204C6576656C696E67003F20284CA7
:105710002C522C462C4229206F7574206F66206213
:105720006F756E64732E0A003F50726F6265207051
:105730006F696E74732028592920697320696D7010
:105740006C61757369626C652028322D32292E0ACE
:10575000003F50726F626520706F696E747320280D
:10576000582920697320696D706C61757369626C6A
:10577000652028322D32292E0A003F2856296572CD
:10578000626F7365206C6576656C20697320696D46
:10579000706C61757369626C652028302D34292E18
:1057A0000A0043757272656E742066696C653A20F2
:1057B00000456E642066696C65206C6973740A002C
:1057C000426567696E2066696C65206C6973740A4E
:1057D00000416476616E6365204B3D003F4B20764F
:1057E000616C7565206F7574206F662072616E67DD
:1057F000652028302D3130292E0A004D31313720D7
:10580000486F7420456E642048656174696E672E28
:105810002E2E0A4D31303420533137302054300A87
:10582000473238204F310A473120593235205A311A
:10583000302046353030300A4D3130392052313742
:10584000302054300A4D3131372052657769706904
:105850006E67206E6F7A7A6C650A54300A47312081
:1058600058343520593137342046353030300A47E6
:1058700031205A310A4D31303920523137300A4700
:1058800031205834352059313734204634303030C7
:105890000A473120583435205931373420463430C6
:1058A00030300A47312058343520593137342046BA
:1058B000343030300A4731205834352059313734AC
:1058C0002046343030300A473120583435205931A1
:1058D00037342046343030300A47312058343520B0
:1058E000593137342046343030300A47312058346B
:1058F0003520593137342046343030300A47312092
:1059000058343520593137342046343030300A4746
:105910003120583435205931373420463430303036
:105920000A47312058343520593137342046343035
:1059300030300A4731205834352059313734204629
:10594000343030300A47312058343520593137341B
:105950002046343030300A4731205A31350A4D3133
:1059600030362053323535200A4730205830205900
:10597000300A4D31303920523136302054300A4D02
:105980003130370A007370726561644379636C6506
:1059900000737465616C746843686F700020647292
:1059A00069766572206D6F64653A0900737072657F
:1059B00061644379636C6500737465616C746843FA
:1059C000686F700020647269766572206D6F64651F
:1059D0003A09007370726561644379636C650073A2
:1059E0007465616C746843686F70002064726976D6
:1059F0006572206D6F64653A090073707265616449
:105A00004379636C6500737465616C746843686F97
:105A1000700020647269766572206D6F64653A0962
:105A20000020686F6D696E672073656E73697469B5
:105A3000766974793A200020686F6D696E6720730B
:105A4000656E73697469766974793A20002073749D
:105A500065616C746843686F70206D617820737045
:105A60006565643A200020737465616C74684368EE
:105A70006F70206D61782073706565643A20002036
:105A8000737465616C746843686F70206D61782011
:105A900073706565643A200020737465616C746886
:105AA00043686F70206D61782073706565643A207B
:105AB00000207072657761726E20666C616720638A
:105AC0006C65617265640A00207072657761726E40
:105AD00020666C616720636C65617265640A0020F2
:105AE0007072657761726E20666C616720636C65A9
:105AF000617265640A00207072657761726E20665B
:105B00006C616720636C65617265640A0066616C34
:105B100073650074727565002074656D70657261DF
:105B200074757265207072657761726E2074726927
:105B30006767657265643A200066616C736500741E
:105B4000727565002074656D70657261747572653B
:105B5000207072657761726E207472696767657212
:105B600065643A200066616C736500747275650047
:105B70002074656D706572617475726520707265F0
:105B80007761726E207472696767657265643A2026
:105B90000066616C73650074727565002074656DD4
:105BA0007065726174757265207072657761726E6E
:105BB000207472696767657265643A2000206472B8
:105BC000697665722063757272656E743A20002082
:105BD0006472697665722063757272656E743A20BC
:105BE00000206472697665722063757272656E74E6
:105BF0003A2000206472697665722063757272655E
:105C00006E743A20004D6163726F20746F6F206C68
:105C10006F6E672E0A0020466C6F773A2000206472
:105C20003A0020693A0020703A00204500205A00CE
:105C3000205900204D393220580043290A00616262
:105C40006C656420286D696E2074656D7020006439
:105C5000697300656E00436F6C64206578747275BB
:105C60006465732061726520002054002052004159
:105C70006363656C65726174696F6E3A20500049A8
:105C80006E76616C69642065787472756465720AF9
:105C90000020643A0020693A0020703A00536C6595
:105CA00065702E2E2E0047322F473320626164200C
:105CB000706172616D65746572730A0050726F6213
:105CC00065205A204F66667365743A2000446F6EF3
:105CD0006520736176696E672066696C652E0A00BF
:105CE00053442072656164206572726F720A0044C9
:105CF0006F6E65207072696E74696E672066696C7C
:105D0000650A0053544F505045442E20005072698C
:105D10006E7465722073746F70706564206475654D
:105D200020746F206572726F72732E20466978201E
:105D3000746865206572726F7220616E642075737D
:105D400065204D39393920746F2072657374617222
:105D5000742E202854656D706572617475726520AB
:105D600069732072657365742E205365742069749D
:105D70002061667465722072657374617274696EF5
:105D800067290A004E6F20436865636B73756D2049
:105D900077697468206C696E65206E756D626572D6
:105DA0002C204C617374204C696E653A20004E6F54
:105DB00020436865636B73756D2077697468206C28
:105DC000696E65206E756D6265722C204C6173740E
:105DD000204C696E653A2000636865636B73756D6E
:105DE000206D69736D617463682C204C617374203D
:105DF0004C696E653A20004C696E65204E756D6287
:105E00006572206973206E6F74204C617374204C2E
:105E1000696E65204E756D6265722B312C204C6168
:105E20007374204C696E653A20004D313130005258
:105E30006573656E643A20002042002050006F6B4D
:105E400000220A00656E7175657565696E672022AE
:105E500000504944204175746F74756E6520666109
:105E6000696C656421204261642065787472756490
:105E70006572206E756D6265720A0042656420630A
:105E80006F6F6C696E672E2E2E0042656420686508
:105E90006174696E672E2E2E006F6B00307800479C
:105EA0003238205A0A47302058383020593139309A
:105EB0002046333030300A4D313137205072696E10
:105EC000742061626F727465642E002020506C61D2
:105ED0006E6E657242756666657242797465733A74
:105EE00020002046726565204D656D6F72793A20FD
:105EF00000436F6D70696C65643A204D61722032A9
:105F00003920323031390A00207C20417574686FA5
:105F1000723A2028416C657068204F626A6563742C
:105F20007320496E632E2C204C756C7A426F74205E
:105F3000476974205265706F7369746F7279290AAA
:105F40000000204C61737420557064617465643A7C
:105F50002000322E302E302E3130350A004D617245
:105F60006C696E0020536F667477617265205265AC
:105F70007365740A00205761746368646F67205208
:105F8000657365740A002042726F776E206F7574B6
:105F90002052657365740A002045787465726E61DD
:105FA0006C2052657365740A00506F776572557086
:105FB0000A0073746172740A004B494C4C45442EBC
:105FC00020005072696E7465722068616C7465643B
:105FD0002E206B696C6C28292063616C6C656421D0
:105FE0000A004B494C4C20636175736564206279EB
:105FF000204B494C4C20627574746F6E2F70696E23
:106000000A004B494C4C20636175736564206279CA
:1060100020746F6F206D75636820696E61637469A9
:1060200076652074696D65202D2063757272656ECA
:106030007420636F6D6D616E643A20004D313034B1
:1060400020533137302054300A4D313137204C65E0
:1060500076656C696E67205820417869730A47320B
:10606000380A473020583136302046393939390A14
:106070004730205A352046363030300A4739310A09
:106080004D3231312053300A4D3430300A4D3930E1
:1060900036205A3630300A4730205A2D31352046C6
:1060A0003530300A4730205A3520463530300A47DF
:1060B00039300A4D3430300A4D393036205A3936AD
:1060C000300A4D3231312053310A4732380A4D31CE
:1060D0003137204C6576656C696E6720646F6E653C
:1060E0002E0A4731320A4D31303920523136300ACA
:1060F0004D3131372050726F62696E67206265647E
:106100000070726F62655F726577697065005072CA
:106110006F62696E67206661696C6564004D31313C
:106120003720426564206C6576656C696E67206611
:1061300061696C65642E0A4730205A31300A473055
:106140002045300A4D333030205032352053383816
:10615000300A4D333030205035302053300A4D3323
:1061600030302050323520533838300A4D333030FB
:10617000205035302053300A4D33303020503235E6
:1061800020533838300A47342053310070726F6220
:10619000655F6661696C65640050726F74656374F5
:1061A00065642050696E0A0025311D402924301C89
:1061B0004527232F1B0A0743222B1A42043803FFCB
:1061C0003604080606000100925050870991F8AA8B
:1061D00061D9C8DFAA01AC01A801AE01299111243F
:1061E0001FBECFEFD1E2DEBFCDBF00E00CBF15E098
:1061F000A0E0B2E0E8EBFFEE02E00BBF02C00790C8
:106200000D92A83BB107D9F729E1A8EBB5E001C091
:106210001D92A73BB207E1F710E3CEEED0E300E01A
:1062200006C021970109802FFE010F94EC6FC43E38
:10623000D10780E00807A9F70E944F440D94CB775F
:106240000C9400001F920F920FB60F9211242F93FF
:106250003F938F939F93AF93BF938091B905909194
:10626000BA05A091BB05B091BC053091B80523E0FB
:10627000230F2D3720F40196A11DB11D05C026E87E
:10628000230F0296A11DB11D2093B8058093B90577
:106290009093BA05A093BB05B093BC058091BD0552
:1062A0009091BE05A091BF05B091C0050196A11DBA
:1062B000B11D8093BD059093BE05A093BF05B0931B
:1062C000C005BF91AF919F918F913F912F910F90FA
:1062D0000FBE0F901F9018952FB7F8946091B905D5
:1062E0007091BA058091BB059091BC052FBF0895B0
:1062F0003FB7F8948091BD059091BE05A091BF0570
:10630000B091C00526B5A89B05C02F3F19F0019696
:10631000A11DB11D3FBFBA2FA92F982F8827820F2B
:10632000911DA11DB11DBC01CD0142E0660F771F7B
:10633000881F991F4A95D1F708958F929F92AF9227
:10634000BF92CF92DF92EF92FF926B017C01D0DF80
:106350004B015C01C114D104E104F104F1F091D3CB
:10636000C7DFDC01CB0188199909AA09BB09883E5E
:106370009340A105B10570F321E0C21AD108E108EC
:10638000F10888EE880E83E0981EA11CB11CC11490
:10639000D104E104F10421F7DDCFFF90EF90DF900D
:1063A000CF90BF90AF909F908F900895789484B5D0
:1063B000826084BD84B5816084BD85B5826085BD01
:1063C00085B5816085BDEEE6F0E0808181608083E7
:1063D000E1E8F0E0108280818260808380818160CA
:1063E0008083E0E8F0E0808181608083E1EBF0E091
:1063F000808184608083E0EBF0E080818160808335
:10640000E1E9F0E080818260808380818160808327
:10641000E0E9F0E0808181608083E1EAF0E0808162
:1064200082608083808181608083E0EAF0E0808107
:1064300081608083E1E2F1E08081826080838081FD
:1064400081608083E0E2F1E0808181608083EAE71F
:10645000F0E080818460808380818260808380819D
:10646000816080838081806880831092C10008955C
:106470001F93CF93DF93182FEB0161E016D1209784
:1064800011F460E004C0CF3FD10531F461E0812F09
:10649000DF91CF911F9145C1E12FF0E0E556FC4F10
:1064A000E4914E2F50E0FA013197E231F10508F006
:1064B0009DC08827EE58FF4F8F4F0D94EC6F84B529
:1064C000806884BDC7BD97C084B5806284BDC8BDE7
:1064D00092C080918000806880938000D093890072
:1064E000C093880088C08091800080628093800083
:1064F000D0938B00C0938A007EC08091800088601A
:1065000080938000D0938D00C0938C0074C08091E4
:10651000B00080688093B000C093B3006CC08091DD
:10652000B00080628093B000C093B40064C08091DA
:106530009000806880939000D0939900C093980059
:106540005AC080919000806280939000D0939B000D
:10655000C0939A0050C08091900088608093900012
:10656000D0939D00C0939C0046C08091A00080689D
:106570008093A0008091A0008F7B8093A000D09397
:10658000A900C093A80037C08091A00080628093CA
:10659000A000D093AB00C093AA002DC08091A000B2
:1065A00088608093A000D093AD00C093AC0023C05E
:1065B00080912001806880932001D0932901C093AD
:1065C000280119C080912001806280932001D0931E
:1065D0002B01C0932A010FC0809120018860809315
:1065E0002001D0932D01C0932C0105C0C038D105E6
:1065F0000CF04CCF46CFDF91CF911F91089590E0E2
:10660000FC013197E231F10508F04EC08827EC57C4
:10661000FF4F8F4F0D94EC6F809180008F7703C0F8
:10662000809180008F7D809380000895809180000C
:10663000877FF9CF84B58F7702C084B58F7D84BD05
:1066400008958091B0008F7703C08091B0008F7D56
:106650008093B0000895809190008F7707C080915B
:1066600090008F7D03C080919000877F8093900081
:1066700008958091A0008F7707C08091A0008F7D42
:1066800003C08091A000877F8093A000089580912F
:1066900020018F7707C0809120018F7D03C08091FA
:1066A0002001877F809320010895CF93DF9390E0AE
:1066B000FC01EF51FC4F2491FC01E95DFB4F8491FB
:1066C000882361F190E0880F991FFC01EF55FB4F83
:1066D000C591D491FC01E957FB4FA591B49161118B
:1066E00009C09FB7F8948881209582238883EC9114
:1066F0002E230BC0623061F49FB7F8943881822F4B
:10670000809583238883EC912E2B2C939FBF06C00A
:106710008FB7F894E8812E2B28838FBFDF91CF911C
:1067200008951F93CF93DF93282F30E0F901E556AA
:10673000FC4F8491F901EF51FC4FD491F901E95DCF
:10674000FB4FC491CC23C1F0162F811158DFEC2FE1
:10675000F0E0EE0FFF1FE957FB4FA591B4918FB703
:10676000F894111105C09C91ED2FE095E92302C02A
:10677000EC91ED2BEC938FBFDF91CF911F9108959A
:10678000CF93DF93282F30E0F901E556FC4F849139
:10679000F901EF51FC4FD491F901E95DFB4FC49130
:1067A000CC2389F081112BDFEC2FF0E0EE0FFF1FDF
:1067B000E359FB4FA591B491EC91ED2381E090E07A
:1067C00021F480E002C080E090E0DF91CF91089555
:1067D00008951F920F920FB60F9211240BB60F92CD
:1067E0002F933F934F935F936F937F938F939F93D9
:1067F000AF93BF93EF93FF93E0910402F0910502F2
:106800001995FF91EF91BF91AF919F918F917F91DA
:106810006F915F914F913F912F910F900BBE0F9011
:106820000FBE0F901F9018951F920F920FB60F92E8
:1068300011240BB60F922F933F934F935F936F9357
:106840007F938F939F93AF93BF93EF93FF93E091C9
:106850000602F09107021995FF91EF91BF91AF9158
:106860009F918F917F916F915F914F913F912F9168
:106870000F900BBE0F900FBE0F901F9018951F9298
:106880000F920FB60F9211240BB60F922F933F93D6
:106890004F935F936F937F938F939F93AF93BF9328
:1068A000EF93FF93E0910802F09109021995FF918F
:1068B000EF91BF91AF919F918F917F916F915F9178
:1068C0004F913F912F910F900BBE0F900FBE0F90E5
:1068D0001F9018951F920F920FB60F9211240BB6AE
:1068E0000F922F933F934F935F936F937F938F9369
:1068F0009F93AF93BF93EF93FF93E0910A02F091C0
:106900000B021995FF91EF91BF91AF919F918F91DC
:106910007F916F915F914F913F912F910F900BBE9F
:106920000F900FBE0F901F9018951F920F920FB6E9
:106930000F9211240BB60F922F933F934F935F93B7
:106940006F937F938F939F93AF93BF93EF93FF9337
:10695000E0910002F09101021995FF91EF91BF9132
:10696000AF919F918F917F916F915F914F913F91E7
:106970002F910F900BBE0F900FBE0F901F90189588
:106980001F920F920FB60F9211240BB60F922F93F6
:106990003F934F935F936F937F938F939F93AF93A7
:1069A000BF93EF93FF93E0910202F09103021995D8
:1069B000FF91EF91BF91AF919F918F917F916F91D7
:1069C0005F914F913F912F910F900BBE0F900FBE93
:1069D0000F901F9018951F920F920FB60F921124CF
:1069E0000BB60F922F933F934F935F936F937F93C9
:1069F0008F939F93AF93BF93EF93FF93E0910C021C
:106A0000F0910D021995FF91EF91BF91AF919F9178
:106A10008F917F916F915F914F913F912F910F9047
:106A20000BBE0F900FBE0F901F9018951F920F92E4
:106A30000FB60F9211240BB60F922F933F934F93E3
:106A40005F936F937F938F939F93AF93BF93EF93D6
:106A5000FF93E0910E02F0910F021995FF91EF91D3
:106A6000BF91AF919F918F917F916F915F914F9166
:106A70003F912F910F900BBE0F900FBE0F901F9064
:106A8000189508951F93CF93DF93EC011D821C820C
:106A90001F821E82198681E0888782E28A871F868C
:106AA0001E86FE01B396CE01C1962FEF2193E81703
:106AB000F907E1F711E018A3CE0165D51F8B188EF9
:106AC000198E80E48A8F1B8E84E998E39AAB89AB98
:106AD000DF91CF911F910895DB01ED91FC91199405
:106AE000EF92FF921F93CF93DF931F921F92CDB728
:106AF000DEB77C01DC01D196ED91FC91D29782E06A
:106B000069837A83199520E030E04AE069817A81CF
:106B1000C701E2DF182FD701D196ED91FC91D297F2
:106B200083E01995D701D196ED91FC91D29780E041
:106B30001995812F0F900F90DF91CF911F91FF90AA
:106B4000EF9008950F931F93CF93DF93EC018B0188
:106B5000E9A9FAA982E01995E9A9FAA981E01995AC
:106B600020E030E044E1B801CE01B6DF9E012D5CAB
:106B70003F4F47E1B801CE01AFDFE9A9FAA980E0B4
:106B8000DF91CF911F910F911994EF92FF921F9374
:106B9000CF93DF93EC017B01E9A9FAA982E0199573
:106BA000E9A9FAA981E0199520E030E045E1B701B3
:106BB000CE0192DF182F882339F09E012D5C3F4FC4
:106BC00047E1B701CE0188DFE9A9FAA980E019956C
:106BD000812FDF91CF911F91FF90EF900895CF9378
:106BE000DF931F92CDB7DEB79E012F5F3F4F46E484
:106BF00073DF89810F90DF91CF910895CF93DF9359
:106C00001F92CDB7DEB79E012F5F3F4F47E464DF91
:106C100089810F90DF91CF91089520E030E048E422
:106C20005BCFCF93DF93EC016A817B81D8DF8883D0
:106C30006A817B81CE01E2DF89836A817B81CE011B
:106C4000ECDF8B879E012D5C3F4F6A817B8147E1A2
:106C5000CE01DF91CF9140CFCF93DF93EC016A81DA
:106C60007B813EDF882319F0CE01DBDF81E0DF91FD
:106C7000CF9108958F929F92AF92BF92CF92EF9251
:106C80000F93CF93DF931F921F92CDB7DEB74C01C6
:106C90005B012A834983F6DEF401B382A282498133
:106CA00047A32A8120A705A3E4A2C3A2C4010F9091
:106CB0000F90DF91CF910F91EF90CF90BF90AF9059
:106CC0009F908F90C9CFFC01628173813BCFCF939E
:106CD000DF93EC01EE85FF85309709F019956A8105
:106CE0007B81CE01DF91CF9150CF0F93FC01828148
:106CF0009381648F458F278F068F9F01245E3F4FBE
:106D00004BE3BC01CF010F91E7CEFC0160A30895D6
:106D1000BF92CF92DF92EF92FF920F931F93CF9388
:106D2000DF936C01D62FB42EC22F7801CC2369F0EB
:106D3000F701049120E04B2D6D2FC601D6DFFFEF48
:106D4000EF1AFF0AC150D85FF1CFDF91CF911F91A9
:106D50000F91FF90EF90DF90CF90BF9008958F92AA
:106D60009F92AF92BF92CF92DF92EF92FF920F93DA
:106D70001F93CF93DF935C01C62EC42FD22ED02F4A
:106D8000220F220F220F1ED0882379F0DC0F8D2CCA
:106D9000912CCD1751F087012D2D4C2F6C2DC50155
:106DA000B7DFE80CF91CCF5FF4CFDF91CF911F91D3
:106DB0000F91FF90EF90DF90CF90BF90AF909F909A
:106DC0008F9008950F93FC010150040F84A996A998
:106DD000941718F0081728F402C0081750F0041789
:106DE00040F42150260F83A995A9961720F428175F
:106DF00020F480E007C0281720F481E0261710F067
:106E0000F8CF81E00F91089581E008952EE93FE0E9
:106E1000009729F0F9013197F1F70197F9CF08951B
:106E2000FC01128280818150838314820895FC01C9
:106E300080819281980F92832181921760F49481CE
:106E40009F5F94839381890F821710F08FEF820FD9
:106E5000838381E0089580E00895FC0191E08381BF
:106E6000861708F490E031E0461708F030E0832FF1
:106E7000892B21E05281451708F420E02823832F35
:106E80008923822B0895DC01FB01108212968C91DC
:106E90001297818315968C91159781508283139652
:106EA0008C9183830895FB0141812381213029F056
:106EB000233031F468EF640F04C0642F485F01C0D1
:106EC000642FCBCFDC0115962C9115971696ED917A
:106ED000FC911797CF01820F911D820F911D119286
:106EE000E817F907E1F70895FC01A681B7818281CF
:106EF000481B8581483018F0A80FB11D4770382F06
:106F0000369536953695562F577080E890E002C03A
:106F1000959587955A95E2F7439F402D11246695E4
:106F200066956695E62FF0E0E40FF11DEA0FFB1F72
:106F30003081222311F0832B02C08095832380832C
:106F40000895FB014181DC0112962C9112974217A2
:106F500060F013962C911397241738F060811596E2
:106F60002C91621710F42481BFCF0895CF92DF9245
:106F7000FF920F931F93CF93DF936C01EB01FA8085
:106F80009B81913051F030F0923049F0933051F4C0
:106F90001FEF09C010E001E007C011E004C010E0DD
:106FA0000FEF02C010E000E0F7FE03C0BE01C60113
:106FB000C8DF9881900F98839981910F9983FF0C76
:106FC00099F7DF91CF911F910F91FF90DF90CF90B4
:106FD00008950F931F93CF93DF938901FB01C28123
:106FE000D3814233D9F058F44531E1F0473109F10A
:106FF000443141F5CE0166DFCE0112DF23C04634B5
:10700000E1F04734E1F04B33E9F4B901CE014BDF55
:107010008823C1F0B801CE01A9DF14C0B901CE01A7
:1070200090DF10C0CE0103DF882369F0CE014ADF74
:1070300009C0B901CE0127DF05C08D8101C089815A
:10704000F801808381E0DF91CF911F910F91089526
:10705000CF92DF92EF92FF920F931F93CF93DF9324
:107060007C01D62FD42EC22F122FC62EC20E6C2D0D
:10707000611B183038F00FEF20E04D2DC70135DED1
:107080001850F5CF6C2F687F6D0F2C2F277071F083
:1070900097E029272F5F27700FEF10E001C0000F46
:1070A0002A95EAF720E04D2DC7011FDEDF91CF9131
:1070B0001F910F91FF90EF90DF90CF900895EF9286
:1070C000FF920F931F93CF93DF937C01D62F122F44
:1070D000C42F040F212F4C2F6D2FC701B9DFCF5FB5
:1070E0000C13F8CFDF91CF911F910F91FF90EF908C
:1070F0000895DF92EF92FF920F931F93CF93DF9348
:10710000EC01162FF42EE22E5DDE882329F02E2DC1
:107110004F2D612FCE01D3DFDF91CF911F910F91C2
:10712000FF90EF90DF9008950895FC01E60FF11DA8
:10713000849190E0982F88273196E4918E0F911DCD
:107140000895FC0184910895FCDF882321F08230AA
:1071500011F083E0089586E0089580E00895FC0131
:107160008081089566E0E1CF68E0DFCF0A96FC01F8
:10717000849108950B96FC0184910895DC01149686
:10718000ED91FC911597319684910895BF92CF921D
:10719000DF92EF92FF920F931F93CF93DF938C01B7
:1071A000E62EDC011496CD91DC911597CE01C9DF56
:1071B000F82EF80184819581C7DFC82EF1E0FF1217
:1071C00003C02FE0B22E02C0BB24BA94D80114969B
:1071D0008D919C911597CADFF82EF80184819581D5
:1071E000C9DFD82ED80114968D919C911597BCDFDC
:1071F000B0E6BE1538F4009729F0C80FD91F91E604
:10720000F92E0FC0F80184819581ACDFF0E4FE1502
:1072100038F4009729F0C80FD91F81E4F82E01C077
:107220006196DE1490F4D80150961C9250975396B4
:107230001C92539754961C92549751961C925197B6
:1072400052961C9280E090E066C0DF1460F38C2DB3
:1072500090E0FE0124912F3F11F4219657C0FE10BB
:107260004CC0D80114968D919C9115976ADF9E01B0
:107270002F5F3F4FFE01882311F08230E1F48491AB
:10728000D80153968C935397F901249154962C93DB
:107290005497FE013396E4915096EC935097FE017B
:1072A0003496E4915196EC935197FE013596E49112
:1072B0005296EC9320C08491982F9F709250D801E1
:1072C00052969C93529782958F7051968C935197BA
:1072D000F9012491822F8F7054968C9354972295A4
:1072E0002F7053962C935397FE013296E491E295BA
:1072F000EF705096EC93CE010EC0FE013296E491F1
:10730000EB219C012E0F311DC20FD31FFD1409F478
:107310008ACFF3949ECFDF91CF911F910F91FF9071
:10732000EF90DF90CF90BF9008954F925F926F9251
:107330007F929F92AF92BF92CF92DF92EF92FF9295
:107340000F931F93CF93DF931F92CDB7DEB72C011E
:10735000C62E942E622F1ADF7C01892B09F43AC0C5
:10736000F20184819581F0DEB82EF201138904893F
:107370008189C80E8289981AD92CD01A212F4D2DB7
:107380006C2DC2011FDD882311F1EB0CF11C195F7C
:10739000169516951695612E712CD914C1F03C2DB9
:1073A00057018A2D8E19811770F4F501049120E0A0
:1073B0004D2D632FC201398398DCFFEFAF1ABF0A4E
:1073C0003981385FEECFE60CF71CD394E6CFF2019B
:1073D000808901C080E00F90DF91CF911F910F91C4
:1073E000FF90EF90DF90CF90BF90AF909F907F90F5
:1073F0006F905F904F9008950F931F93CF93DF93FB
:1074000000D0CDB7DEB78C01DC015596ED91FC9133
:1074100056972B834A83698319954A81480F2B819C
:107420006981C8010F900F900F90DF91CF911F914C
:107430000F917BCFAF92BF92DF92EF92FF920F93AB
:107440001F93CF93DF931F921F92CDB7DEB77C01BE
:10745000D62E042FDC015596ED91FC915697298389
:107460003A831995080F2981A22E3A81B32E10E094
:10747000F50121915F01222339F0402F6D2DC701C5
:1074800054DFD80E180FF4CF812F0F900F90DF919B
:10749000CF911F910F91FF90EF90DF90BF90AF9031
:1074A0000895DF92EF92FF920F931F93CF93DF9394
:1074B0007C01D62FD42E8901DC015596ED91FC91EB
:1074C00056971995D80EC0E0F8012491222349F06F
:1074D0004D2D6D2FC70129DFD80FC80F0F5F1F4F2C
:1074E000F3CF8C2FDF91CF911F910F91FF90EF90F1
:1074F000DF900895DC0114962D913C91159721158C
:10750000310509F43FC057968C915797F9018111C5
:1075100008C03596E4915896EC935897F9013C963B
:1075200011C0813041F43F96E4915896EC935897FE
:10753000F901709607C03D96E4915896EC935897E0
:10754000F9013E96E4915996EC93599758968C918F
:107550005897082E000C990B59962C915997821B1D
:10756000910927FD93955A962C915A97203441F012
:10757000829FC001112426E0969587952A95E1F710
:107580005B968C9308952DEA38E3FC01368B258BAE
:107590000895CF92DF92EF92FF920F931F93CF93B4
:1075A000DF938C017B016A01CB01FA011995D82F79
:1075B000882311F1682FC801E9DDF801C189C1955F
:1075C000FFEFEF1AFF0AC701F6011995F8018823AA
:1075D00051F08089C80FC701F6011995D82F682F7F
:1075E000C801D4DDEDCFD03221F091898389890F94
:1075F00001C080898C0F01C080E0DF91CF911F9185
:107600000F91FF90EF90DF90CF9008954FEA58E3ED
:10761000C0CFCF93DF93FC01248135812617370734
:1076200041F0EC017583648365DF8DEA98E39E8BFE
:107630008D8BDF91CF9108954F925F926F927F92E1
:10764000AF92BF92CF92DF92EF92FF920F931F9370
:10765000CF93DF93CDB7DEB729013A019B01AC018F
:1076600024193509460957098A899B89AC89BD893E
:10767000BC01CD016A197B098C099D090F946C6FBF
:10768000A801970124193509460957090F94D06FAD
:10769000CA01B9016A0D7B1D8C1D9D1DDF91CF9123
:1076A0001F910F91FF90EF90DF90CF90BF90AF9020
:1076B0007F906F905F904F90089580E090E00895E4
:1076C0000895CF92DF92EF92FF920F931F93CF9383
:1076D000DF936C017A018B01C0E0D0E0CE15DF05AD
:1076E00089F0D8016D918D01D601ED91FC91019049
:1076F000F081E02DC6011995892B11F47E0102C09D
:107700002196ECCFC701DF91CF911F910F91FF9090
:10771000EF90DF90CF900895DC01ED91FC91019006
:10772000F081E02D1994CF93CFB7F8948091C405E0
:10773000811127C0ECE5F4E08491E6E1F4E0949156
:10774000E82FF0E0EE0FFF1FEF55FB4FA591B4912E
:10775000EC91E92321F461E085E30E94913361E03B
:1077600085E30E9455338CB580618CBD8CB58064F7
:107770008CBD61E084E30E94553361E083E30E94A5
:1077800055338091C4058F5F8093C405CFBFCF91DF
:107790000895CF92EF920F93FC0113AE14AE15AE85
:1077A000049668DA0F91EF90CF900895CF92DF9210
:1077B000EF92FF921F93CF93DF93EC0180E090E074
:1077C0000F94046D25ED34E045E352E40F94A26E6E
:1077D00020E030E04AE754E40F946B6C6B017C01CD
:1077E0002AE037ED43EA5CE369857A858B859C85E1
:1077F0000F948B6B9B01AC01C701B6010F94A26E75
:1078000026E636E646EA5EE30F946B6C20E030E055
:1078100040E85FE30F948A6B0F94D86C162FE881D1
:10782000F9810480F581E02D603118F561E0CE0129
:1078300019952AE037ED43EA5CE369857A858B8503
:107840009C850F948B6B9B01AC01C701B6010F9413
:10785000A26E2CEE31E548E35EE30F946B6C20E002
:1078600030E040E85FE30F948A6B0F94D86C162FDA
:1078700003C060E0CE011995612FCE01C6D2612F01
:1078800070E080E090E00F94066D2D853E854F8579
:1078900058890F94A26E0F94D86CCE01DF91CF91CE
:1078A0001F91FF90EF90DF90CF9092C2FC0125874F
:1078B00036874787508B7ACFCF92DF92EF92FF9235
:1078C000CF93DF93EC01DED2682F70E06F5F7F4FC4
:1078D000072E000C880B990B0F94066D20E030E00A
:1078E00040E05DE30F94A26E6B017C01E881F981B9
:1078F0000680F781E02DCE011995811105C026E69D
:1079000036E646EA5EE304C02CEE31E548E35EE38A
:10791000C701B6010F94A26E6B017C012AE037ED1E
:1079200043EA5CE369857A858B859C850F948B6B34
:107930009B01AC01C701B6010F946B6C25ED34E0DF
:1079400045EB5FE30F946B6C20E030E04AE754E4D2
:107950000F94A26E0F94D86CCB01DF91CF91FF9062
:10796000EF90DF90CF900895DC01ED91FC910084C1
:10797000F185E02D1995611571058105910539F0A5
:107980006F3F7F4F8F4F9F4F21F080E0089582E03F
:10799000089581E00895DC01ED91FC910484F58562
:1079A000E02D199583500895DC01ED91FC9100883C
:1079B000F189E02D19958F5F08956031710509F403
:1079C00041C088F46230710509F454C020F4672B7B
:1079D00009F458C008956430710509F443C0683053
:1079E0007105C1F1089560347105E1F020F4603251
:1079F000710501F108956038710561F061157140FC
:107A000009F048C0DC01ED91FC910288F389E02D7A
:107A100060E03FC0DC01ED91FC910288F389E02D2C
:107A200061E037C0DC01ED91FC910288F389E02D23
:107A300062E02FC0DC01ED91FC910288F389E02D1A
:107A400063E027C0DC01ED91FC910288F389E02D11
:107A500064E01FC0DC01ED91FC910288F389E02D08
:107A600065E017C0DC01ED91FC910288F389E02DFF
:107A700066E00FC0DC01ED91FC910288F389E02DF6
:107A800067E007C0DC01ED91FC910288F389E02DED
:107A900068E019940895DC01ED91FC910488F58962
:107AA000E02D1995893048F4E82FF0E0EE0FFF1F24
:107AB000EA5EFC4F80819181089580E090E0089516
:107AC000DC01ED91FC91008CF18DE02D1995843055
:107AD00030F4E82FF0E0EE5EFC4F8081089580E006
:107AE0000895DC01ED91FC910280F381E02D61E0CD
:107AF0001995862F0895FC0185810895DC0115965E
:107B00006C931597ED91FC91262F30E040E050E00A
:107B10000190F081E02D61E11994DC01ED91FC917F
:107B20000280F381E02D62E11994FC012681378106
:107B30008085482F4F70842FB90190E00895DC01B3
:107B40009A01462F4F7016962C93169717963C93D2
:107B50001797942F9F7018968C911897807F892B78
:107B600018968C931897ED91FC91119750E0019025
:107B7000F081E02D63E1CD011994FC0167A170A5AE
:107B800092A581A591700895DC0197964C939797E3
:107B900098965C93989799966C9399979A968C91EE
:107BA0009A9770FB80F99A968C939A97ED91FC9135
:107BB00011979A01AB0151700190F081E02D6DE6B3
:107BC000CD011994DC016F7097962C919797207FC7
:107BD000262B97962C939797ED91FC911197989659
:107BE0003C91989799964C9199979A965C9151707F
:107BF0000190F081E02D6DE61994DC016F7098968C
:107C00003C919897307F362B98963C939897ED91BE
:107C1000FC91119797962C91979799964C919997DB
:107C20009A965C9151700190F081E02D6DE6199467
:107C3000DC016F7799964C9199974078462B9996ED
:107C40004C939997ED91FC91119797962C9197975A
:107C500098963C9198979A965C9151700190F0811A
:107C6000E02D6DE61994FC0191A5990F9595292FAA
:107C7000092E000C330B20743327220F331F892F5A
:107C80008F77822B0895DC01ED91FC910280F381C6
:107C9000E02D6FE61994DC01ED91FC910084F185F3
:107CA000E02D1995CB0193700895DC01ED91FC91C5
:107CB0000084F185E02D199577FB882780F90895D8
:107CC000DC01ED91FC910084F185E02D19958F7117
:107CD0000895DC01ED91FC910084F185E02D19956A
:107CE000892F81700895DC01ED91FC910084F1856C
:107CF000E02D199591FB882780F90895DC01ED911D
:107D0000FC910084F185E02D199592FB882780F97C
:107D10000895DC01ED91FC910084F185E02D199529
:107D200093FB882780F90895DC01ED91FC91008494
:107D3000F185E02D199594FB882780F90895DC01E1
:107D4000ED91FC910084F185E02D199595FB882734
:107D500080F90895DC01ED91FC910084F185E02D1E
:107D6000199596FB882780F90895DC01ED91FC9127
:107D70000084F185E02D199597FB882780F90895F7
:107D8000FC01228133818481482F4F70842FB901F7
:107D900090E00895DC019A01462F4F7012962C93C3
:107DA000129713963C931397942F9F7014968C916F
:107DB0001497807F892B14968C931497ED91FC91E6
:107DC000119750E00190F081E02D60E1CD01199410
:107DD000DC016F7112968C911297807E682B12963F
:107DE0006C931297ED91FC911197262F13963C916D
:107DF000139714968C911497482F4F7050E0019070
:107E0000F081E02D60E1CD011994DC016F711396D2
:107E10008C911397807E682B13966C931397ED913A
:107E2000FC91119712962C911297362F14968C91E3
:107E30001497482F4F7050E00190F081E02D60E1E1
:107E4000CD011994DC016F7014968C911497807F8A
:107E5000682B14966C931497ED91FC9111971296E0
:107E60002C91129713963C911397462F4F7050E028
:107E70000190F081E02D60E1CD011994FC01828137
:107E80008F710895FC0183818F710895DC01677003
:107E9000962F9295907F92966C9192976F78692B1E
:107EA00092966C939297ED91FC91119792962D91E9
:107EB0003D914D915C9195970190F081E02D6CE69C
:107EC000CD011994DC0192968C91929760FB87F911
:107ED00092968C9392976695677093968C919397F0
:107EE000887F682B93966C939397ED91FC911197F3
:107EF00092962D913D914D915C9195970190F081D5
:107F0000E02D6CE6CD011994DC0193968C9193974A
:107F100060FB87F993968C93939761FB882780F990
:107F200094966C9194976E7F682B94966C9394972B
:107F3000ED91FC91119792962D913D914D915C910F
:107F400095970190F081E02D6CE6CD011994DC014C
:107F500094962C91949760FB21F994962C93949786
:107F6000ED91FC91119792962D913D914D915C91DF
:107F700095970190F081E02D6CE619946F70DC010B
:107F800095962C919597207F622B95966C9395975B
:107F9000ED91FC91119792962D913D914D915C91AF
:107FA00095970190F081E02D6CE61994CF93DF93C3
:107FB000EC01E881F9810280F381E02D6CE61995EE
:107FC0006AA37BA38CA39DA3DF91CF910895CF9348
:107FD000DF93EC01EBDF8AA182958770DF91CF916F
:107FE0000895CF93DF93EC01E1DF9AA1991F9927C0
:107FF000991F8BA18770880F892BDF91CF910895EE
:10800000CF93DF93EC01D2DF9BA1991F9927991F92
:108010008CA18170880F892BDF91CF910895CF9328
:10802000DF93EC01C3DF8CA186958170DF91CF9146
:108030000895CF93DF93EC01B9DF8DA18F70DF91AD
:10804000CF910895DC0192964D935D936D937C934F
:108050009597ED91FC910190F081E02D9A01AB0193
:108060006CE619946F70DC0192962C919297207FA8
:10807000622B92966C939297ED91FC911197929648
:108080002D913D914D915C9195970190F081E02D5E
:108090006CE61994CF93DF93EC0188DF8AA18F708F
:1080A000DF91CF910895CF92DF92EF92CF93DF933C
:1080B000EC01E881F9810280F381E02D60E01995FF
:1080C0006B01E82E23E0E222CA8ADB8A2E2D237080
:1080D0009C899C7F922B9C8B8E2DB60190E0DF912A
:1080E000CF91EF90DF90CF900895DC019A01462F59
:1080F000437052962C93529753963C935397942FD8
:10810000937054968C9154978C7F892B54968C93B2
:108110005497ED91FC91119750E00190F081E02D82
:1081200060E0CD011994DC0152968C91529760FB6E
:1081300082F952968C935297ED91FC911197282FCA
:1081400053963C91539754968C915497482F437073
:1081500050E00190F081E02D60E0CD011994DC0148
:1081600052968C91529760FB84F952968C93529759
:10817000ED91FC911197282F53963C91539754966B
:108180008C915497482F437050E00190F081E02D7E
:1081900060E0CD011994DC0153968C91539760FBFC
:1081A00080F953968C935397ED91FC9111975296C9
:1081B0002C915297382F54968C915497482F437096
:1081C00050E00190F081E02D60E0CD011994CF9353
:1081D000DF93EC0168DF8A8982FB882780F9DF91D1
:1081E000CF910895FC0123A534A585A5482F4F7391
:1081F000842FB90190E00895DC019A01462F4F7356
:108200009B962C939B979C963C939C97942F9F7343
:108210009D968C919D97807C892B9D968C939D97A4
:10822000ED91FC91119750E00190F081E02D60E715
:10823000CD011994CF93DF93EC0161E088810E9416
:10824000553361E08C810E94553362E08A810E943F
:108250005533E881F981EF51FC4FE491EE83EA81D7
:10826000FB81EF51FC4FE491EF83EC81FD81EF51F5
:10827000FC4FE491E887DF91CF9108959F92AF92F0
:10828000BF92CF92DF92EF92FF920F931F93CF9303
:10829000DF938C01942E87E0C82ED12CE12CF12C99
:1082A000C0E0A62EB12CC501911019C00E2C02C041
:1082B000959587950A94E2F780FF02C061E001C0BE
:1082C00060E0F80180810E94913361E0F8018481CF
:1082D0000E949133F8018281911016C007C00C2CC6
:1082E00002C0959587950A94E2F7E6CF0E94C033C5
:1082F00021E030E0892B11F420E030E00E2C01C0A9
:10830000220F0A94EAF70DC00E94C03321E030E04A
:10831000892B11F420E030E00C2C01C0220F0A94CC
:10832000EAF7C22B60E0F80184810E949133FFEFED
:10833000EF1AFF0A81E0C81AD108E8E0EE16F1044E
:1083400009F0B1CF8C2FDF91CF911F910F91FF904A
:10835000EF90DF90CF90BF90AF909F9008950F93D4
:108360001F93CF93DF938C01D62F672F41E086DFD9
:10837000C82F41E06D2FC80181DF2C2F30E0322F54
:108380002227A901482BCA01DF91CF911F910F919C
:1083900008950F93FC0130E080E092E1AAE7B0E09D
:1083A000481759076A077B0740F4B695A795979534
:1083B00087953F5F3630A1F737E091E0932722237E
:1083C00011F020E501C020E7892F86950C70082B5D
:1083D000022B0083917091830F9108952091C30522
:1083E000222399F04FB7F8942091C305213059F416
:1083F0002DB32093C1053DB32091C20520952323C1
:108400002DBB4FBF02C04093C1058CBD9DBD0895DB
:108410008EBD00000DB407FEFDCF8EB508950CB4DF
:1084200005FC0DC09EBD00000DB407FEFDCF9EB53E
:108430008EBD00000DB407FEFDCF8EB508958EBD34
:1084400000000DB407FEFDCF8EB59EBD00000DB43B
:1084500007FEFDCF9EB508958091C305882361F086
:108460009FB7F8942091C3058091C105213019F47C
:108470008DBB9FBF08958FBF0895CF93DF93FC01FD
:10848000128213828481807F8483158216821782F0
:108490008085807F8087218732874387548780E06B
:1084A00090E0A0E0BFE385879687A787B08B8CE23A
:1084B00093E091838083128A138A84898C7F848BD2
:1084C000158A168A8789807F878B108E118E828D00
:1084D000807F828F138E148E158E868D8E7F868F71
:1084E000178E10A281A1807881A3DF01929685E08A
:1084F000ED0119928A95E9F717A210A611A682A597
:108500008E7F82A713A614A685A5807C85A786A545
:108510008C7F86A770AB67A712AA11AADF91CF91B3
:108520000895FC0187A50C949133AF92BF92CF922E
:10853000DF92EF92FF920F93CF93DF931F921F92E0
:10854000CDB7DEB75C01F62EFC0181A992A9892B7B
:1085500009F44EC060E0C501E4DF41E06F2DF50194
:1085600081A992A98BDE60E070E0F50181A992A952
:10857000F6DE60E070E0F50181A992A9F0DE61E02D
:10858000C501CFDF60E0C501CCDF41E06F2DF50113
:1085900081A992A973DEF501818B41E060E081A998
:1085A00092A96CDEC82ED12CE12CF12CFE2CED2CE6
:1085B000DC2CCC2441E060E0F50181A992A95EDECB
:1085C000C82AFE2CED2CDC2CCC2441E060E0F50127
:1085D00081A992A953DEC82AFE2CED2CDC2CCC24D8
:1085E00041E060E0F50181A992A948DEC82A41C0B6
:1085F0004091100250911102609112027091130289
:108600000CE021E0CE010196C4DE89819A81E6DE8C
:1086100060E0C50186DF8F2DFBDE80E090E0FFDEAD
:1086200080E090E0FCDE61E0C5017BDF60E0C50139
:1086300078DF8F2DEDDEF501818B80E0E9DEC82E3D
:10864000D12CE12CF12CFE2CED2CDC2CCC2480E068
:10865000DFDEC82AFE2CED2CDC2CCC2480E0D8DE1A
:10866000C82AFE2CED2CDC2CCC2480E0D1DEC82ADC
:10867000F3DE61E0C50155DFC701B6010F900F9031
:10868000DF91CF910F91FF90EF90DF90CF90BF904F
:10869000AF9008954F925F926F927F928F929F92C8
:1086A000AF92BF92EF92FF920F931F93CF93DF93FE
:1086B0001F921F92CDB7DEB77C0149015A01162FD8
:1086C0001068FC0181A992A9250166247724892BD1
:1086D000A9F060E0C70125DF41E0612FF70181A922
:1086E00092A9CCDDF701818BB20181A992A937DE75
:1086F000B401F70181A992A932DE1CC04091100299
:108700005091110260911202709113020CE021E06D
:10871000CE0101963EDE89819A8160DE60E0C7016C
:1087200000DF812F75DEF701818BC20178DEC40185
:1087300076DE92DE61E0C701F4DE0F900F90DF91EC
:10874000CF911F910F91FF90EF90BF90AF909F90AE
:108750008F907F906F905F904F900895CF93DF93AD
:10876000EC0161E08FA50E94553361E0CE01D9DEB6
:1087700089A99AA9009709F05DDD8A899B892C89CE
:10878000A22FA370AC016A2F70E0CE01AEDC4AA12B
:108790005BA16CA17DA1CE0155DC4FA158A569A5B7
:1087A0007AA57170CE01F0D98BA59CA52DA5A22F1D
:1087B000AF73AC016A2F70E0CE011EDD8A819B8110
:1087C0002C81A22FAF70AC016A2F70E0CE01E2DAEB
:1087D00068E0CE0147DCE881F9810688F789E02D61
:1087E00061E0CE01DF91CF911994DC01ED91FC9114
:1087F0000280F381E02D64E01994F7DF64FB8827A1
:1088000080F90895CF93DF93EC01F7DF811105C064
:10881000CE0140DC91E0811101C090E0892FDF9111
:10882000CF910895FC01258936898789482F4F709B
:10883000842FB90190E00895DC019A01462F4F7012
:1088400055962C93559756963C935697942F9F7018
:1088500057968C915797807F892B57968C93579773
:10886000ED91FC91119750E00190F081E02D64E1D1
:10887000CD011994FC01208D318D828D482F4F70D0
:10888000842FB90190E00895DC01ED91FC91028004
:10889000F381E02D61E71995862F089508950E94D0
:1088A000D631FCDF0F94CD6AC0E0D0E00F945F6B4F
:1088B0002097E1F30E940000F9CF0E945982409175
:1088C000770D909138022091800D3091810D60914B
:1088D0006402709165022627372760915C0D7091C4
:1088E0005D0D26273727949FA0011124440F452FA3
:1088F000441F550B519524273527A9014827CA0144
:108900002091CA053091CB052817390731F0909393
:10891000CB058093CA0581E0089580E00895E3EADD
:10892000F7E080E09191992311F08927FBCF909196
:10893000CC0591110BC091E02091C905281301C00D
:1089400090E09093C80591E09093CC059091C80574
:1089500091118093C90581E0911101C080E00895D3
:108960000E945982982F81E02091C705291302C0E7
:1089700080E008959093C70508955D9A88E28A95EE
:108980000000E9F78091D4058E7F8093D405089587
:108990005D988091D4058E7F8093D405089588EFEB
:1089A0000E94B55088E28A950000E9F708958AEFA1
:1089B0000E94B55088E28A950000E9F708958091F9
:1089C000D405982F9370913029F081608D7F80932A
:1089D000D405EDCF0895CF93C82F807F0E94B55066
:1089E0008C2F8295807F0E94B55088E28A95000086
:1089F000E9F7CF910895CF93DF931F92CDB7DEB7FC
:108A00009091D405292F2370233039F09160926022
:108A10009093D4058983C3DF89810F90DF91CF9133
:108A2000DACF1F93CF93DF931F92CDB7DEB7182F06
:108A3000811102C080E201C084E2611102C090E0B5
:108A400001C092E0892B6983D6DF9091D40510FB99
:108A500092F9892F698160FB83F98093D4050F9087
:108A6000DF91CF911F9108956091D40562FB992702
:108A700090F9891721F063FB662760F9D2CF08953A
:108A8000CF93C82F81E0F0DFC11102C082E201C0A4
:108A900083E2B1DF9091D405C0FB94F99093D405A3
:108AA000CF9108959091D405929591708913E8CF54
:108AB000089561E081E0B5DF61E081E0B2DF80E050
:108AC000DFCFCF93C82F80E0CFDF8C2F8F738068EC
:108AD000CF9191CFCF93C82F80E0C6DF8C2F8F73BB
:108AE0008064CF9188CF1F93CF93DF931F92CDB730
:108AF000DEB7182F81E06983B7DF6981862F806830
:108B00007ADF812F8F7080680F90DF91CF911F9156
:108B100072CF80E0A9DF81E06EDF6FE070E080E07F
:108B200090E00C949D3129DFF4DF61E081E079DF92
:108B30002FCF23DFBEDFEDDF61E081E072DF28CFE2
:108B4000CF93C82F85E0BDDF3ADFC11102C0C6E078
:108B500001C0C4E080E03FDF8C2FCF913CCFCF92AB
:108B6000DF92EF92FF921F93CF93DF931F921F929A
:108B7000CDB7DEB769837A83ADDF21DF6981C62E89
:108B80007A81D72E11E1115059F0F601E590F49059
:108B90008F2D21DF8E2D1FDF82E0C80ED11CF3CF79
:108BA0000F900F90DF91CF911F91FF90EF90DF908A
:108BB000CF900895CF93DF93C0E06C2F80E093DFD8
:108BC000FEDED1E1D15029F080E005DF80E003DF57
:108BD000F9CFCF5FC03289F7DF91CF910895CF925F
:108BE000DF92EF92FF920F931F93CF93DF931F9229
:108BF000CDB7DEB7982F623010F06250985FC62E66
:108C0000C29480EFC8228A01D12C6D2D6C0D892F62
:108C1000998369DFD4DEF801E590F4908F2DDBDED7
:108C20008E2DD9DED3940E5F1F4F998180E1D8122B
:108C3000ECCF0F90DF91CF911F910F91FF90EF90AC
:108C4000DF90CF90089580E02DDF69ED77E180E03F
:108C500090E085DF69EB77E180E190E080DF69E912
:108C600077E180E290E07BDF69E777E180E390E005
:108C700076DF49E158E160E080E0B1DF49EF57E19C
:108C800061E080E0ACDF49E557E161E085E0A7DF26
:108C900080E056CFCF93DF93EC018991882311F0C8
:108CA0009ADEFBCFDF91CF9108950F931F93CF935F
:108CB000DF93CDB7DEB727970FB6F894DEBF0FBEB0
:108CC000CDBF6330B1F038F46130B1F0623049F5B6
:108CD00025E437E113C0653031F040F0663009F526
:108CE00025E537E10BC021E537E108C02DE437E188
:108CF00005C029E437E102C021E437E19F938F9357
:108D00003F932F938E010F5F1F4F1F930F930F946D
:108D1000B174C801BFDF0F900F900F900F900F90AC
:108D20000F9027960FB6F894DEBF0FBECDBFDF9130
:108D3000CF911F910F9108950F931F93CF938C01A3
:108D4000C62FF80181918F01882329F0CC2319F0D7
:108D500042DEC150F6CFCF911F910F910895CF926F
:108D6000DF92EF92FF920F931F93CF93DF93CDB7D4
:108D7000DEB727970FB6F894DEBF0FBECDBF8C01CC
:108D800088E09FDEF80160817181828193812CE30C
:108D9000C22ED12CE12CF12CA70196010F94AE6FBD
:108DA000CA01B901A70196010F94AE6F8E010F5F42
:108DB0001F4F2436310598F47F936F933F932F9381
:108DC0008BE297E19F938F931F930F930F94B1744E
:108DD0000FB6F894DEBF0FBECDBF85E012C07F9303
:108DE0006F933F932F9383E297E19F938F931F930A
:108DF0000F930F94B1740FB6F894DEBF0FBECDBFC2
:108E000086E0F801E80FF11D80E28083D8DD66E09E
:108E1000C80192DF27960FB6F894DEBF0FBECDBF14
:108E2000DF91CF911F910F91FF90EF90DF90CF9046
:108E30000895CF93DF93FC018491EF01219688235D
:108E400019F0C9DDFE01F8CFDF91CF910895CF92DF
:108E5000DF92EF92FF920F931F93CF93DF93C42E75
:108E6000623010F06250805F982F9170D92EC82F19
:108E7000C695D62FD295D07F89E3E82E88E1F82ECB
:108E800001E0F7011491602F6D0F8C2F2CDE97DD20
:108E9000CC2051F0D11002C0812F01C080E09BDDB9
:108EA000DD2021F0812F03C080E095DD80E093DD9F
:108EB0000F5FFFEFEF1AFF0A053019F7DF91CF912F
:108EC0001F910F91FF90EF90DF90CF9008958F92B8
:108ED0009F92AF92BF92DF92EF92FF920F931F93F8
:108EE000CF93DF93D82E69E10F947B6F20E1929F9F
:108EF000C001112469E170E00F949B6F80E090E85D
:108F00005C0102C0B594A7946A95E2F711E0ED2CDC
:108F1000F12C612F8CE0E7DD52DD20E030E000E055
:108F2000490189E1880E911CE814F90434F42E15E6
:108F30003F0534F0C0E0D0E004C0CFEFDFEF01C068
:108F4000E501113051F01D3041F0033011F4C160E2
:108F500006C0011104C0D06802C0CFEFDFEF8D2F33
:108F60003ADD8C2F38DD0F5F940124363105C1F6D0
:108F70001F5F1E3071F68CE0A4DD21DD80E22BDD69
:108F800029E02D1530F464E0C7018FDE8EE397E110
:108F900005C063E0C70189DE8AE397E1DF91CF91E5
:108FA0001F910F91FF90EF90DF90BF90AF909F9037
:108FB0008F903FCFCF93C82F0E941D87C11104C04F
:108FC0009091C605981721F08093C605CF917FCF69
:108FD000CF9108951F93CF93DF931F92CDB7DEB744
:108FE000182F80E169836DDDEADC6981662349F031
:108FF000111102C012E001C010E080E0ECDC812F12
:1090000003C080E2E8DC80E20F90DF91CF911F91F6
:10901000E2CCCF92DF92EF92FF920F93CF93DF9348
:10902000C82F6B017A01D22F813049F028F08230AD
:1090300049F0833039F008C081E043DD05C081E1AB
:1090400040DD02C089E03DDDBADC63E0C6012DDE13
:10905000DD2341F08AE1BFDC63E0C70126DE0111B8
:1090600006C015C0002399F085E397E1E2DE41E0F8
:109070004D276C2F85E0EBDE4D2F6C2F89E0DF91C3
:10908000CF910F91FF90EF90DF90CF90E0CEDF91E6
:10909000CF910F91FF90EF90DF90CF9008950F93B5
:1090A000CF936115710589F0C1E0681779073CF429
:1090B0009C01261B370B2330310544F406C09B016D
:1090C000281B390B233031050CF4C0E02091140229
:1090D00021702C1711F001E001C0042F2C2FAB01DF
:1090E000BC0180E096DF80911402C0FB80F9809380
:1090F0001402CF910F9108950F93CF9361157105CD
:1091000089F0C1E0681779073CF49C01261B370BF6
:109110002330310544F406C09B01281B390B233052
:1091200031050CF4C0E02091140222FB222720F923
:109130002C1711F001E001C0042F2C2FAB01BC0152
:1091400081E067DF80911402C0FB82F980931402F2
:10915000CF910F910895CF93C82F86E0B2DC2FDC1A
:1091600063E08C2F90E0A1DD85E2CF9134CCCF93EA
:10917000DF93EC0186E1A5DC22DC63E0CE0195DD26
:1091800085E2DF91CF9127CC4F925F926F927F92D1
:109190008F929F92AF92BF92CF92DF92EF92FF9207
:1091A0001F93CF93DF9300D01F92CDB7DEB7F82E79
:1091B000811104C082DB882309F467C00E945982B0
:1091C000182F0F94F06669837A838B839C83A09019
:1091D0006402B09065026091580D7091590D8091B4
:1091E0005A0D90915B0D0F94D36C2B013C01C090F4
:1091F0005C0DD0905D0D8090800D9090810D609100
:109200007C0D70917D0D80917E0D90917F0D0F945E
:10921000D36CDC01CB014F2DB40141DF4F2DB601E2
:10922000C2016ADF2091770DE22EF12C11110DC0E1
:109230009091380297FD09C0929F90011124790105
:10924000EE0CEF2CEE1CFF08F19424E62E9DC001DD
:109250002F9D900D112481589F4F6FEF70E00F9458
:109260009B6F862F78DFCE01019679DDC5017FDF08
:10927000EF2811F0812F64DC61E01C141D041CF048
:1092800060E080E001C0812FA5DE0F900F900F906D
:109290000F90DF91CF911F91FF90EF90DF90CF90D3
:1092A000BF90AF909F908F907F906F905F904F9006
:1092B0000895CF9388E105DC82DB83EA97E00E9482
:1092C0006681C82F66E183EA97E036DDC63120F477
:1092D00080E281DBCF5FFACFCF910895811103C087
:1092E0001EDB882311F0E5DF3BCB0895CF93C82F19
:1092F00044DB8C2F49DF8C2FF1DF8C2F5BDECF918D
:1093000047CB3BDBD6DB05DC55DC9DDC81E0EEDFCB
:109310003FCB80E0EBCF9091C505981729F0809363
:10932000C5058111EECFFFCB0895E2EEF5E083AFE6
:1093300064AF0895EF92FF920F931F93CF93DF9343
:109340007A016F3F71058105910509F058F482EEAD
:1093500095E00E948C3B86EE95E00E94BE38282F57
:1093600030E014C0C0911D06D0911E064D2F50E074
:10937000EC2FF0E08B019C01BF0186EE95E0ADD1B2
:10938000C80FC0931D06D0931E069C01C901DF9132
:10939000CF911F910F91FF90EF900895EF92FF9260
:1093A0000F931F93CF93DF938B01C2EED5E0FBACFD
:1093B000ECAC4E2D50E06F2D70E09C0186EE95E0F8
:1093C000E4D1F80EFBAEECAEDF91CF911F910F917F
:1093D000FF90EF900895EF92FF920F931F93CF931A
:1093E000DF938B01C2EED5E0FBACECAC4E2D50E030
:1093F0006F2D70E09C0186EE95E013D2F80EFBAE67
:10940000ECAEDF91CF911F910F91FF90EF900895F7
:109410000F931F93CF93DF93CDB7DEB728970FB687
:10942000F894DEBF0FBECDBF8A0123E0660F771F21
:109430002A95E1F7680F791F48E050E0CE010196C8
:109440000F94E57329813A81F80180819181281771
:10945000390790F08217930760F09C8182819817FA
:1094600058F081E090E03B812381231738F080E0C1
:1094700005C081E090E002C08FEF9FEF28960FB605
:10948000F894DEBF0FBECDBFDF91CF911F910F913A
:109490000895EF92FF920F931F93CF93DF93EC0108
:1094A0008B017A018A859B858617970731F0888121
:1094B00099810E94093B1B870A87888599850196B7
:1094C00089F00E811F81B701888199810E94063B36
:1094D000080F111D888599858017910718F481E080
:1094E00090E011C06E818A81680F97014C8188815C
:1094F00099810E941A3A2E813F81280F311D3F83A6
:109500002E8380E090E0DF91CF911F910F91FF902B
:10951000EF9008954F925F926F927F928F929F92F9
:10952000AF92BF92CF92DF92EF92FF920F931F9371
:10953000CF93DF93CDB7DEB72D970FB6F894DEBF8C
:109540000FBECDBF6C012A013B01490158011B86AA
:109550001C86CE0101967C0188E0F70111928A9564
:10956000E9F7DB01CA0127E0B695A795979587959E
:109570002A95D1F79A838983F42FFF77FD878F2F60
:1095800080588B838C831A8619864F3F510561055D
:10959000710509F018F460E070E026C06091D7050D
:1095A0007091D8058E01075F1F4F970148E05AE47C
:1095B0008091D5059091D6050E94B77F97FDEBCF9E
:1095C00069857A8583E0660F771F8A95E1F7809138
:1095D000D5059091D605680F791F48E050E0C70186
:1095E0000F94E5736F8178856115710519F44B86C9
:1095F000B60106C0C616D70619F08D8580688B8720
:10960000AE01455F5F4FC401F50119952D960FB668
:10961000F894DEBF0FBECDBFDF91CF911F910F91A8
:10962000FF90EF90DF90CF90BF90AF909F908F9082
:109630007F906F905F904F9008956F927F928F927E
:109640009F92AF92BF92CF92DF92EF92FF920F93D1
:109650001F93CF93DF9300D01F92CDB7DEB76C017D
:109660007B013A015901480119821A821B821C822E
:10967000AE014F5F5F4FB301C7010E9417807C01AD
:1096800049815A816B817C814115510561057105C4
:1096900029F084019501C6013DDFE6CF0F900F90C0
:1096A0000F900F90DF91CF911F910F91FF90EF904E
:1096B000DF90CF90BF90AF909F908F907F906F90F2
:1096C000089521E02093D905E5EDF5E091838083AD
:1096D0007383628380E090E008957F92AF92BF929F
:1096E000CF92DF92EF92FF920F931F93CF93DF936E
:1096F000CDB7DEB72C970FB6F894DEBF0FBECDBF47
:109700006C01762EF72F842FE52FB901A801D60121
:109710001496AD90BC9015979091D90591110AC0FF
:109720002DE738E1482F672DC6010E94513A80E0AD
:1097300090E019C0DA82C9827B82FC838D83EE833C
:1097400018861F82FA86E9861C861B8609E41AE4BD
:109750009E012F5F3F4FC501DDDEB501C6010E94AE
:10976000093B8F8198852C960FB6F894DEBF0FBE0B
:10977000CDBFDF91CF911F910F91FF90EF90DF90C0
:10978000CF90BF90AF907F900895CF92DF92EF92ED
:10979000FF920F931F93CF93DF93CDB7DEB72C9734
:1097A0000FB6F894DEBF0FBECDBF7C01C901F70133
:1097B000C480D5802091D905211108C02DE538E15C
:1097C000C7010E94513A80E090E01CC0FA82E98211
:1097D0006B837C834D835E8318861F821A8709877B
:1097E0001C861B8609E41AE49E012F5F3F4F41EB64
:1097F0005FE7BC01C60121DFB601C7010E94093B3A
:109800008F8198852C960FB6F894DEBF0FBECDBF22
:10981000DF91CF911F910F91FF90EF90DF90CF904C
:109820000895CF92DF92EF92FF920F931F93CF9301
:10983000DF93CDB7DEB72C970FB6F894DEBF0FBE1F
:10984000CDBF7C01C901F701C480D5802091D90525
:10985000211108C02DE338E1C7010E94513A80E090
:1098600090E01CC0FA82E9826B837C834D835E8327
:1098700018861F821A8709871C861B8609E41AE44A
:109880009E012F5F3F4F44EB5FE7BC01C601D5DE71
:10989000B601C7010E94093B8F8198852C960FB6AF
:1098A000F894DEBF0FBECDBFDF91CF911F910F9116
:1098B000FF90EF90DF90CF900895CF93DF93EC016E
:1098C000262F4CAD6BAD04960E94FC392BAD082EB3
:1098D000000C990B820F911D8BAF81E090E0DF911E
:1098E000CF9108950F939CE0899F802D112421E052
:1098F000280F2093E105845F8093E00590E00296B5
:1099000040911A0650E08417950714F480E033C0A4
:10991000822F90E020911C0630E082179307B4F765
:109920006623A9F061E086EE95E00E9485364091BD
:10993000E1054E5F0BE020E860E086EE95E00E94D6
:10994000793860E086EE95E00E94853605C061E0DA
:1099500086EE95E00E9485366091E00580911A06BA
:109960006817A0F29091E10580911C06891770F2AA
:1099700080E0DBDC81E00F910895CF93DF93FC0161
:1099800085ADEF012496811105C081E085AFCE0140
:109990000E942C36CE01DF91CF910C9463366FEF8D
:1099A0007FEF19CD6FEF7FEFF9CC4FEF5FEFC2CCB8
:1099B000482F50E02091DF05022E000C330B421798
:1099C000530781F08093DF05813031F468E571E25F
:1099D00086EE95E00C94093B68E679E186EE95E029
:1099E0000C94093B0895EF92FF920F9382EE95E05D
:1099F000C4DF8AE1E82E8FE1F82E00E428E040E0A1
:109A000060E086EE95E00E94AF366BEB74E086EE88
:109A100095E00E94093B26E433E041E169E386EEEC
:109A200095E00E941A3A6BE27DE086EE95E00E9496
:109A3000093B2DE433E04CE16AE386EE95E00E94B9
:109A40001A3A66E870E186EE95E00E94093B2DE542
:109A500033E049E26BE386EE95E00E941A3A66E84D
:109A600070E186EE95E00E94093B29E633E04EE383
:109A70006DE386EE95E00E941A3A2BE633E04EE362
:109A800062E486EE95E00E941A3A86EE95E00E9426
:109A900067368111AECF64EC79E080E090E00E94FF
:109AA000CD9E68E679E186EE95E00F91FF90EF900C
:109AB0000C94093B61E08AE19FE195DF64EC79E079
:109AC00080E090E00C94CD9ECF92DF92EF92FF92D7
:109AD0000F931F93CF93DF93EDDFC091E6050091C5
:109AE000E705D0E0BE016853710977FF02C06F5FE0
:109AF0007F4F75956795D62E82EE95E03EDFCE01BD
:109B0000C69796958795182FC257D109D695C795B0
:109B10004EEEC42EC00EDAEFD00F85E9E82E8EE1AE
:109B2000F82E03E127E04CE06D2D86EE95E00E94D3
:109B3000AF3683E03DDF2BE633E04C2D612F86EE20
:109B400095E00E941A3A25E733E04D2F6C2F86EE00
:109B500095E00E941A3A86EE95E00E9467368111E0
:109B6000DCCF64EC79E080E090E0DF91CF911F9151
:109B70000F91FF90EF90DF90CF900C94CD9E60E01E
:109B800070E088E591E29DCD1F93CF93DF930E9413
:109B90009945C091E705C695C69582EE95E0EDDE44
:109BA000DC2FDD0F1D2F1C0F83E002DF6C2F80E008
:109BB000BCDB83EA97E0F6DE6D2F80E0B6DB8AEA55
:109BC00098E1EDDE612F80E0B0DB8DE998E1E7DE22
:109BD00086EE95E00E9467368111E6CFDF91CF9146
:109BE0001F9108950895CF93E62F6CE0869F602D16
:109BF000112481E0860F8093E105645F6093E005A6
:109C0000462F50E04E5F5F4F20911A0630E042171A
:109C100053070CF445C090E020911C0630E08217F9
:109C200093070CF03DC0CE2F8EE37FDB65E470E040
:109C300080E090E0BADE61E36C0F062E000C770B3B
:109C4000880B990BB2DE60E270E080E090E0ADDE60
:109C500060917C0D70917D0D80917E0D90917F0DB6
:109C60000F94D36CCB010E94D89F9CDE6FE270E012
:109C700080E090E09ADE0E945982811109C085E05F
:109C8000C89FF0011124E559F24F8481811108C069
:109C90008091800D9091810D0E94D89FCF9182CEAE
:109CA000CF910895CF92DF92EF92FF920F931F937F
:109CB000CF93DF931F921F92CDB7DEB77B01622F48
:109CC000498310DE4981882309F440C0442309F107
:109CD00001151105F1F4C7010E94878126E130E0EA
:109CE000281B310937FF02C02F5F3F4F359527955D
:109CF00030E82158822F830F87FD0CC060E270E0AE
:109D000080E090E02A83398350DE398131502A8106
:109D1000F1CF30E8C32ED12CB601C7015CDB760150
:109D2000E81AF90A0115110511F41E2D06C0FF24C9
:109D3000B701C80133DB1E2D181B173038F060E265
:109D400070E080E090E031DE181BF7CF0F900F90AD
:109D5000DF91CF911F910F91FF90EF90DF90CF9007
:109D600008950F93CF93DF93982F862FEA01692FE1
:109D7000B9DD882309F168E770E0CE012CDBC8E784
:109D8000C81BC73038F060E270E080E090E00DDE84
:109D9000C81BF7CF6091E0058AE7C7DA602F000F94
:109DA000770B880B990B01DE60E270E080E090E0B9
:109DB000DF91CF910F91F9CDDF91CF910F91089560
:109DC000CF92DF92EF92FF920F931F93CF93DF9387
:109DD000982F862F6A017901692F84DD882309F481
:109DE00042C0C701002321F00E948781182F03C0C1
:109DF0000E946681182FC4E1D0E0C11BD1098C2FCD
:109E0000880FC80FCC0FD0E0BE01C601E4DAC81B32
:109E10006AE370E080E090E0C8DDC73038F060E2CF
:109E200070E080E090E0C1DDC81BF7CF8AEF189F9B
:109E3000802D11246091E005805877DAC701002356
:109E400049F0DF91CF911F910F91FF90EF90DF903C
:109E5000CF90A5CDDF91CF911F910F91FF90EF9003
:109E6000DF90CF909FCDDF91CF911F910F91FF9009
:109E7000EF90DF90CF900895BF92CF92DF92EF9254
:109E8000FF920F931F93CF93DF936C017B010E948E
:109E90008781C82FC7010E94668104E110E0081B7A
:109EA00011098C2F90E0BB24B394081719071CF0FC
:109EB000B12CC5E201C0CFE12C2F30E0A9014E5FEB
:109EC0005F4F80911A0690E04817590744F02950D7
:109ED000310980911C0690E0821793079CF5D0E031
:109EE000E114F104B1F16AE370E080E090E05DDD3F
:109EF000BB2081F0C45F80911A06C81750F12C2F47
:109F000030E02950310980911C0690E082179307B8
:109F10001CF41FC0DD23E9F0802F880F800F6C2F09
:109F2000880F03DA60E270E080E090E03EDDC70178
:109F3000DF91CF911F910F91FF90EF90DF90CF9025
:109F4000BF9030CD6C2F80E0F0D9C60128DDD1E084
:109F5000C7CFDF91CF911F910F91FF90EF90DF90CE
:109F6000CF90BF900895EF92FF920F93CF93DF931E
:109F7000D82FC62F7901682F8C2FB4DC8823D9F015
:109F8000002329F062E070E080E090E00EDD2D2FEC
:109F90004C2F65E1C7010E940A826EE770E0FED98E
:109FA000CEE7C81BC73038F060E270E080E090E098
:109FB000FCDCC81BF7CFDF91CF910F91FF90EF90A2
:109FC00008958F929F92AF92BF92CF92DF92EF92BD
:109FD000FF920F936B017C018090DB059090DC0574
:109FE000A090DD05B090DE05A50194010F94646C8E
:109FF000882301F120E030E0A901C701B6010F94E8
:10A00000646C882351F0A5019401C701B6010F9437
:10A01000646C87FD04C081E003C080E001C08FEF65
:10A020008093DA05C092DB05D092DC05E092DD0575
:10A03000F092DE0580911A06813128F480911C0689
:10A04000833008F048C080911A06853128F4809149
:10A050001C06843108F04FC080911A068F3308F037
:10A0600057C080911C068F3208F452C088E0E82E59
:10A0700089E1F82E00E123E04FE265E086EE95E00D
:10A080000E94AF3698E3E92E99E1F92E23E04FE2E2
:10A090006AE586EE95E00E94AF368091DA0540E3EE
:10A0A000481B2EEEE22E28E1F22E0DE022E06EE6B5
:10A0B00086EE95E00E94AF368091DA0541E3481BB9
:10A0C00034EDE32E38E1F32E22E069E186EE95E0EF
:10A0D0000E94AF361DC08091DA0544E0481B59EB61
:10A0E000E52E58E1F52E0CE022E062E486EE95E0E4
:10A0F0000E94AF36A8CF41EDE42E48E1F42E01E0F6
:10A1000023E044E16CE386EE95E00E94AF36A4CFF5
:10A110000F91FF90EF90DF90CF90BF90AF909F9006
:10A120008F900895CF92EF920F93CF93DF93C2EE6B
:10A13000D5E01B821A828DE893E099838883CC2432
:10A14000CA94EE24EA9402E522E143E165E172E07B
:10A15000CE010E94C93B89E993E099838883DF910E
:10A16000CF910F91EF90CF9008955A9887FD52C0EC
:10A170005B9800000000000000005A9A5A98282FAF
:10A18000220F86FD53C05B98000000000000000015
:10A190005A9A5A98922F990F26FD46C05B98000054
:10A1A0000000000000005A9A5A98892F880F96FDE7
:10A1B00039C05B9800000000000000005A9A5A98CD
:10A1C000982F990F86FD2CC05B98000000000000BE
:10A1D00000005A9A5A98892F880F96FD1FC05B98E5
:10A1E00000000000000000005A9A5A98982F990F1A
:10A1F00086FD12C05B9800000000000000005A9A23
:10A200005A9896FD15C05B98000000000000000001
:10A210005A9A08955B9AADCF5B9AEDCF5B9AE0CFE7
:10A220005B9AD3CF5B9AC6CF5B9AB9CF5B9AACCF20
:10A230005B9AEACF2F923F925F927F929F92AF926A
:10A24000BF92CF92DF92EF92FF920F931F93CF9323
:10A25000DF937C011B01942E69018AE0481709F401
:10A260007BC0A5E14A134EC0DB011296ED91FC9133
:10A2700013971281C681D7815D9A88E28A95000082
:10A28000E9F700EE010F80E1582E510E98E2792E89
:10A2900088EF6BDF872D8A950000E9F7103208F010
:10A2A00046C0812F8077806860DF812F8295807F14
:10A2B0005CDF872D8A950000E9F780E856DF80E0B3
:10A2C00054DF872D8A950000E9F78AEF4EDF872D4E
:10A2D0008A950000E9F75E01B0E1AB0EB11C888100
:10A2E000807F43DF89918295807F3FDFCA15DB0540
:10A2F000B1F7872D8A950000E9F71F5F0F5F1511F1
:10A30000C7CF5D989601492DB101C701DF91CF916B
:10A310001F910F91FF90EF90DF90CF90BF90AF9083
:10A320009F907F905F903F902F900C94E937802F03
:10A33000807780681ADF802F8295807F16DF872DD7
:10A340008A950000E9F780E810DF80E80EDF872DAE
:10A350008A950000E9F7B9CF559A5D98539A5B98B2
:10A36000529A5A9A5D9AC8E28C2F8A950000E9F7B2
:10A3700088E790E00E94063788EFF7DE8C2F8A95F9
:10A380000000E9F780E2F1DE80E0EFDE8C2F8A95B5
:10A390000000E9F780E0E9DE80E8E7DE8C2F8A95AF
:10A3A0000000E9F780E0E1DE80E1DFDE8C2F8A95B6
:10A3B0000000E9F78FE090E00E94063780E2D5DEEA
:10A3C00080E4D3DE8C2F8A950000E9F780E2CDDEB1
:10A3D00080E6CBDECA950000E9F710E0D8E208E29B
:10A3E000812F80778068C1DE812F8295807FBDDEDE
:10A3F0008D2F8A950000E9F780E8B7DE80E0B5DEB2
:10A400008D2F8A950000E9F78AEFAFDE8D2F8A95B0
:10A410000000E9F7C0E280E0A8DE80E0A6DE9D2F24
:10A420009A950000E9F7C150B1F788EF9EDE802FC2
:10A430008A950000E9F71F5F103209F0D1CF80E064
:10A4400094DE80EC92DE88E28A950000E9F75D9860
:10A4500059CF0E94CA8F41E050E060E070E0811166
:10A4600003C040E050E0BA0140939507509396072F
:10A47000609397077093980710926F0781E080931D
:10A48000490783E0809323020895CF92DF92EF92F1
:10A49000FF920F931F93CF93DF930E94C7906C019D
:10A4A00061E081E00E948478C0916F07D0E081E094
:10A4B000C81AD108C11117C080913807811104C092
:10A4C0000E94548281119BC080912302882359F0FD
:10A4D00081E090913807911180E004E024E044E7A6
:10A4E0005AE26D2F3EDC6CEF79E083E899E00E9440
:10A4F000AE968091FC098F3201F18091090A83FFA9
:10A500001CC0C130C1F480913807813021F40E9411
:10A51000548281117CC080912302882361F081E004
:10A5200090913807913009F080E000E22EE340E797
:10A530005AE26D2F16DC92E001C091E08091230277
:10A54000882309F454C0760111E01C0F8FEFE81640
:10A55000F80609F44CC0C91345C060E070E0C701BB
:10A560000E94EF8C9091090A8091380794FF22C0D5
:10A570008C1354C00E945482882309F44FC08CEF7E
:10A5800099E00E94748F10926F0782E090E0A0E043
:10A59000B0E08093950790939607A0939707B093A8
:10A5A000980781E08093490710929A0783E080938F
:10A5B000230250C08C1304C00E94548281113DC0FC
:10A5C00080912302882361F081E0909138079C13E9
:10A5D00080E000E020EB39E144E55AE26D2FC3DC76
:10A5E000912F01C09F5F81E0E81AF108AFCFDF5FD4
:10A5F000CF5FD53009F05ECF909337072BC00E9414
:10A60000C97780914907882309F45ECF23C021DFF1
:10A6100080914907882309F47ECF1CC080912302D2
:10A620008823F1F281E0909138079C1380E001E0EB
:10A6300020EB39E142E65AE2D1CF8CEF99E00E945B
:10A640007A8B0E94C3770E94FD86809149078823F8
:10A6500009F4B6CFDF91CF911F910F91FF90EF904A
:10A66000DF90CF900895CF93DF93EC01CB01BA0137
:10A670000F94066D0F94D86C6883DF91CF91089585
:10A68000CF93DF93EC01CB01BA010F94066D2FE657
:10A6900032E143E85AE30F94A26E688379838A8398
:10A6A0009B83DF91CF91089563E373E580E693E5A3
:10A6B0000C94DD7760E473E58DE793E50C94DD772A
:10A6C0000F94066D0F94D86C862F0C94119FCF9326
:10A6D000DF9300D01F92CDB7DEB769837A838B8377
:10A6E0009C8360E2CE0101960E9450A10F900F90D2
:10A6F0000F900F90DF91CF9108950F94066D2FE684
:10A7000032E143E85AE30F94A26EE1CF2F923F92D9
:10A710004F925F926F927F928F929F92AF92BF9271
:10A72000CF92DF92EF92FF920F931F93CF93DF931D
:10A73000CDB7DEB727970FB6F894DEBF0FBECDBFFB
:10A740001C017F836E83CA01B901E982FA820B83FF
:10A750001C839C2C8D2CAD8220E030E04AE754E431
:10A760000F94A26E0F94D36C2B013C0120E030E0DB
:10A770004AE754E4EE81FF81608171818281938197
:10A780000F94A26E0F94D36C5B016C01A418B508F2
:10A79000C608D70820E030E04AE754E4C801B70112
:10A7A0000F94A26E0F94D36C7B018C01E418F50812
:10A7B00006091709FD81FF938F929F928AE5882EE3
:10A7C00083E5982EA30192016E817F81C1010E94D1
:10A7D00044760F900F900F9027960FB6F894DEBF37
:10A7E0000FBECDBFDF91CF911F910F91FF90EF90E2
:10A7F000DF90CF90BF90AF909F908F907F906F90A1
:10A800005F904F903F902F9008958F929F92AF92BC
:10A81000BF92CF92DF92EF92FF920F931F93CF934D
:10A82000DF9361E081E00E948478D0916F07C0E0FF
:10A83000D11119C080913807811104C00E9454823F
:10A840008111C4C080912302882309F4B6C081E03D
:10A8500090913807911180E004E024E04FEA5AE239
:10A860006C2F7FDAAAC0D130E1F4809138078130B3
:10A8700021F40E9454828111B1C080912302882367
:10A8800009F49BC011E080913807813009F010E095
:10A890008091E7150E94119F00E09C0149E95AE26E
:10A8A00089C0D23009F580913807823021F40E94A6
:10A8B00054828111B8C080912302882309F47DC09D
:10A8C00011E080913807823009F010E06091E815BE
:10A8D0007091E9158091EA159091EB15F8DE00E092
:10A8E0009C0145E95AE266C0D33009F580913807EA
:10A8F000833021F40E9454828111AEC080912302E2
:10A90000882309F45AC011E080913807833009F098
:10A9100010E06091EC157091ED158091EE1590911D
:10A92000EF15D5DE00E09C0141E95AE243C0D43086
:10A9300001F580913807843021F40E9454828111FE
:10A94000A4C0809123028823C1F111E080913807CF
:10A95000843009F010E06091F0157091F11580914C
:10A96000F2159091F315B3DE00E09C014DE85AE238
:10A9700021C0D53011F580913807853021F40E942F
:10A98000548281119BC0809123028823B1F011E091
:10A9900080913807853009F010E060918102709154
:10A9A0008202809183029091840291DE00E09C01FA
:10A9B00049E75AE26C2F812F03DACF5FDF5FC530A2
:10A9C00009F036CF86E08093370790C00E94C977A0
:10A9D00080914907882309F435CF88C081E00E941F
:10A9E0004982A090E715B12CC12CD12C1F921F9247
:10A9F0001F9244E5842E43E5942EE12CF12C87012F
:10AA0000EA9420E030E0A90167EE75E184EA9AE279
:10AA10000E9444760F900F900F90809149078823F1
:10AA200009F42BCF63C081E00E944982A12CC12C84
:10AA3000D12C16E6E12EFE2C0EE111E420E030E0F0
:10AA4000A90168EE75E187E99AE260DE8091490725
:10AA5000882309F430CF4AC081E00E944982A12CAA
:10AA6000C12CD12C16E6E12EFE2C0EE111E420E0E3
:10AA700030E0A9016CEE75E183E99AE247DE80914E
:10AA80004907882309F43ACF31C081E00E94498206
:10AA9000A12CC12CD12C16E6E12EFE2C0EE111E4E6
:10AAA00020E030E0A90160EF75E18FE89AE22EDE48
:10AAB00080914907882309F444CF18C081E00E949F
:10AAC0004982A12CC12CD12C16E6E12EFE2C0EE1E0
:10AAD00011E420E030E0A90161E872E083E89AE245
:10AAE00015DE80914907882309F44DCFDF91CF917E
:10AAF0001F910F91FF90EF90DF90CF90BF90AF909C
:10AB00009F908F900895CF93DF93EC01CB01BA0112
:10AB10000F94066D2AE037ED43E25CE30F94A26EDA
:10AB2000688379838A839B83DF91CF910895CF9344
:10AB3000DF93EC01CB01BA010F94066D6883798332
:10AB40008A839B83DF91CF910895CF93DF93EC01AC
:10AB5000CB01BA010F94066D20E030E048EC52E4DE
:10AB60000F94A26E688379838A839B83DF91CF9150
:10AB70000895CF93DF93EC01CB01BA010F94066DDA
:10AB800020E030E048EC52E40F94A26E0F94D86CB1
:10AB9000688379838A839B83DF91CF910895CF93D4
:10ABA000DF93EC01CB01BA010F94066D2AE037ED7B
:10ABB00043E25CE30F94A26E688379838A839B836C
:10ABC000DF91CF91089563E875E582E296E50C94F4
:10ABD000DD7767E975E58FE796E50C94DD7765EA43
:10ABE00075E58FE396E50C94DD7769EB75E58BE908
:10ABF00096E50C94DD776FEC75E585E096E50C94B1
:10AC0000DD770D94691E0D94B01ECF93DF9300D0B5
:10AC10001F92CDB7DEB70F94066D2AE037ED43E201
:10AC20005CE30F94A26E69837A838B839C83CE014D
:10AC300001960E94A0A20F900F900F900F90DF91AD
:10AC4000CF910895CF93DF9300D01F92CDB7DEB799
:10AC50000F94066D2AE037ED43E25CE30F94A26E99
:10AC600069837A838B839C83CE0101960E943AA0EC
:10AC70000F900F900F900F90DF91CF910895CF9389
:10AC8000DF9300D01F92CDB7DEB70F94066D20E0A2
:10AC900030E048EC52E40F94A26E69837A838B8390
:10ACA0009C83CE0101960E94E8A10F900F900F9017
:10ACB0000F90DF91CF910895CF92DF92EF92FF92A4
:10ACC0006B017C0120E030E0A9010F94646C87FDEA
:10ACD00005C020E030E040E05FE304C020E030E069
:10ACE00040E05FEBC701B6010F948B6B0F94D36C00
:10ACF000CB01FF90EF90DF90CF900C94D89F0F94F2
:10AD0000066DDACFCF93DF9300D01F92CDB7DEB7B9
:10AD10000F94D86C0F94046D69837A838B839C8322
:10AD2000CE0101960E94E8A10F900F900F900F9016
:10AD3000DF91CF9108950F94066D20E030E048EC4C
:10AD400052E40F94A26EDECFCF93DF931F921F9237
:10AD5000CDB7DEB789839A830E94227640E050E027
:10AD6000BA0189819A810F900F90DF91CF910C9455
:10AD70009E770F931F93CF93DF9361E081E00E9452
:10AD80008478C0916F07D0E0C1111AC08091380754
:10AD9000811104C00E9454828111E8C08091230275
:10ADA000882309F461C081E090913807911180E017
:10ADB00004E024E046EF5AE26D2F0E94B14E54C0E9
:10ADC000C130D9F480913807813021F40E94548237
:10ADD0008111D4C080912302882309F445C081E009
:10ADE00090913807913009F080E003E02EE34DEEBA
:10ADF0005AE26D2F0E94B14E37C0C230D1F480911B
:10AE00003807823021F40E9454828111C0C08091A1
:10AE10002302882349F181E090913807923009F0AC
:10AE200080E003E02EE340EE5AE26D2F0E94B14E27
:10AE30001BC0C330C9F480913807833021F40E94CD
:10AE400054828111ADC080912302882369F081E092
:10AE500090913807933009F080E003E02EE34BED4A
:10AE60005AE26D2F0E94B14E0E94877781111DC05A
:10AE7000C430E9F480913807843021F40E94548270
:10AE8000811197C080912302882309F49BC081E03F
:10AE900090913807943009F080E003E02EE342ED12
:10AEA0005AE26D2F0E94B14E8DC014E001C015E032
:10AEB000C1131BC0809138078C1304C00E945482B8
:10AEC000811182C080912302882371F081E09091EA
:10AED00038079C1380E003E02EE349EC5AE26D2F23
:10AEE0000E94B14E1C2F01C01C2F81E0810FC8139E
:10AEF00018C0809138078C1304C00E9454828111BD
:10AF00006CC080912302882361F081E09091380722
:10AF10009C1380E003E02EE34DEB5AE26D2F0E947C
:10AF2000B14E82E0810FC81318C0809138078C138E
:10AF300004C00E945482811159C080912302882349
:10AF400061F081E0909138079C1380E003E02EE3EC
:10AF500044EB5AE26D2F0E94B14EDF5FCF5FD530D8
:10AF600009F012CF1D5F1093370748C00E94C977C0
:10AF700080914907882309F411CF40C08CEA99E5F4
:10AF8000E3DE80914907882309F424CF37C08BE49E
:10AF90009FE5DADE80914907882309F438CF2EC077
:10AFA00083EC9CE5D1DE80914907882309F44BCFDF
:10AFB00025C084E79BE5C8DE80914907882309F412
:10AFC00061CF1CC015E091CF85E094E5BDDE809196
:10AFD0004907882309F476CF11C080E09DE7B4DEED
:10AFE00080914907882309F48CCF08C086E798E54B
:10AFF000ABDE80914907882309F49FCFDF91CF9181
:10B000001F910F9108952F923F924F925F926F92EE
:10B010007F928F929F92AF92BF92CF92DF92EF92E8
:10B02000FF920F931F93CF93DF93CDB7DEB7279790
:10B030000FB6F894DEBF0FBECDBF1C017F836E83B9
:10B040009C2C8D2CA982CA01B9010F94D36C9B0151
:10B05000AC01EE81FF8160817181828193812A83BD
:10B060003B834C835D830F94D36C2A813B814C815D
:10B070005D815B016C01A21AB30AC40AD50AC8013A
:10B08000B7010F94D36C2A813B814C815D817B0198
:10B090008C01E21AF30A040B150BF981FF938F92CE
:10B0A0009F9289EE882E85E5982E6E817F81C10161
:10B0B0000E9444760F900F900F9027960FB6F89449
:10B0C000DEBF0FBECDBFDF91CF911F910F91FF90DB
:10B0D000EF90DF90CF90BF90AF909F908F907F9038
:10B0E0006F905F904F903F902F9008956F927F9256
:10B0F0008F929F92AF92BF92CF92DF92EF92FF9288
:10B100000F931F93CF93DF9300D01F92CDB7DEB77D
:10B1100061E081E00E94847860906F07712C61107B
:10B120001AC080913807811104C00E945482811195
:10B1300098C080912302882309F48AC081E090910D
:10B140003807911180E004E024E044ED5CE2672DD3
:10B150000E94B14E7DC081E068122CC080913807FA
:10B16000813021F40E945482811183C08091230296
:10B17000882309F46DC011E080913807813009F00F
:10B1800010E08091650F9091660FA091670FB091CC
:10B19000680F89839A83AB83BC83CE0101960E949A
:10B1A0003AA000E09C0140EC5CE2672D812F0E94F8
:10B1B000E04E4EC082E0681225C080913807823090
:10B1C00021F40E945482811185C08091230288233A
:10B1D00009F43EC011E080913807823009F010E098
:10B1E0006091D70C7091D80C8091D90C9091DA0CA9
:10B1F00063DD00E09C014CEA5CE2672D812F0E9438
:10B20000E04E26C083E0681223C080913807833067
:10B2100021F40E945482811175C0809123028823F9
:10B22000B9F011E080913807833009F010E06091A7
:10B23000DB0C7091DC0C8091DD0C9091DE0C3CDD20
:10B2400000E09C014CE95CE2672D812F0E94E04EFA
:10B250007394639485E0781262CF84E0809337071B
:10B2600068C00E94C97780914907882309F461CF9B
:10B2700060C020E030E048EC52E46091650F7091CE
:10B28000660F8091670F9091680F0F94A26E0F94D4
:10B29000D36C1F921F921F9223EE822E25E5922ED1
:10B2A0005B016C011CE3E12E16E8F12E01E010E0D9
:10B2B00020E030E0A90165E67FE08AEC9CE20E9494
:10B2C00044760F900F900F9080914907882309F4DE
:10B2D0004DCF2FC081E00E944982A12CC12CD12CDE
:10B2E000E12CF12C08E413E420E030E0A90167ED43
:10B2F0007CE086EB9CE287DE80914907882309F495
:10B3000064CF17C081E00E944982A12CC12CD12CAE
:10B31000E12CF12C08E413E420E030E0A9016BED0E
:10B320007CE084EA9CE26FDE80914907882309F47F
:10B3300074CF0F900F900F900F90DF91CF911F91CE
:10B340000F91FF90EF90DF90CF90BF90AF909F90C4
:10B350008F907F906F900895AF92CF92DF92EF928F
:10B36000FF920F931F93CF93DF9361E081E00E94E0
:10B370008478D0916F07C0E0D1111AC0809138074E
:10B38000811104C00E945482811103C18091230263
:10B39000882309F4F5C081E090913807911180E08D
:10B3A00004E024E04AE85CE26C2F0E94B14EE8C061
:10B3B000D13029F580913807813021F40E945482E0
:10B3C0008111EFC080912302882309F4D9C011E0D4
:10B3D00080913807813009F010E06091171070916A
:10B3E00018108091191090911A1066DC00E09C01F1
:10B3F0004CE75CE26C2F812F0E94E04EC1C0D2303E
:10B4000029F580913807823021F40E9454828111FD
:10B41000E2C080912302882309F4B2C011E0809138
:10B420003807823009F010E060911B1070911C10F9
:10B4300080911D1090911E103FDC00E09C014EE6B3
:10B440005CE26C2F812F0E94E04E9AC0D33029F528
:10B4500080913807833021F40E9454828111D5C035
:10B4600080912302882309F48BC011E08091380772
:10B47000833009F010E060911F10709120108091CE
:10B4800021109091221018DC00E09C0140E65CE263
:10B490006C2F812F0E94E04E73C0D43029F580912B
:10B4A0003807843021F40E9454828111C8C08091F1
:10B4B0002302882309F464C011E0809138078430A6
:10B4C00009F010E0609123107091241080912510F4
:10B4D00090912610F1DB00E09C0142E55CE26C2FCC
:10B4E000812F0E94E04E4CC0D53029F5809138075D
:10B4F000853021F40E9454828111BBC080912302C7
:10B50000882309F43DC011E080913807853009F0A7
:10B5100010E060913310709134108091351090914B
:10B520003610CADB00E09C0148E45CE26C2F812FFE
:10B530000E94E04E25C0D63019F58091380786303C
:10B5400021F40E9454828111ADC08091230288238E
:10B55000B9F011E080913807863009F010E0609171
:10B560003710709138108091391090913A10A4DB07
:10B5700000E09C0144E35CE26C2F812F0E94E04ECE
:10B58000CF5FDF5FC53009F0F7CE87E080933707E4
:10B59000A1C00E94C97780914907882309F4F6CE9B
:10B5A00099C081E00E944982A12CC12CD12CE12CB0
:10B5B00010ECF12E09E714E420E030E040E85FE30E
:10B5C00067E170E183E89CE21EDD809149078823F2
:10B5D00009F4F8CE7FC081E00E944982A12CC12CE1
:10B5E000D12CE12C10ECF12E09E714E420E030E03E
:10B5F00040E85FE36BE170E185E79CE204DD809168
:10B600004907882309F405CF65C081E00E9449827B
:10B61000A12CC12CD12CE12C10ECF12E09E714E463
:10B6200020E030E040E85FE36FE170E187E69CE214
:10B63000EADC80914907882309F412CF4BC081E0EE
:10B640000E944982A12CC12CD12CE12C10ECF12EAE
:10B6500009E714E420E030E040E85FE363E270E1F2
:10B6600089E59CE2D0DC80914907882309F41FCF4B
:10B6700031C081E00E944982A12CC12CD12CE12C47
:10B6800010ECF12E09E714E420E030E0A90163E3B7
:10B6900070E18DE49CE2B7DC80914907882309F4CE
:10B6A0002DCF18C081E00E944982A12CC12CD12C41
:10B6B000E12C10ECF12E09E714E420E030E0A901C0
:10B6C00067E370E18EE39CE29EDC8091490788236A
:10B6D00009F43BCFDF91CF911F910F91FF90EF9035
:10B6E000DF90CF90AF900895AF92CF92DF92EF921C
:10B6F000FF920F931F93CF93DF9361E081E00E944D
:10B700008478D0916F07C0E0D1111AC080913807BA
:10B71000811104C00E9454828111B4C0809123021F
:10B72000882309F4A7C081E090913807911180E047
:10B7300004E024E044E55BE26C2F0E94B14E9AC025
:10B74000D13029F580913807813021F40E9454824C
:10B750008111A0C080912302882309F48BC011E0DD
:10B7600080913807813009F010E0609107107091E6
:10B7700008108091091090910A109EDA00E09C0157
:10B7800040E45BE26C2F812F0E94E04E73C0D23008
:10B7900029F580913807823021F40E94548281116A
:10B7A00095C080912302882309F464C011E0809140
:10B7B0003807823009F010E060910B1070910C1086
:10B7C00080910D1090910E1077DA00E09C014CE210
:10B7D0005BE26C2F812F0E94E04E4CC0D33029F5E4
:10B7E00080913807833021F40E94548281118AC0ED
:10B7F00080912302882309F43DC011E0809138072D
:10B80000833009F010E060910F107091101080915A
:10B8100011109091121050DA00E09C0148E15BE2B7
:10B820006C2F812F0E94E04E25C0D43019F58091F5
:10B830003807843021F40E94548281117FC08091A6
:10B8400023028823B9F011E080913807843009F091
:10B8500010E0609113107091141080911510909168
:10B8600016102ADA00E09C0144E05BE26C2F812F85
:10B870000E94E04ECF5FDF5FC53009F045CFC09337
:10B88000370777C00E94C97780914907882309F458
:10B8900045CF6FC081E00E944982A12C63E0C62E93
:10B8A00066E5D62EE12C1CE3F12E0CE116E420E037
:10B8B00030E040EA50E467E070E18AE49BE2A3DB19
:10B8C00080914907882309F445CF53C081E00E9445
:10B8D0004982A12C43E0C42E46E5D42EE12C1CE382
:10B8E000F12E0CE116E420E030E040EA50E46BE099
:10B8F00070E186E39BE287DB80914907882309F4A6
:10B9000050CF37C081E00E944982A12C23E0C22E93
:10B9100026E5D22EE12C1CE3F12E0CE116E420E00A
:10B9200030E040EA50E46FE070E182E29BE26BDBE2
:10B9300080914907882309F45BCF1BC081E00E94F6
:10B940004982A12C83E0C82E86E5D82EE12C1CE389
:10B95000F12E0CE116E420E030E040EA50E463E12F
:10B9600070E18EE09BE24FDB80914907882309F468
:10B9700066CFDF91CF911F910F91FF90EF90DF90F5
:10B98000CF90AF9008956F927F928F929F92AF92D7
:10B99000BF92CF92DF92EF92FF920F931F93CF93BC
:10B9A000DF9300D01F92CDB7DEB761E081E00E9447
:10B9B000847860906F07712C61101AC080913807ED
:10B9C000811104C00E9454828111BFC08091230262
:10B9D000882309F4B2C081E090913807911180E08A
:10B9E00004E024E046EA5BE2672D0E94B14EA5C068
:10B9F00021E0621225C080913807813021F40E9435
:10BA000054828111AAC080912302882309F495C031
:10BA100011E080913807813009F010E06091C30F88
:10BA20007091C40F8091C50F9091C60F45D900E069
:10BA30009C0146E95BE2672D812F0E94E04E7DC0AC
:10BA400082E0681225C080913807823021F40E947C
:10BA5000548281119CC080912302882309F46DC017
:10BA600011E080913807823009F010E06091C70F33
:10BA70007091C80F8091C90F9091CA0F1DD900E035
:10BA80009C0146E85BE2672D812F0E94E04E55C085
:10BA900023E062122CC080913807833021F40E9489
:10BAA000548281118EC080912302882309F445C0FD
:10BAB00011E080913807833009F010E08091CB0FBE
:10BAC0009091CC0FA091CD0FB091CE0F89839A8326
:10BAD000AB83BC83CE0101960E94A0A200E09C0132
:10BAE00046E75BE2672D812F0E94E04E26C084E08E
:10BAF000681223C080913807843021F40E94548258
:10BB0000811199C0809123028823B9F011E08091BE
:10BB10003807843009F010E06091CF0F7091D00F9A
:10BB20008091D10F9091D20FC7D800E09C0146E6DA
:10BB30005BE2672D812F0E94E04E7394639425E0B1
:10BB400072123ACF709237078FC00E94C9778091E6
:10BB50004907882309F43ACF87C081E00E944982CF
:10BB6000A12CC12CD12CE12C10E8F12E07E714E414
:10BB700020E030E040E85FE363EC7FE08EE99BE2A9
:10BB800042DA80914907882309F43DCF6DC081E0F6
:10BB90000E944982A12CC12CD12CE12C10E8F12E5D
:10BBA00007E714E420E030E040E85FE367EC7FE083
:10BBB0008EE89BE228DA80914907882309F44BCF6D
:10BBC00053C081E00E94498220E030E048EC52E41A
:10BBD0006091CB0F7091CC0F8091CD0F9091CE0FD3
:10BBE0000F94A26E0F94D36C5B016C012AE0A21A31
:10BBF000B108C108D1081F921F921F929BEF892E96
:10BC000095E5992E1EEAE12E12E8F12E01E010E0F2
:10BC10002AE030E040E050E06BEC7FE08EE79BE212
:10BC20000E9444760F900F900F90809149078823CF
:10BC300009F439CF19C081E00E944982A12CC12C9E
:10BC4000D12CE12C10E8F12E07E714E420E030E0DD
:10BC500040E85FE36FEC7FE08EE69BE2D4D9809111
:10BC60004907882309F44ECF0F900F900F900F9043
:10BC7000DF91CF911F910F91FF90EF90DF90CF90C8
:10BC8000BF90AF909F908F907F906F9008952F926C
:10BC90003F924F925F926F927F928F929F92AF925C
:10BCA000BF92CF92DF92EF92FF920F931F93CF93A9
:10BCB000DF93CDB7DEB727970FB6F894DEBF0FBE80
:10BCC000CDBF1C017F836E83CA01B901E982FA826C
:10BCD0000B831C839C2C8D2CAD822AE037ED43E234
:10BCE0005CE30F94A26E0F94D36C2B013C012AE00D
:10BCF00037ED43E25CE3EE81FF81608171818281F7
:10BD000093810F94A26E0F94D36C5B016C01A41805
:10BD1000B508C608D7082AE037ED43E25CE3C8015E
:10BD2000B7010F94A26E0F94D36C7B018C01E418C1
:10BD3000F50806091709FD81FF938F929F928FEEF8
:10BD4000882E85E5982EA30192016E817F81C10125
:10BD50000E9444760F900F900F9027960FB6F8949C
:10BD6000DEBF0FBECDBFDF91CF911F910F91FF902E
:10BD7000EF90DF90CF90BF90AF909F908F907F908B
:10BD80006F905F904F903F902F9008952F923F9229
:10BD90004F925F926F927F928F929F92AF92BF92DB
:10BDA000CF92DF92EF92FF920F931F93CF93DF9387
:10BDB000CDB7DEB727970FB6F894DEBF0FBECDBF65
:10BDC0001C017F836E83E982FA820B831C839C2C87
:10BDD0008D2CAD82CA01B9010F94046D2AE037EDB4
:10BDE00043E25CE30F94A26E0F94D36C2B013C01F1
:10BDF000EE81FF8160817181828193810F94046D56
:10BE00002AE037ED43E25CE30F94A26E0F94D36C0B
:10BE10005B016C01A418B508C608D708C801B701B2
:10BE20000F94046D2AE037ED43E25CE30F94A26EB9
:10BE30000F94D36C7B018C01E418F50806091709EF
:10BE4000FD81FF938F929F9285EF882E85E5982E36
:10BE5000A30192016E817F81C1010E9444760F90FF
:10BE60000F900F9027960FB6F894DEBF0FBECDBF90
:10BE7000DF91CF911F910F91FF90EF90DF90CF90C6
:10BE8000BF90AF909F908F907F906F905F904F90FA
:10BE90003F902F9008959F92AF92BF92CF92DF92E2
:10BEA000EF92FF920F931F93CF93DF9300D01F92D7
:10BEB000CDB7DEB761E081E00E94847890906F0793
:10BEC000B12C91101AC080913807811104C00E94D2
:10BED0005482811152C180912302882309F444C104
:10BEE00081E090913807911180E004E024E042E283
:10BEF0005CE26B2D0E94B14E37C181E098122CC0DC
:10BF000080913807813021F40E94548281113DC113
:10BF100080912302882309F427C111E0809138071A
:10BF2000813009F010E08091271090912810A091A5
:10BF30002910B0912A1089839A83AB83BC83CE01E8
:10BF400001960E94E8A100E09C0146E15CE26B2DB5
:10BF5000812F0E94E04E08C182E098122CC080918F
:10BF60003807823021F40E945482811128C18091C7
:10BF70002302882309F4F8C011E080913807823049
:10BF800009F010E080912B1090912C10A0912D10B1
:10BF9000B0912E1089839A83AB83BC83CE01019626
:10BFA0000E94E8A100E09C0142E05CE26B2D812F41
:10BFB0000E94E04ED9C083E098122CC080913807CF
:10BFC000833021F40E945482811113C18091230295
:10BFD000882309F4C9C011E080913807833009F043
:10BFE00010E080912F1090913010A0913110B091FD
:10BFF000321089839A83AB83BC83CE0101960E9461
:10C00000E8A100E09C0140EF5BE26B2D812F0E94D4
:10C01000E04EAAC084E0981228C08091380784308E
:10C0200021F40E9454828111FEC080912302882352
:10C0300009F49AC011E080913807843009F010E0CB
:10C040006091F30F7091F40F8091F50F9091F60FBE
:10C050000F94046D0E94825600E09C0142EE5BE268
:10C060006B2D812F0E94E04E7FC085E0981228C082
:10C0700080913807853021F40E9454828111F0C0EC
:10C0800080912302882309F46FC011E08091380762
:10C09000853009F010E06091F70F7091F80F8091F2
:10C0A000F90F9091FA0F0F94046D0E94825600E0F0
:10C0B0009C0144ED5BE26B2D812F0E94E04E54C049
:10C0C00086E0981228C080913807863021F40E94BB
:10C0D00054828111E2C080912302882309F444C074
:10C0E00011E080913807863009F010E06091FB0F75
:10C0F0007091FC0F8091FD0F9091FE0F0F94046DD5
:10C100000E94825600E09C0146EC5BE26B2D812F81
:10C110000E94E04E29C087E0981226C0809138071F
:10C12000873021F40E9454828111D4C0809123026F
:10C130008823D1F011E080913807873009F010E0B2
:10C140006091FF0F7091001080910110909102108A
:10C150000F94046D0E94825600E09C0148EB5BE264
:10C160006B2D812F0E94E04EB394939485E0B8121A
:10C17000A8CE88E080933707C9C00E94C977809114
:10C180004907882309F4A7CEC1C081E00E944982F3
:10C19000A12CC12CD12CE12C1CE5F12E01EC17E4D3
:10C1A00020E030E040E251E467E270E18CE19CE2A3
:10C1B0006EDD80914907882309F4AACEA7C081E0EB
:10C1C0000E944982A12CC12CD12CE12C1CE5F12E1E
:10C1D00001EC17E420E030E048EC52E46BE270E15F
:10C1E0008CE09CE254DD80914907882309F4BFCE9E
:10C1F0008DC081E00E944982A12CC12CD12CE12C60
:10C200001CE5F12E01EC17E420E030E048EC52E4AC
:10C210006FE270E189EF9BE23ADD80914907882364
:10C2200009F4D4CE73C081E00E944982A12C61E060
:10C23000C62E66E5D62E18EBE12E12E8F12E01E0AF
:10C2400010E024E630E040E050E063EF7FE089EE6C
:10C250009BE29CDD80914907882309F4E6CE56C015
:10C2600081E00E944982A12C41E0C42E46E5D42EF3
:10C2700018EBE12E12E8F12E01E010E024E630E0A8
:10C2800040E050E067EF7FE08BED9BE27FDD809147
:10C290004907882309F4F4CE39C081E00E9449821D
:10C2A000A12C21E0C22E26E5D22E18EBE12E12E8B9
:10C2B000F12E01E010E02AE030E040E050E06BEFCA
:10C2C0007FE08DEC9BE262DD80914907882309F4D1
:10C2D00002CF1CC081E00E944982A12C81E0C82EBF
:10C2E00086E5D82E18EBE12E12E8F12E01E010E0E1
:10C2F00024E630E040E050E06FEF7FE08FEB9BE220
:10C3000045DD80914907882309F410CF0F900F90E5
:10C310000F900F90DF91CF911F910F91FF90EF90B1
:10C32000DF90CF90BF90AF909F9008950F93CF93E1
:10C33000DF9361E081E00E948478C0916F07D0E0D4
:10C34000C11118C080913807811104C00E94548225
:10C350008111B5C080912302882361F081E0909122
:10C360003807911180E004E024E04BEF5DE26D2F8F
:10C370000E94B14E80913B0F8770873009F058C002
:10C38000C130D9F480913807813021F40E94548261
:10C3900081119DC080912302882309F4C0C081E0EF
:10C3A00090913807913009F080E003E02EE344EFEC
:10C3B0005DE26D2F0E94B14EB2C0C230D9F48091BF
:10C3C0003807823021F40E94548281118AC0809102
:10C3D0002302882309F4A3C081E0909138079230AA
:10C3E00009F080E003E02EE34DEE5DE26D2F0E9448
:10C3F000B14E95C0C330D1F580913807833021F418
:10C400000E945482811177C080912302882309F40D
:10C4100086C081E090913807933009F080E003E016
:10C420002EE346EE5DE26D2F0E94B14E84E03EC0E9
:10C43000C130F1F480913807813021F40E94548298
:10C44000811163C080912302882309F46AC081E0CE
:10C4500090913807913009F080E000E22EE348ED3A
:10C460005DE26D2F0E94B14E82E020C084E001C0E9
:10C4700082E0C8131BC0809138078C1304C00E944F
:10C480005482811150C080912302882371F081E091
:10C49000909138079C1380E003E02EE34EEC5DE2C0
:10C4A0006D2F0E94B14E8C2F01C08C2FDF5FCF5FAC
:10C4B000D53009F045CF8F5F809337073DC00E948C
:10C4C000C97780914907882309F444CF35C089E6AC
:10C4D00096E60E94A45680914907882309F45ACF12
:10C4E0002BC08EE696E60E94A456809149078823C9
:10C4F00009F46DCF21C083E796E60E94A45680918F
:10C500004907882309F480CF17C082EE9DE20E947C
:10C51000427680914907882309F494CF0DC084E0C6
:10C52000C5CF82E0C3CF88E796E60E94A4568091EB
:10C530004907882309F4A7CFDF91CF910F91089580
:10C54000CF92DF92EF92FF92CF93C82F0E946C316F
:10C550006B017C0124EA30E74DE75FE360918607D9
:10C560007091870780918807909189070F94646C78
:10C5700087FD05C04AEF50E060E070E003C040E096
:10C5800050E0BA01C40ED51EE61EF71EC092820707
:10C59000D0928307E0928407F0928507C09324022B
:10C5A000CF91FF90EF90DF90CF9008953F924F9200
:10C5B0005F926F927F928F929F92AF92BF92CF9233
:10C5C000DF92EF92FF920F931F93CF93DF93CDB73C
:10C5D000DEB72A970FB6F894DEBF0FBECDBF9A879D
:10C5E0008987362E0E945482882329F010929F0753
:10C5F0000E94C977E8C02091950730919607409135
:10C600009707509198072D833E834F835887232B9C
:10C61000242B252B09F49EC034E0339E8001112485
:10C62000F801E659FD4F408051806280738020E020
:10C6300030E04AE754E4C301B2010F948A6B4B0126
:10C640005C0120E030E04AE754E4C301B2010F94FA
:10C650008B6B6B017C0180915F028823D1F141E0FB
:10C66000341639F13416A0F052E0351232C0809001
:10C67000570290905802A0905902B0905A02C09070
:10C680005B02D0905C02E0905D02F0905E0221C0FF
:10C690008090470290904802A0904902B0904A02D0
:10C6A000C0904B02D0904C02E0904D02F0904E02B0
:10C6B00010C080904F0290905002A0905102B09014
:10C6C0005202C0905302D0905402E0905502F09074
:10C6D00056026D817E818F8198850F94066D209121
:10C6E00086073091870740918807509189070F94FA
:10C6F000A26E9B01AC01C301B2010F948B6B065972
:10C700001D4FD8016D937D938D939C9313972D812D
:10C710003E814F81588557FF0DC0A50194010F94AC
:10C72000646C87FF12C0D8018D929D92AD92BC922D
:10C7300013970BC0A70196010F94676E18162CF47F
:10C74000F801C082D182E282F382832DF9DE81E09A
:10C7500080932302109295071092960710929707E4
:10C760001092980780912302882369F124E0329E79
:10C77000F0011124E659FD4F80819181A281B3819E
:10C7800089839A83AB83BC832DEC3CEC4CEC5DE35A
:10C79000609186077091870780918807909189073B
:10C7A0000F94676E87FD05C0CE0101960E94D8A048
:10C7B00005C060E2CE0101960E9450A1BC018985AE
:10C7C0009A850E943C4F2A960FB6F894DEBF0FBEA2
:10C7D000CDBFDF91CF911F910F91FF90EF90DF9030
:10C7E000CF90BF90AF909F908F907F906F905F9011
:10C7F0004F903F90089560E083E79EE2D7CE61E0DE
:10C800008CE69EE2D3CE62E085E69EE2CFCECF9369
:10C81000DF9300D01F92CDB7DEB70E9454828823E9
:10C8200029F010929F070E94C9775DC0609195071B
:10C8300070919607809197079091980761157105FF
:10C840008105910569F10F94066D2091860730915D
:10C85000870740918807509189070F94A26E9B012A
:10C86000AC0160917602709177028091780290918C
:10C8700079020F948B6B60937602709377028093AA
:10C8800078029093790283E05BDE81E0809323025B
:10C89000109295071092960710929707109298079A
:10C8A000809123028823F9F02091220730912307F9
:10C8B000409124075091250760917602709177028C
:10C8C00080917802909179020F948A6B69837A83C0
:10C8D0008B839C83CE0101960E94D8A0BC0184E08A
:10C8E0009EE20E943C4F0F900F900F900F90DF91AF
:10C8F000CF91089521E020939F076093860770935E
:10C900008707809388079093890740E050E0BA0139
:10C9100080912007909121070C949E7760E070E051
:10C9200080E291E4E7CF60E070E080E89FE3E2CF4F
:10C930006DEC7CEC8CEC9DE3DDCFFF920F931F93AD
:10C94000CF93DF93F82E709321076093200761E067
:10C9500081E00E948478D0916F07C0E091E081E08F
:10C96000F816A9F1F81628F082E0F81609F45DC06F
:10C970008AC0D111FBC09923D9F0809138071816CD
:10C98000BCF0409195075091960760919707709180
:10C9900098074F5F5F4F6F4F7F4F409395075093BE
:10C9A000960760939707709398078F5F8093380777
:10C9B00080912302882309F44AC100E010E021E0BD
:10C9C00041E06EE57EE28C2F0E94524E40C1D111B3
:10C9D000CDC09923D9F0809138071816BCF040914A
:10C9E00095075091960760919707709198074F5F50
:10C9F0005F4F6F4F7F4F409395075093960760931B
:10CA00009707709398078F5F809338078091230270
:10CA1000882309F41CC100E010E021E041E067E553
:10CA20007EE28C2F0E94524E12C1D1119FC09923D9
:10CA3000D9F0809138071816BCF0409195075091B5
:10CA4000960760919707709198074F5F5F4F6F4F00
:10CA50007F4F409395075093960760939707709385
:10CA600098078F5F8093380780912302882309F409
:10CA7000EEC000E010E021E041E060E57EE28C2FB6
:10CA80000E94524EE4C0409176025091770260912C
:10CA900078027091790240932207509323076093A4
:10CAA000240770932507D1112CC09923D9F08091C8
:10CAB00038071816BCF04091950750919607609181
:10CAC0009707709198074F5F5F4F6F4F7F4F40936D
:10CAD00095075093960760939707709398078F5F19
:10CAE0008093380780912302882309F4E8C000E08E
:10CAF00010E021E041E066E47EE28C2F0E94524E7D
:10CB0000DEC083E0F81232C060917C0D70917D0D23
:10CB100080917E0D90917F0D2091400D211126C0B6
:10CB20000F94D36C20913402309135026217730751
:10CB3000ECF4D130C9F480913807813021F40E949F
:10CB4000548281118EC080912302882369F081E094
:10CB500090913807913009F080E004E024E046E34A
:10CB60005EE26C2F0E94B14E82E072C0D130D9F4E7
:10CB700080913807813021F40E945482811179C05C
:10CB800080912302882309F462C081E090913807E4
:10CB9000913009F080E004E024E04CE25EE26C2F8A
:10CBA0000E94B14E54C0D230D9F4809138078230FF
:10CBB00021F40E945482811164C080912302882351
:10CBC00009F445C081E090913807923009F080E087
:10CBD00003E02EE342E25EE26C2F0E94B14E37C0CA
:10CBE000D330D1F480913807833021F40E945482ED
:10CBF000811151C080912302882349F181E09091F5
:10CC00003807933009F080E003E02EE349E15EE26B
:10CC10006C2F0E94B14E1BC0D430C9F480913807EC
:10CC2000843021F40E94548281113FC080912302FC
:10CC3000882369F081E090913807943009F080E012
:10CC400003E02EE34EE05EE26C2F0E94B14E85E0E1
:10CC5000CF5FDF5F90E0C53009F081CE809337076A
:10CC600032C00E94C97780914907882309F46BCFAD
:10CC70002AC00E94C97780914907882309F480CF90
:10CC800022C08EE894E60E94A4568091490788232A
:10CC900009F493CF18C083E994E60E94A4568091CA
:10CCA0004907882309F4A6CF0EC088E994E60E94BC
:10CCB000A45680914907882309F4B8CF04C083E0C3
:10CCC000F812C5CF21CFDF91CF911F910F91FF9027
:10CCD00008954FEF6BEF73E680E02FCE4FEF6FEFCD
:10CCE00073E681E02ACE4FEF63E074E682E025CE62
:10CCF0004FEF67E074E683E020CE0F93CF93DF938E
:10CD000061E081E00E948478D0916F07C0E0D1118A
:10CD10001AC080913807811104C00E945482811189
:10CD2000A9C080912302882309F49BC081E09091DF
:10CD30003807911180E004E024E049EC5DE26C2FBB
:10CD40000E94B14E8EC0D130D9F480913807813025
:10CD500021F40E945482811195C08091230288237E
:10CD600009F47FC081E090913807913009F080E0AC
:10CD700003E02EE34FEB5DE26C2F0E94B14E71C0D9
:10CD8000D230D9F480913807823021F40E94548245
:10CD9000811182C080912302882309F462C081E05E
:10CDA00090913807923009F080E000E22EE341EBE9
:10CDB0005DE26C2F0E94B14E54C0D330D9F4809103
:10CDC0003807833021F40E94548281116FC0809112
:10CDD0002302882309F445C081E0909138079330FD
:10CDE00009F080E000E22EE34AE05DE26C2F0E9451
:10CDF000B14E37C0D430D1F480913807843021F45B
:10CE00000E94548281115CC080912302882349F1E1
:10CE100081E090913807943009F080E000E22EE341
:10CE20004BEF5CE26C2F0E94B14E1BC0D530C9F4B1
:10CE300080913807853021F40E94548281114AC0C4
:10CE400080912302882369F081E090913807953022
:10CE500009F080E000E22EE346EE5CE26C2F0E94D7
:10CE6000B14ECF5FDF5FC53009F051CF86E08093D0
:10CE7000370739C00E94C97780914907882309F490
:10CE800050CF31C086E991E60E94A45680914907AF
:10CE9000882309F462CF27C08BEB9DE20E94427683
:10CEA00080914907882309F475CF1DC087E19DE271
:10CEB0000E94427680914907882309F488CF13C0E5
:10CEC00081EA93E00E94427680914907882309F421
:10CED0009BCF09C087EF9CE20E9442768091490770
:10CEE000882309F4ADCFDF91CF910F910895CF93AF
:10CEF000DF93EC01CB01BA010F94066D0F94D36C54
:10CF000079836883DF91CF91089567E777E688E1B9
:10CF100098E60C94DD770F931F93CF93DF9361E036
:10CF200081E00E948478C0916F07D0E081E0C11158
:10CF30002CC08823D9F0809138071816BCF0409196
:10CF400095075091960760919707709198074F5FEA
:10CF50005F4F6F4F7F4F40939507509396076093B5
:10CF60009707709398078F5F80933807809123020B
:10CF7000882309F441C000E010E020E041E06DEDBD
:10CF80007FE28D2F0E94524E37C0C130D1F4809184
:10CF90003807813021F40E945482811137C080917A
:10CFA0002302882349F181E090913807913009F0FC
:10CFB00080E000E22EE342ED5FE26D2F0E94B14E71
:10CFC0001BC0C230C9F480913807823021F40E941E
:10CFD0005482811122C080912302882369F081E06C
:10CFE00090913807923009F080E000E22EE34EEB9A
:10CFF0005FE26D2F0E94B14EDF5FCF5F80E0D530E2
:10D0000009F095CF83E0809337070DC0C093DF0C04
:10D0100080914907882319F206C0C093DF0C8091E4
:10D0200049078823C1F2DF91CF911F910F91089595
:10D030000F94066D0F94D36CCB010C94D89FEF9294
:10D04000FF920F931F93CF93DF93CDB7DEB72B974C
:10D050000FB6F894DEBF0FBECDBF7C01409127070D
:10D06000842F042E000C990B20912807223051F0B8
:10D07000233019F02CE030E30AC047FF06C028E156
:10D0800030E305C02AE230E302C021E230E39F939F
:10D090004F933F932F938E010F5F1F4F1F930F935B
:10D0A0000F94B17440913202509133024F505109A4
:10D0B00097010F900F900F900F900F900F904E15BB
:10D0C0005F050CF49A013093810D2093800D80E070
:10D0D0000E94CDCAC8010E9494792B960FB6F8948D
:10D0E000DEBF0FBECDBFDF91CF911F910F91FF909B
:10D0F000EF900895E091270787E1E802F0011124FD
:10D10000E858F24F808591859ACF5F926F927F9217
:10D110008F929F92AF92BF92CF92DF92EF92FF9247
:10D120000F931F93CF93DF93582E8093280760931C
:10D13000270761E081E00E948478D0916F07C0E00A
:10D1400081E02AE7622E28E6722ED11138C08823AA
:10D15000D9F0809138071816BCF04091950750918E
:10D16000960760919707709198074F5F5F4F6F4FD9
:10D170007F4F40939507509396076093970770935E
:10D1800098078F5F8093380780912302882309F4E2
:10D1900094C022E0521649F033E0531203C06EEE01
:10D1A0007FE205C06EED7FE202C06EEF7FE200E03D
:10D1B00010E021E041E08C2F0E94524E7EC0D13021
:10D1C000D9F480913807813021F40E945482811172
:10D1D0007DC080912302882309F46FC081E0909183
:10D1E0003807913009F080E004E024E049E650E39C
:10D1F0006C2F0E94B14E61C0D230D9F480913807B3
:10D20000823021F40E945482811168C080912302EF
:10D21000882309F452C081E090913807923009F0D8
:10D2200080E000E22EE34DE550E36C2F0E94B14E0A
:10D2300044C0D330D1F480913807833021F40E9468
:10D240005482811156C0809123028823B1F181E07C
:10D2500090913807933009F080E000E22EE341E539
:10D2600050E36C2F0E94B14E28C0D43031F580912C
:10D270003807843021F40E945482811145C0809186
:10D2800023028823D1F011E080913807843009F01F
:10D2900010E02091270737E12303F0011124E8581B
:10D2A000F24F808591850E94D89F00E09C0143E366
:10D2B00050E36C2F812F0E94E04ECF5FDF5F80E054
:10D2C000C53009F042CFC093370755C00E94C977D7
:10D2D00080914907882309F47CCF4DC080913307A2
:10D2E00090913407ACDE80914907882309F48ECFF2
:10D2F00042C08091350790913607A1DE80914907A1
:10D30000882309F4A0CF37C081E00E944982609150
:10D31000270727E16203B0011124FB01E858F24F0F
:10D32000A084B184C501BB0CAA0BBB0B5C016D01D1
:10D3300038E7A31AB108C108D1086058724F1F928C
:10D340007F926F9285E8882E87E6982E1AEAE12E62
:10D35000F12C00E010E028E730E040E050E082E40B
:10D3600090E30E9444760F900F900F9080914907B0
:10D37000882309F484CFDF91CF911F910F91FF9003
:10D38000EF90DF90CF90BF90AF909F908F907F9065
:10D390006F905F90089560E081E0B7CE8F929F928A
:10D3A000AF92BF92CF92DF92EF92FF920F931F93B3
:10D3B000CF93DF934C015B016A0160E085E00E943E
:10D3C0008478D0916F07F12C82E0E82ED1111AC039
:10D3D00080912302882321F180912602823041F03E
:10D3E000833019F463E97FE205C061E87FE202C09F
:10D3F00063EA7FE200E010E021E041E08F2D0E942F
:10D40000524E0EC0D13061F480912302882341F046
:10D4100000E010E020E041E0B4018F2D0E94524E68
:10D42000A114B10481F0D23081F4809123028823C9
:10D4300009F46EC000E010E020E041E0B5018F2D5E
:10D440000E94524E65C0C2E001C0C3E0C114D104C5
:10D4500091F0DC130FC080912302882351F000E08B
:10D4600010E020E041E0B6018F2D0E94524ECD2FFA
:10D4700001C0CD2FCF5F21E030E0A114B10411F441
:10D4800020E030E081E090E0C114D10411F480E0AC
:10D4900090E0820F931F029781F0DC130DC0809102
:10D4A0002302882349F000E010E020E041E06CEB2B
:10D4B0007FE28F2D0E94524ECF5FDC1314C080910B
:10D4C0002302882371F000E010E021E040E061EBEE
:10D4D0007FE28F2D0E94524E609126078F2D0E9471
:10D4E000F34DE0922302F394DF5F85E0F8126ECFF4
:10D4F000CF5FC0933707DF91CF911F910F91FF90BE
:10D50000EF90DF90CF90BF90AF909F908F90089555
:10D51000C3E0C114D10409F0ADCFADCF40E050E07D
:10D5200060E070E086E79FE239CF4DE65FE26DE5AF
:10D530007FE284E59FE232CF40E050E064E47FE2A6
:10D540008BE39FE22BCF40E050E06CE27FE28DE185
:10D550009FE224CF40E050E06EE07FE281E09FE276
:10D560001DCF45EF5EE264EE7EE284ED9EE216CFD3
:10D5700040E050E066EC7EE28DEB9EE20FCF40E0B3
:10D5800050E06DEA7EE280EA9EE208CF40E050E0A3
:10D5900063E97EE282E99EE201CF40E050E063E889
:10D5A0007EE28AE79EE2FACE611160932602409302
:10D5B0002607082E000C990BAA0BBB0B8C3091058B
:10D5C00098F5FC018827EA56FF4F8F4F0D94EC6FBA
:10D5D00085E99AE61FC08CE99AE61CC08FEB9AE6B3
:10D5E00019C081EB9AE616C088EB9AE613C08DEC61
:10D5F0009AE610C086EC9AE60DC08AEA9AE60AC05E
:10D6000083EA9AE607C01092DF0C8BE897E602C027
:10D610008EE89AE6009741F021E020939F0740E0D2
:10D6200050E0BA010C949E770C94C37780918A07DE
:10D63000882321F010929F070E94C9770C945A4DBD
:10D640009091090A93FB882780F993FF06C081E037
:10D6500090913908911101C080E00895F1DF88238D
:10D6600039F08091090A82FB882780F991E08927A7
:10D6700008950F93CF93DF9361E081E00E94847857
:10D68000D0916F07C0E0D1111AC080913807811185
:10D6900004C00E945482811152C0809123028823C9
:10D6A00009F444C081E090913807911180E004E0D2
:10D6B00024E044E351E36C2F0E94B14E37C0D130D7
:10D6C000D1F480913807813021F40E945482811175
:10D6D0003EC080912302882349F181E09091380770
:10D6E000913009F080E003E02EE343E251E36C2F38
:10D6F0000E94B14E1BC0D230C9F4809138078230ED
:10D7000021F40E94548281112CC08091230288232D
:10D7100069F081E090913807923009F080E003E0F1
:10D720002EE345E151E36C2F0E94B14ECF5FDF5FE6
:10D73000C53009F0A8CF83E0809337071AC00E9454
:10D74000C97780914907882309F4A7CF12C086E1E1
:10D750009BE60E94A45680914907882309F4B9CF1B
:10D7600008C083E592E70E94A45680914907882368
:10D7700061F2DF91CF910F91089540E061E080E088
:10D7800013DF8BE591E30F94175B0D94B50D66DF06
:10D79000882321F087E591E30F94175B0C949AC5D9
:10D7A0001092AF19109290028091090A80628093C2
:10D7B000090A0E94A2C56FEF89E491E30E94FC83ED
:10D7C0000C94C3770F93CF93DF9361E081E00E94C5
:10D7D0008478D0916F07C0E08C2F8D0FC9F48091B1
:10D7E0003807811104C00E945482811133C0809196
:10D7F0002302882341F181E090913807911180E064
:10D8000004E024E044E451E36C2F0E94B14E1BC0BD
:10D810008130C9F480913807813021F40E9454820C
:10D8200081111FC080912302882369F081E09091CB
:10D830003807913009F080E000E22EE349E351E33C
:10D840006C2F0E94B14ECF5FC53031F682E08093DD
:10D8500037070CC00E94C97780914907882339F2A5
:10D8600005C09EDF809149078823E1F2DF91CF91C7
:10D870000F910895EF92FF920F931F93CF93DF9331
:10D8800061E081E00E948478C0916F0710E0C111CF
:10D8900018C080913807811104C00E945482811100
:10D8A00083C180912302882361F081E09091380741
:10D8B000911180E004E024E049E051E3612F0E94EF
:10D8C000B14E0E948777D82F9091090A93FBEE24DE
:10D8D000E0F893FF03C0B4DEF82E01C0F12CDD2385
:10D8E00009F458C0C130D9F480913807813021F44F
:10D8F0000E945482811160C180912302882309F41F
:10D900006CC181E090913807913009F080E000E22D
:10D910002EE34DEF50E3612F0E94B14E5EC1C23045
:10D92000D9F480913807823021F40E945482811109
:10D930004AC180912302882309F44FC181E090916C
:10D940003807923009F080E003E02EE342EF50E325
:10D95000612F0E94B14E41C1C33009F047C0809190
:10D960003807833021F40E945482811138C180919C
:10D970002302882309F431C181E090913807933064
:10D9800009F080E003E02EE34DEE50E3612F0E94AA
:10D99000B14E23C18091A219823029F05FDE81113E
:10D9A00002C0D1E004C0C13009F423C1D2E0CD13DC
:10D9B0001BC0809138078C1304C00E9454828111CF
:10D9C0003AC180912302882371F081E09091380759
:10D9D0009C1380E003E02EE347ED50E3612F0E94AB
:10D9E000B14EDC2F01C0DC2FDF5F01C0D4E0CD13CE
:10D9F0001BC0809138078C1304C00E94548281118F
:10DA000024C180912302882371F081E0909138072E
:10DA10009C1380E003E02EE34BEC50E3612F0E9467
:10DA2000B14EDC2F01C0DC2F81E08D0FC81318C070
:10DA3000809138078C1304C00E94548281110FC159
:10DA400080912302882361F081E0909138079C1334
:10DA500080E003E02EE34DEB50E3612F0E94B14ED6
:10DA600082E08D0F4091800D5091810D9091400D7D
:10DA7000911107C0209134023091350242175307AB
:10DA8000DCF0C81333C0809138078C1304C00E94A7
:10DA900054828111EEC080912302882339F181E004
:10DAA000909138079C1380E000E22EE345EA50E3B2
:10DAB000612F0E94B14E1AC0C81318C08091380758
:10DAC0008C1304C00E9454828111DDC08091230216
:10DAD000882361F081E0909138079C1380E003E097
:10DAE0002EE345E950E3612F0E94B14EDD5FCD1377
:10DAF00018C0809138078C1304C00E945482811191
:10DB0000CCC080912302882361F081E09091380796
:10DB10009C1380E003E02EE347E850E3612F0E946E
:10DB2000B14E91E09D0FEE20E9F0F11035C0C91320
:10DB300031C0809138078C1304C00E945482811137
:10DB4000B6C080912302882329F181E090913807A3
:10DB50009C1380E003E02EE349E750E3612F0E942D
:10DB6000B14E18C0C91316C0809138078C1302C07B
:10DB70000E94548280912302882361F081E0909179
:10DB800038079C1380E000E22EE34EE650E3612F5D
:10DB90000E94B14E92E09D0F1F5FCF5F153009F0DC
:10DBA00076CE909337078CC00E94C9778091490741
:10DBB000882309F476CE84C0E0DD8091490788236C
:10DBC00009F49ACE7DC082EE9BE60E94A456809115
:10DBD0004907882309F4ADCE73C0D4E025CF81EA8C
:10DBE0009FE60E94A45680914907882309F4BFCE7E
:10DBF00067C080913807813021F40E9454828111DE
:10DC000012C0809123028823A1F081E0909138070F
:10DC1000913009F080E000E22EE340EE50E3612F06
:10DC20000E94B14E06C0B3DD80914907882349F3B5
:10DC300047C0D2E0D9CE8DE796E60E94A4568091E7
:10DC40004907882309F4BDCE3BC084E893E70E94CE
:10DC5000A45680914907882309F4D3CE31C084EFBC
:10DC600094E70E94A45680914907882309F4E8CEDE
:10DC700027C085EB90E30E94427680914907882374
:10DC800009F409CF1DC08BEC99E60E94A45680913F
:10DC90004907882309F41ACF13C089E39BE60E9441
:10DCA000A45680914907882309F42BCF09C085E445
:10DCB00092E50E94A45680914907882309F441CF38
:10DCC000DF91CF911F910F91FF90EF900895609198
:10DCD000760D70E080E00C941DC660917E0270911C
:10DCE0007F02072E000C880B990B0F94066D2AE01B
:10DCF00037ED43E25CE30F94A26E60937A02709377
:10DD00007B0280937C0290937D020895CF93DF93F2
:10DD1000EC01CB01BA010F94066D0F94D86C6883A7
:10DD2000DF91CF91089540E050E0BA018FE49FE683
:10DD30000E949E771092290710922A0710922B07B3
:10DD400010922C0781E080939F07089540E050E0F7
:10DD5000BA0183E59FE60E949E77109229071092F0
:10DD60002A0710922B0710922C0781E080939F07BF
:10DD7000089580E00C94CDCA66E87EE682EC9EE6CB
:10DD80000C94DD770F94066D0F94D86C862F0C944D
:10DD9000409FBF92CF92DF92EF92FF920F931F931B
:10DDA000CF93DF9300D01F92CDB7DEB7B82E8B0193
:10DDB0000E945482882329F010929F070E94C977FD
:10DDC00060C0C0909507D0909607E0909707F090BC
:10DDD0009807C114D104E104F10439F110929507B8
:10DDE00010929607109297071092980781E08093FF
:10DDF0002302B6018B2D0E9486D00D2C000CEE085C
:10DE0000FF088091290790912A07A0912B07B091D4
:10DE10002C07C80ED91EEA1EFB1EC0922907D092FD
:10DE20002A07E0922B07F0922C0780912302882387
:10DE300041F124E0B29EC0011124FC01ED52F04FEB
:10DE40007F016091290770912A0780912B0790919B
:10DE50002C070F94066D9B01AC01F7016081718165
:10DE6000828193810F94A26E69837A838B839C83D2
:10DE700060E2CE0101960E9450A1BC01C8010E943F
:10DE80003C4F0F900F900F900F90DF91CF911F910B
:10DE90000F91FF90EF90DF90CF90BF9008956AEDC3
:10DEA00071E380E076CF6FEC71E381E072CF4F9247
:10DEB0005F926F927F928F929F92AF92BF92CF921A
:10DEC000DF92EF92FF920F931F93CF93DF93F901AD
:10DED000D8019E2C9A01550F440B550BEB01A880DD
:10DEE000B9806501BB0CEE08FF0856016701A21A54
:10DEF000B30AC40AD50A2F01FF0F66087708830109
:10DF00007201E21AF30A040B150B9F92BF93AF93B1
:10DF1000E5E88E2EE7E69E2EB7D60F900F900F9075
:10DF2000DF91CF911F910F91FF90EF90DF90CF90F5
:10DF3000BF90AF909F908F907F906F905F904F9029
:10DF400008956F927F928F929F92AF92BF92CF92DD
:10DF5000DF92EF92FF920F931F93CF93DF9361E0D5
:10DF600081E00E948478D0916F07C0E027E6622E9E
:10DF70002EE6722ED1111AC080913807811104C08B
:10DF80000E945482811121C180912302882309F4C7
:10DF900013C181E090913807911180E004E024E002
:10DFA0004AEC51E36C2F0E94B14E06C1D13011F5FD
:10DFB00080913807813021F40E94548281110CC174
:10DFC00080912302882309F4F7C011E0809138077B
:10DFD000813009F010E080916402909165020E9406
:10DFE000D89F00E09C014EEB51E36C2F812F0E94E3
:10DFF000E04EE2C0D23011F580913807823021F432
:10E000000E9454828111FAC080912302882309F46E
:10E01000D3C011E080913807823009F010E0809180
:10E02000800D9091810D0E94D89F00E09C0140EBF3
:10E0300051E36C2F812F0E94E04EBEC0D33011F50A
:10E0400080913807833021F40E9454828111EBC003
:10E0500080912302882309F4AFC011E08091380732
:10E06000833009F010E080915C0D90915D0D0E946D
:10E07000D89F00E09C0148EA51E36C2F812F0E9459
:10E08000E04E9AC0D43001F580913807843021F4F5
:10E090000E9454828111DCC080912302882309F4FC
:10E0A0008BC011E080913807843009F010E0809136
:10E0B000760D0E94409F00E09C0144E951E36C2FE3
:10E0C000812F0E94E04E78C0D53011F5809138073D
:10E0D000853021F40E9454828111DEC08091230298
:10E0E000882309F469C011E080913807853009F070
:10E0F00010E080917E0290917F020E94D89F00E004
:10E100009C014AE851E36C2F812F0E94E04E54C0DD
:10E11000D630D9F480913807863021F40E94548299
:10E120008111CCC080912302882309F445C081E08D
:10E1300090913807963009F080E003E02EE34FE736
:10E1400051E36C2F0E94B14E37C0D730D1F480918B
:10E150003807873021F40E9454828111BCC080911D
:10E160002302882349F181E090913807973009F024
:10E1700080E003E02EE344E751E36C2F0E94B14EB0
:10E180001BC0D830C9F480913807883021F40E9430
:10E1900054828111ADC080912302882369F081E00F
:10E1A00090913807983009F080E003E02EE345E6CF
:10E1B00051E36C2F0E94B14ECF5FDF5FC53009F095
:10E1C000D9CE89E0809337079FC0E3D68091490775
:10E1D000882309F4D9CE98C0E12C00E010E027EEA6
:10E1E00033E04AE050E064E672E084EC91E35FDE05
:10E1F00080914907882309F4E3CE86C081E00E941C
:10E200004982E12C09EB1EE622E231E040E050E0D9
:10E2100060E87DE087EB91E34ADE8091490788233F
:10E2200009F4F2CE71C081E00E944982E12C0AE13A
:10E230001BEC2CE830E040E050E06CE57DE08CEA3F
:10E2400091E335DE80914907882309F401CF5CC052
:10E2500081E00E944982A090760DB12CC12CD12C76
:10E260001F927F926F928CEB882E8EE6982EE12C77
:10E27000F12C8701EA9420E030E0A90166E77DE017
:10E280008EE991E301D50F900F900F90809149078F
:10E29000882309F401CF38C0E12C0DE61EE627EEF5
:10E2A00033E04AE050E06EE772E08FE891E3FFDD93
:10E2B00080914907882309F411CF26C0C3D440E0D8
:10E2C00050E0BA0183E99EE639D680914907882358
:10E2D00009F428CF19C0B6D440E050E0BA0186EA6C
:10E2E0009EE62CD680914907882309F438CF0CC0CC
:10E2F000A9D440E050E0BA018CEF98E71FD6809196
:10E300004907882309F447CFDF91CF911F910F91DF
:10E31000FF90EF90DF90CF90BF90AF909F908F9045
:10E320007F906F9008954F925F926F927F92AF921D
:10E33000BF92CF92DF92EF92FF92CF93DF93EB01E8
:10E34000FC0160817181828193812CE3C22ED12CEA
:10E35000E12CF12CA70196010F94AE6FB62EA72EDB
:10E36000CA01B901A70196010F94AE6F6B017C0140
:10E37000CA01B90128E130E040E050E00F94AE6FEF
:10E380002B013C01C9016DE671E00F94876F6115A7
:10E390007105D9F0AF92BF92DF92CF925F924F9208
:10E3A0009F938F937F936F938DE092E39F938F93CF
:10E3B000DF93CF930F94B1748DB79EB70E960FB6BF
:10E3C000F8949EBF0FBE8DBF61C00097C9F0AF9299
:10E3D000BF92DF92CF925F924F929F938F938DEF78
:10E3E00091E39F938F93DF93CF930F94B174EDB725
:10E3F000FEB73C960FB6F894FEBF0FBEEDBF46C009
:10E400004114510461047104B9F0AF92BF92DF92DC
:10E41000CF925F924F9281EF91E39F938F93DF931F
:10E42000CF930F94B1748DB79EB70A960FB6F89438
:10E430009EBF0FBE8DBF2AC0C114D104E104F104F8
:10E44000A9F0AF92BF92DF92CF9289EE91E39F93B2
:10E450008F93DF93CF930F94B174EDB7FEB73896D7
:10E460000FB6F894FEBF0FBEEDBF10C0AF92BF92C3
:10E4700085EE91E39F938F93DF93CF930F94B174C5
:10E480000F900F900F900F900F900F90DF91CF9102
:10E49000FF90EF90DF90CF90BF90AF907F906F9004
:10E4A0005F904F9008952F923F924F925F926F929C
:10E4B0007F928F929F92AF92BF92CF92DF92EF9214
:10E4C000FF920F931F93CF93DF93CDB7DEB76F9774
:10E4D0000FB6F894DEBF0FBECDBF0E9454828823D2
:10E4E00011F057D5F0C02090A30D3090A40D80916D
:10E4F000A50D9091A60D9F8F8E8F8091A70D909165
:10E50000A80DA091A90DB091AA0D8A8F9B8FAC8FF9
:10E51000BD8F4090AB0D5090AC0D6090AD0D7090E4
:10E52000AE0D8090AF0D9090B00DA090B10DB09059
:10E53000B20D60E085E0E8D5E0906F07F12CDE01D8
:10E5400011966D01E1100DC0809123028823E1F046
:10E55000C1010E940EA08C0120E040E062E772E35E
:10E5600010C0B1E0EB1210C080912302882361F04B
:10E570008E8D9F8D0E940EA08C0120E040E066E60B
:10E5800072E38F2D0E94524E8A8D9B8DAC8DBD8D76
:10E590008E8B9F8BA88FB98FB601CE014696C3DEB6
:10E5A00092E0E9120BC0809123028823B1F000E0D1
:10E5B00010E020E040E064E572E30CC0A3E0EA1262
:10E5C0000CC080912302882341F0860120E040E0C6
:10E5D00061E572E38F2D0E94524E4E8A5F8A688EEB
:10E5E000798EB601CE0146969EDEB4E0EB120BC0EA
:10E5F000809123028823B1F000E010E020E040E0A9
:10E600006FE372E30CC085E0E8120CC08091230236
:10E61000882341F0860120E040E06CE372E38F2D17
:10E620000E94524E20E030E048EC52E4C501B401B3
:10E630000F946B6C0F94D36CCB016AE070E00F9475
:10E640009B6F9F938F9320E030E04AE754E4C5012D
:10E65000B4010F946B6C0F94D36C9F938F937F9343
:10E660006F93A4E3B2E3BF93AF93DF92CF920F9483
:10E67000B1740FB6F894DEBF0FBECDBFB6E0EB129B
:10E680000BC0809123028823B1F000E010E020E06D
:10E6900040E064E272E30CC087E0E8120CC08091B5
:10E6A0002302882341F0860120E040E061E272E32A
:10E6B0008F2D0E94524EF394E39495E0F91242CFCD
:10E6C00088E0809337076F960FB6F894DEBF0FBED1
:10E6D000CDBFDF91CF911F910F91FF90EF90DF9011
:10E6E000CF90BF90AF909F908F907F906F905F90F2
:10E6F0004F903F902F90089560E070E080E00E947E
:10E700001DC60E9467CB3FC42F923F924F925F92EB
:10E710006F927F928F929F92AF92BF92CF92DF9231
:10E72000EF92FF920F931F93CF93DF9361E081E00D
:10E73000EBD420906F07312C67E6462E6EE6562EFE
:10E74000CAE1DBEC79EB672E7EE6772E21101AC04A
:10E7500080913807811104C00E9454828111AFC09A
:10E7600080912302882309F477C081E090913807D3
:10E77000911180E004E024E043EB52E3632D0E941A
:10E78000B14E6AC081E0281222C0809138078130E2
:10E7900021F40E945482811199C080912302882320
:10E7A00009F45AC011E080913807813009F010E077
:10E7B0008091800D9091810D0E94D89F00E09C0176
:10E7C00045EA52E3632D812F0E94E04E45C092E05E
:10E7D000291221C080913807823021F40E9454828E
:10E7E00081119DC0809123028823B1F111E08091B5
:10E7F0003807823009F010E080915C0D90915D0D3A
:10E800000E94D89F00E09C014DE952E3632D812FC7
:10E810000E94E04E21C083E028121EC0809138077C
:10E82000833021F40E9454828111A1C0809123027F
:10E83000882391F011E080913807833009F010E0CF
:10E840008091760D0E94119F00E09C0149E852E3FF
:10E85000632D812F0E94E04E8091800D9091810D5B
:10E8600020915C0D30915D0D232B11F4892BF1F07B
:10E8700094E0291219C080913807843021F40E9455
:10E880005482811198C080912302882369F081E02D
:10E8900090913807943009F080E000E22EE340E8E0
:10E8A00052E3632D0E94B14E85E001C084E03394B1
:10E8B000239495E039124ACF8093370782C069D3F9
:10E8C00080914907882309F44BCF7BC081E00E94E7
:10E8D0004982A090800DB090810D0B2C000CCC08CB
:10E8E000DD081F927F926F9245E8842E47E6942EB2
:10E8F00012E2E12EFF24F39400E010E020E030E08B
:10E90000A90160E87DE08CEA92E3BED10F900F9000
:10E910000F9080914907882309F43FCF52C081E0CE
:10E920000E944982A0905C0DB0905D0D0B2C000CF4
:10E93000CC08DD081F92DF93CF9325E8822E27E6CF
:10E94000922E1CE8E12EF12C00E010E020E030E0F7
:10E95000A9016CE57DE081EA92E396D10F900F90DA
:10E960000F9080914907882309F43CCF2AC081E0A9
:10E970000E944982A090760DB12CC12CD12C1F92FF
:10E980005F924F9284E5882E83E5982EE12CF12C3E
:10E990008701EA9420E030E0A90166E77DE083E9A1
:10E9A00092E372D10F900F900F90809149078823C6
:10E9B00009F43CCF06C0A0DE80914907882309F402
:10E9C00062CFDF91CF911F910F91FF90EF90DF9079
:10E9D000CF90BF90AF909F908F907F906F905F90FF
:10E9E0004F903F902F9008950F931F93CF93DF93F5
:10E9F00061E081E089D3D0916F07C0E0D11117C0E9
:10EA000080913807811104C00E94548281119EC0F8
:10EA100080912302882309F43EC081E09091380759
:10EA2000911180E004E024E047E053E331C0D130AD
:10EA3000B9F480913807813021F40E945482811109
:10EA40008CC080912302882331F181E090913807B6
:10EA5000913009F080E003E02EE345EF52E318C067
:10EA6000D230C9F480913807823021F40E94548258
:10EA7000811180C080912302882369F081E0909108
:10EA80003807923009F080E003E02EE346EE52E3CF
:10EA90006C2F0E94B14E3BD2182FD330D9F4809105
:10EAA0003807833021F40E945482811170C0809114
:10EAB0002302882309F47EC081E0909138079330C7
:10EAC00009F080E000E22EE347ED52E36C2F0E9454
:10EAD000B14E70C0811171C0D430B9F48091380743
:10EAE000843021F40E945482811158C08091230205
:10EAF000882319F181E090913807943009F080E083
:10EB000000E22EE349EC52E315C0D530B1F4809118
:10EB10003807853009F449C080912302882369F0C1
:10EB200081E090913807953009F080E000E22EE313
:10EB300048EB52E36C2F0E94B14E86E0CF5FDF5F5F
:10EB4000C53009F05BCF8093370742C022D2809155
:10EB50004907882309F45CCF3BC074D040E050E003
:10EB6000BA0189EB96E5EAD180914907882309F437
:10EB700068CF2EC067D040E050E0BA018CEF98E734
:10EB8000DDD180914907882309F474CF21C0D4D303
:10EB900080914907882309F48ACF1AC0D0D3809185
:10EBA0004907882309F4A2CF13C00E94548281111F
:10EBB00006C0B2CF112309F4C0CF84E0BFCF0E94BA
:10EBC0007CF081E005D380914907882309F4A4CF24
:10EBD000DF91CF911F910F910895CF93DF93EC01B7
:10EBE000CB01BA010F94066D0F94D36C6883DF914B
:10EBF000CF910895CF93DF93EC01CB01BA010F942D
:10EC0000066D20E030E040E251E40F94A26E0F94D4
:10EC1000D86C79836883DF91CF9108950F94066D46
:10EC20000F94D36C862F0C94669F0F94066D20E092
:10EC300030E040E251E40F94A26E0F94D86CCB0107
:10EC40000C94959F80914A078630D8F496E0899F6E
:10EC5000F0011124E55BF84F209190073091910766
:10EC600031832083409195075091960760919707D3
:10EC70007091980742835383648375838F5F809379
:10EC80004A0708950D94175B2F923F924F925F921F
:10EC90006F927F928F929F92AF92BF92CF92DF92AC
:10ECA000EF92FF920F931F93CF93DF9300D000D08A
:10ECB000CDB7DEB71C012B833C834D835E83698314
:10ECC0007A83C0DF83E0809323023092480720924A
:10ECD000470769817A8170934607609345072B81C6
:10ECE0003C814D815E8120934107309342074093E0
:10ECF000430750934407E0923D07F0923E0700938C
:10ED00003F0710934007A0929507B0929607C092D4
:10ED10009707D092980790929107809290078C8DD8
:10ED20009D8D90933C0780933B078E8D80933A078F
:10ED300026960FB6F894DEBF0FBECDBFDF91CF9100
:10ED40001F910F91FF90EF90DF90CF90BF90AF9009
:10ED50009F908F907F906F905F904F903F902F90FB
:10ED600008954F925F926F927F928F929F92AF928F
:10ED7000BF92CF92DF92EF92FF920F931F93FB010E
:10ED8000722F602FA12FBE2D242F30E040E050E0E5
:10ED9000A080CA2CD12CE12CF12C56016701A21ABB
:10EDA000B30AC40AD50A472E512C612C712C830159
:10EDB0007201E21AF30A040B150BBF93AF936F9322
:10EDC0006CEB862E6EE6962EBF015EDF0F900F90E5
:10EDD0000F901F910F91FF90EF90DF90CF90BF9019
:10EDE000AF909F908F907F906F905F904F9008951D
:10EDF0002F923F924F925F926F927F928F929F924B
:10EE0000AF92BF92CF92DF92EF92FF920F931F9338
:10EE1000CF93DF9300D01F921F92CDB7DEB71C01B6
:10EE20007D836C8349010A831B83E982BA0180E0F8
:10EE300090E00F94046D2DEC3CEC4CEC5DE30F94F2
:10EE4000A26E0F94D36C2B013C01EC81FD8160819B
:10EE5000718180E090E00F94046D2DEC3CEC4CEC63
:10EE60005DE30F94A26E0F94D36C5B016C01A41848
:10EE7000B508C608D708B40180E090E00F94046D8F
:10EE80002DEC3CEC4CEC5DE30F94A26E0F94D36C34
:10EE90007B018C01E418F50806091709F981FF9335
:10EEA0008B818F93EA81EF938FE7882E88E7982EE6
:10EEB000A30192016C817D81C101E6DE0F900F906C
:10EEC0000F900F900F900F900F900F90DF91CF91B8
:10EED0001F910F91FF90EF90DF90CF90BF90AF9078
:10EEE0009F908F907F906F905F904F903F902F906A
:10EEF0000895FB01908181E08927808383E08093DE
:10EF000023024115510511F0FA01199408958091D9
:10EF1000411090913E10891B8F7071F49091090AF5
:10EF200092FB882780F992FD08C081E09091A21998
:10EF3000913019F080E0089581E0089520919007C4
:10EF40003091910728173907E9F090939107809342
:10EF50009007409395075093960760939707709397
:10EF60009807885A914821F410929F0710924A07F7
:10EF70000E94F24D82E08093230281E08093490752
:10EF800010929A07089540E050E0BA0188EA91E8AB
:10EF9000D5CFE0914A07EE2379F0E150E0934A079C
:10EFA00086E0E89FF0011124E55BF84F40E050E077
:10EFB000BA0180819181C2CFE6CF0F931F93CF9387
:10EFC000DF93FC01EB018091950790919607A0914A
:10EFD0009707B0919807B7FF08C010929507109255
:10EFE0009607109297071092980780913D0790918D
:10EFF0003E07A0913F07B09140074091950750917F
:10F000009607609197077091980784179507A60750
:10F01000B70744F48093950790939607A0939707BA
:10F02000B093980780912302882301F180914107D2
:10F0300090914207A0914307B091440740919507F2
:10F040005091960760919707709198078C019D01E8
:10F05000040F151F261F371FC901B8011995BC01E0
:10F0600080914707909148070E943C4F80918A0702
:10F07000811108C080913A078823B9F18091230259
:10F08000882399F180914507909146070097B1F048
:10F0900000914107109142072091430730914407A6
:10F0A0004091950750919607609197077091980746
:10F0B000400F511F621F731FFE011995E0913B071E
:10F0C000F0913C07309741F080913A07811103C0DD
:10F0D00080918A07811119950E945482882329F012
:10F0E000DF91CF911F910F9154CFDF91CF911F915D
:10F0F0000F9108956DEE75E78EE096E75ECF6AEFAB
:10F1000075E785E196E759CF282F10928F078091F8
:10F11000950790919607A0919707B0919807813035
:10F120009048A105B10540F01092950710929607FE
:10F13000109297071092980780919907882331F0D1
:10F14000809195078093380710924907809137077F
:10F150001816FCF4082E000C990B821B91092091C3
:10F160003807022E000C330B2817390794F097FF4D
:10F1700002C080E090E080933807092E000CAA0BB3
:10F18000BB0B8093950790939607A0939707B09336
:10F190009807809138076623C1F090916F0789170F
:10F1A00014F480936F0720916F07022E000C330B2D
:10F1B0002C5F3F4F482F082E000C550B24173507A6
:10F1C00034F4845080936F07089580936F070895F7
:10F1D000882361F063E972E084E690E00F9464664E
:10F1E0006AEB72E084E690E00D94646668EB71E08F
:10F1F00084E190E00D9464668F929F92AF92BF92EB
:10F20000CF92DF92EF92FF920E945482882369F09E
:10F210000E94B2EB10929F07FF90EF90DF90CF908B
:10F22000BF90AF909F908F90B4CE81E080939F0766
:10F230008090950790909607A0909707B0909807B8
:10F2400081149104A104B10409F446C010929507F9
:10F25000109296071092970710929807B401092C04
:10F26000000C880B990B0F94066D2091DB0F3091E9
:10F27000DC0F4091DD0F5091DE0F0F94A26E2091B4
:10F28000130F3091140F4091150F5091160F0F94DA
:10F290008B6B6B017C0120E030E040E050EC0F9480
:10F2A000676E87FD19C020E030E040EA50E4C701F6
:10F2B000B6010F94646C18167CF0B40182E00E94D1
:10F2C00086D0C092130FD092140FE092150FF092D7
:10F2D000160F82E080932302809123028823D9F0C5
:10F2E00083E19FE00E943AA0BC018CE093E30E947E
:10F2F0003C4F6091130F7091140F8091150F9091F6
:10F30000160FFF90EF90DF90CF90BF90AF909F903F
:10F310008F900C94E14FFF90EF90DF90CF90BF90D3
:10F32000AF909F908F90089521E0209339070F941C
:10F330001C5B1092390708950E94EDEB49CF0E94A3
:10F340002EFD46CF6091970E7091980E84E69EE058
:10F350000C94D63B60915C0E70915D0E89E29EE04C
:10F360000C94D63B6091210E7091220E8EEE9DE0A2
:10F370000C94D63B6091E60D7091E70D83EB9DE018
:10F380000C94D63B8F929F92AF92BF92CF92DF9216
:10F39000EF92FF92CF9360910710709108108091C7
:10F3A000091090910A100F94D86C4B015C01C09128
:10F3B0009D0E84E69EE00E944B3DDC0120E136E09C
:10F3C00041EC50E00F9403706B017C01AC2FB0E076
:10F3D000A50194010F9403702227362F472F582F31
:10F3E000C701B6010F94AE6FBA01A901662777274E
:10F3F00084E69EE0CF91FF90EF90DF90CF90BF909A
:10F40000AF909F908F900C949F3D8F929F92AF9260
:10F41000BF92CF92DF92EF92FF92CF9360910B1049
:10F4200070910C1080910D1090910E100F94D86C6B
:10F430004B015C01C091620E89E29EE00E944B3D4F
:10F44000DC0120E136E041EC50E00F9403706B01E9
:10F450007C01AC2FB0E0A50194010F94037022272A
:10F46000362F472F582FC701B6010F94AE6FBA0140
:10F47000A9016627772789E29EE0CF91FF90EF9060
:10F48000DF90CF90BF90AF909F908F900C949F3D56
:10F490008F929F92AF92BF92CF92DF92EF92FF92A4
:10F4A000CF9360910F107091101080911110909176
:10F4B00012100F94D86C4B015C01C091270E8EEE98
:10F4C0009DE00E944B3DDC0120E136E041EC50E044
:10F4D0000F9403706B017C01AC2FB0E0A501940187
:10F4E0000F9403702227362F472F582FC701B601DC
:10F4F0000F94AE6FBA01A901662777278EEE9DE0C3
:10F50000CF91FF90EF90DF90CF90BF90AF909F9002
:10F510008F900C949F3D8F929F92AF92BF92CF920B
:10F52000DF92EF92FF92CF936091131070911410BD
:10F5300080911510909116100F94D86C4B015C01BE
:10F54000C091EC0D83EB9DE00E944B3DDC0120E17E
:10F5500036E041EC50E00F9403706B017C01AC2F5E
:10F56000B0E0A50194010F9403702227362F472F96
:10F57000582FC701B6010F94AE6FBA01A9016627D3
:10F58000772783EB9DE0CF91FF90EF90DF90CF90B6
:10F59000BF90AF909F908F900C949F3D60919E0E76
:10F5A00084E69EE00C94183E6091630E89E29EE032
:10F5B0000C94183E60919C0E84E69EE00C9493405F
:10F5C0006091610E89E29EE00C9493406091260E5A
:10F5D0008EEE9DE00C9493406091EB0D83EB9DE0EB
:10F5E0000C9493400F931F93CF93DF9361E081E0DE
:10F5F0008BDDD0916F07C0E081E0D1112CC0882352
:10F60000D9F0809138071816BCF0409195075091B9
:10F61000960760919707709198074F5F5F4F6F4F04
:10F620007F4F409395075093960760939707709389
:10F6300098078F5F8093380780912302882309F40D
:10F64000AAC000E010E020E041E06DE973E38C2FF8
:10F650000E94524EA0C0D130D1F480913807813041
:10F6600019F422D78111A1C080912302882309F4C3
:10F6700092C081E090913807913009F080E004E079
:10F6800024E041E953E36C2F0E94B14E84C0D23094
:10F69000F9F480913807823019F406D781118CC0B3
:10F6A00080912302882309F476C080919C0E8111F9
:10F6B00003C028E833E302C02CE833E381E09091F3
:10F6C0003807923009F080E001E046E853E360C07B
:10F6D000D330F9F480913807833019F4E5D68111DD
:10F6E00078C080912302882309F455C08091610E6F
:10F6F000811103C02DE733E302C021E833E381E049
:10F7000090913807933009F080E001E04BE753E334
:10F710003FC0D430F1F480913807843019F4C4D656
:10F72000811164C0809123028823A9F18091260E63
:10F73000811103C022E733E302C026E733E381E00F
:10F7400090913807943009F080E001E040E753E3FE
:10F750001FC0D53001F580913807853019F4A4D643
:10F76000811151C0809123028823A9F08091EB0D73
:10F77000811103C026E633E302C02AE633E381E0C9
:10F7800090913807953009F080E001E043E653E3BB
:10F790006C2F0E94E04ECF5FDF5F80E0C53009F044
:10F7A0002CCF86E0809337073AC0F3DB809149077E
:10F7B000882309F459CF33C04AED5AE76CE97EE05B
:10F7C0008FE893E396DB80914907882309F468CF9B
:10F7D00026C040EE5AE761E67EE084E893E389DBE9
:10F7E00080914907882309F47CCF19C046EE5AE777
:10F7F00066E27EE089E793E37CDB8091490788231A
:10F8000009F490CF0CC04CEE5AE76BEE7DE08DE62C
:10F8100093E36FDB80914907882309F4A3CFDF913D
:10F82000CF911F910F9108954F925F926F927F92A7
:10F830008F929F92AF92BF92CF92DF92EF92FF9200
:10F840000F931F93CF93DF9361E081E05DDCD09154
:10F850006F07C0E044ED642E4AE7742E5EEC452E3F
:10F860005AE7552ED11119C080913807811103C074
:10F870001BD6811156C080912302882309F448C009
:10F8800081E090913807911180E004E024E049EB99
:10F8900053E36C2F0E94B14E3BC0D130D1F4809124
:10F8A0003807813019F400D6811142C080912302BB
:10F8B000882371F111E080913807813009F010E060
:10F8C00080919E0E0E94669F00E09C0145EB53E3F1
:10F8D0001BC0D230E9F480913807823019F4E4D5A6
:10F8E000811152C080912302882391F011E0809110
:10F8F0003807823009F010E08091630E0E94669F05
:10F9000000E09C0141EB53E36C2F812F0E94E04EFD
:10F91000CF5FDF5FC53009F0A5CF83E08093370765
:10F920005EC037DB80914907882309F4A4CF57C014
:10F93000A0909E0E8A2DAA0C990BAA0BBB0B5C0102
:10F940006D0120E4A20EB11CC11CD11C1F925F925C
:10F950004F922AE7822E28E7922E1FE7E12EF12C04
:10F9600000E010E020EC3FEF4FEF5FEF6EE97EE04C
:10F9700087EB93E389D90F900F900F9080914907FF
:10F98000882309F493CF2BC0A090630E8A2DAA0C74
:10F99000990BAA0BBB0B5C016D0120E4A20EB11CFC
:10F9A000C11CD11C1F927F926F928AE7882E88E734
:10F9B000982E1FE7E12EF12C00E010E020EC3FEF45
:10F9C0004FEF5FEF63E67EE083EB93E35DD90F904B
:10F9D0000F900F9080914907882309F483CFDF911E
:10F9E000CF911F910F91FF90EF90DF90CF90BF903C
:10F9F000AF909F908F907F906F905F904F90089501
:10FA00000F93CF93DF9361E081E07EDBD0916F07AE
:10FA1000C0E0D11116C080913807811103C044D5D0
:10FA200081117BC080912302882309F46EC081E09C
:10FA300090913807911180E004E024E04BE553E316
:10FA400061C0D130B9F480913807813019F42CD5D8
:10FA500081116AC080912302882309F456C081E095
:10FA600090913807913009F080E003E02EE34CE4F8
:10FA700053E348C0D230B9F480913807823019F48A
:10FA800013D581115BC080912302882309F43DC006
:10FA900081E090913807923009F080E003E02EE396
:10FAA0004BE353E32FC0D330B1F480913807833058
:10FAB00019F4FAD481114CC080912302882329F1D2
:10FAC00081E090913807933009F080E003E02EE365
:10FAD00049E253E317C0D430C1F480913807843031
:10FAE00019F4E2D481113EC080912302882369F089
:10FAF00081E090913807943009F080E003E02EE334
:10FB00004BE153E36C2F0E94B14ECF5FDF5FC530F6
:10FB100009F07FCFC09337072EC03BDA80914907A9
:10FB2000882309F47FCF27C08FEB9DE70E94A4565E
:10FB300080914907882309F48DCF1DC08EEB9EE785
:10FB40000E94A45680914907882309F49CCF13C0D2
:10FB500084E19CE70E94A45680914907882309F418
:10FB6000ABCF09C082EF9AE70E94A4568091490763
:10FB7000882309F4B9CFDF91CF910F910895EF92C7
:10FB80000F931F93CF93DF9361E081E0BDDAD091B3
:10FB90006F07C0E0D11119C080913807811103C0EF
:10FBA00083D4811197C080912302882309F48AC0ED
:10FBB00081E090913807911180E004E024E045EF66
:10FBC00053E36C2F0E94B14E7DC0D130E9F4809197
:10FBD0003807813019F468D4811183C080912302E1
:10FBE000882309F46FC011E080913807813009F053
:10FBF00010E08091970E9091980E0E94959F00E0E2
:10FC00009C0141EF53E35AC0D230E9F480913807A8
:10FC1000823019F449D4811176C08091230288235F
:10FC200009F450C011E080913807823009F010E0EB
:10FC300080915C0E90915D0E0E94959F00E09C016A
:10FC40004DEE53E33BC0D330E1F48091380783306D
:10FC500019F42AD4811169C080912302882391F17B
:10FC600011E080913807833009F010E08091210E77
:10FC70009091220E0E94959F00E09C0149EE53E373
:10FC80001DC0D430F9F480913807843019F40CD4B5
:10FC900081115DC0809123028823A1F011E0809141
:10FCA0003807843009F010E08091E60D9091E70D5F
:10FCB0000E94959F00E09C0143EE53E36C2F812F3F
:10FCC0000E94E04ECF5FDF5FC53009F063CFC09385
:10FCD00037074EC05ED980914907882309F463CF66
:10FCE00047C0E12C02EA19E728EB3BE044E650E08C
:10FCF00067E97EE083EF93E37BD88091490788230F
:10FD000009F46CCF35C0E12C0AEA19E728EB3BE097
:10FD100044E650E06CE57EE08FEE93E369D8809195
:10FD20004907882309F479CF23C0E12C02EB19E7B6
:10FD300028EB3BE044E650E061E27EE08BEE93E3AB
:10FD400057D880914907882309F486CF11C0E12C48
:10FD50000AEB19E728EB3BE044E650E066EE7DE075
:10FD600086EE93E345D880914907882309F492CF22
:10FD7000DF91CF911F910F91EF900895EF920F9324
:10FD80001F93CF93DF9361E081E0BED9D0916F07DD
:10FD9000C0E0D11119C080913807811103C084D30C
:10FDA00081118FC080912302882309F482C081E0F1
:10FDB00090913807911180E004E024E047ED53E38F
:10FDC0006C2F0E94B14E75C0D130D9F480913807A4
:10FDD000813019F469D381117BC08091230288237B
:10FDE00009F467C011E080913807813009F010E014
:10FDF00080919D0E0E94409F00E09C0143ED53E3E3
:10FE000054C0D230D9F480913807823019F44CD3E1
:10FE100081116FC080912302882309F44AC011E048
:10FE200080913807823009F010E08091620E0E94C4
:10FE3000409F00E09C014FEC53E337C0D330D1F436
:10FE400080913807833019F42FD3811163C08091DA
:10FE50002302882371F111E080913807833009F083
:10FE600010E08091270E0E94409F00E09C014BEC27
:10FE700053E31BC0D430E9F480913807843019F47F
:10FE800013D3811158C080912302882391F011E08F
:10FE900080913807843009F010E08091EC0D0E94C9
:10FEA000409F00E09C0145EC53E36C2F812F0E94A2
:10FEB000E04ECF5FDF5FC53009F06BCFC0933707EF
:10FEC0004AC067D880914907882309F46BCF43C0A3
:10FED000E12C02EC19E72FEF40E06DE97EE085EDC3
:10FEE00093E30E94B17680914907882309F475CF86
:10FEF00032C0E12C05E01AE72FEF40E062E67EE039
:10FF000081ED93E30E94B17680914907882309F43B
:10FF100081CF21C0E12C08E41AE72FEF40E067E22F
:10FF20007EE08DEC93E30E94B176809149078823AF
:10FF300009F48DCF10C0E12C0BE81AE72FEF40E059
:10FF40006CEE7DE088EC93E30E94B17680914907E6
:10FF5000882309F498CFDF91CF911F910F91EF90F3
:10FF60000895FC0180810895FC01849108954F92C9
:10FF70005F926F927F928F929F92AF92BF92CF9239
:10FF8000DF92EF92FF920F931F93CF93DF936C0159
:10FF90007B015A012901672B31F088248394912C2D
:10FFA000C0E0D0E019C0F8011182108227C03701EB
:10FFB000680C791C76946794E3012197A201BE0135
:10FFC000C601F50119951816190654F0892BC9F0C8
:10FFD0004301FFEF8F1A9F0AE814F90440F702C0AB
:10FFE0007E01FACFCE15DF0530F4CE0102968816D9
:10FFF000990620F02196F801D183C0838FEF9FEFFF
:020000021000EC
:1000000005C0F801D183C08380E090E0DF91CF91FB
:100010001F910F91FF90EF90DF90CF90BF90AF9026
:100020009F908F907F906F905F904F9008958F92E8
:100030009F92AF92BF92CF92DF92EF92FF920F9377
:100040001F93CF93DF93EC016B017A01FB011995AC
:1000500087FD06C0082F10E020E030E0219620C187
:10006000982F907E903CC1F4082F0F7110E020E093
:1000700030E04801590186E0880C991CAA1CBB1C81
:100080008A95D1F7CE010196F60119958F739501E6
:100090008401082B229604C1982F907F903E19F579
:1000A0008F70882E912CA12CB12C16E0880C991CF5
:1000B000AA1CBB1C1A95D1F7CE010196F601199521
:1000C0008F73882A06E0880C991CAA1CBB1C0A9511
:1000D000D1F7CE010296F60119958F73950184012F
:1000E000082B2396DDC0982F987F903F81F587706D
:1000F000882E912CA12CB12CF6E0880C991CAA1CFE
:10010000BB1CFA95D1F7CE010196F60119958F73B4
:10011000882AA6E0880C991CAA1CBB1CAA95D1F7BA
:10012000CE010296F60119958F73882AB6E0880CE5
:10013000991CAA1CBB1CBA95D1F7CE010396F601F7
:1001400019958F7395018401082B2496A9C0982FC7
:100150009C7F983FE9F58370882E912CA12CB12CBF
:1001600056E0880C991CAA1CBB1C5A95D1F7CE01ED
:100170000196F60119958F73882A66E0880C991C00
:10018000AA1CBB1C6A95D1F7CE010296F6011995FF
:100190008F73882A76E0880C991CAA1CBB1C7A9560
:1001A000D1F7CE010396F60119958F73882AE6E000
:1001B000880C991CAA1CBB1CEA95D1F7CE010496A9
:1001C000F60119958F7395018401082B259668C057
:1001D000982F9E7F9C3F09F04AC08170882E912CF9
:1001E000A12CB12C86E0880C991CAA1CBB1C8A95FA
:1001F000D1F7CE010196F60119958F73882A96E002
:10020000880C991CAA1CBB1C9A95D1F7CE010296AA
:10021000F60119958F73882A26E0880C991CAA1C70
:10022000BB1C2A95D1F7CE010396F60119958F7361
:10023000882A36E0880C991CAA1CBB1C3A95D1F779
:10024000CE010496F60119958F73882A46E0880C32
:10025000991CAA1CBB1C4A95D1F7CE010596F60144
:1002600019958F7395018401082B269619C0982F34
:10027000907C903849F4082F007C003871F4219666
:10028000CE01F6011995F7CF082F0E7F0D3F28F00C
:100290002196CE01F6011995F7CF00E010E0980104
:1002A000E114F10429F0F7010083118322833383E1
:1002B000CE01DF91CF911F910F91FF90EF90DF90D2
:1002C000CF90BF90AF909F908F9008951F93CF9342
:1002D000DF9300D01F92CDB7DEB710E0AE014F5FC5
:1002E0005F4F61EB7FE7A3DE49815A816B817C819F
:1002F000452B462B472B11F01F5FF0CF812F0F901E
:100300000F900F900F90DF91CF911F9108951F9341
:10031000CF93DF9300D01F92CDB7DEB710E0AE01D0
:100320004F5F5F4F64EB7FE782DE49815A816B81CB
:100330007C81452B462B472B11F01F5FF0CF812F7F
:100340000F900F900F900F90DF91CF911F91089514
:1003500010928F0780918A0710928A07882349F0AC
:1003600040E050E0BA018AE39CE60E949E770C943C
:10037000BF4D2091640230916502409195075091E4
:1003800096076091970770919807C901840F951F90
:100390002436310571F4473051056105710514F0BB
:1003A000069732C04A3F5F4F6F4F7F4F54F5069616
:1003B0002BC02436310524F48536910514F504C08C
:1003C0008436910524F41DC08A3091053CF0883EA6
:1003D00043E094072CF087EE93E002C08AE090E0BF
:1003E0002817390761F09093650280936402109298
:1003F00095071092960710929707109298070C9401
:10040000894984E690E0E3CF8A30910504F78AE0D9
:1004100090E0E9CFCF93DF931F92CDB7DEB7809105
:10042000BA09811103C08CEF99E02FC0211103C0DC
:100430008AEB99E02AC08DE0815048F0440F411DBD
:10044000E82FF0E0E450F64F90814927F5CF8091F6
:1004500081078417A9F0409381078AEB99E06983AB
:1004600035DF90E06981861B910997FF02C080E02B
:1004700090E0809392071092930788E08093250282
:100480008091930790E08654964F0F90DF91CF9123
:10049000089580938F0710928B0710928C0710920B
:1004A0008D0710928E07089580918A0710928A070F
:1004B0000895CF92DF92EF92FF920F931F930E94C5
:1004C0006C3100917D0710917E0720917F0730915C
:1004D00080076B017C01C01AD10AE20AF30AF7FC1B
:1004E00013C020917C07209520937C07DC01CB0171
:1004F0008A549C4FAF4FBF4F80937D0790937E07E8
:10050000A0937F07B093800781E090917C079111C1
:1005100001C080E01F910F91FF90EF90DF90CF908E
:100520000895CF9393E09093230281111092A10735
:100530000E946C31DC01CB018C509E4FAF4FBF4FFE
:1005400080939B0790939C07A0939D07B0939E0771
:1005500068E873E182E090E00F946466C6E0C15001
:1005600049F00F94F96562E070E080E090E00E944D
:100570009D31F5CFCF910895AF92BF92CF92DF9288
:10058000EF920F931F93CF93DF9300D01F92CDB7BD
:10059000DEB7809124028F3F09F444C00E946C3181
:1005A000009182071091830720918407309185077D
:1005B000DC01CB01801B910BA20BB30BB7FD32C04A
:1005C00090913E10809141108F5F8F70981751F17C
:1005D000E091240284E0E802F0011124E055FB4F91
:1005E00020E030E040E752E46081718182819381B4
:1005F0000F946B6C69837A838B839C83A12CB12CC1
:100600006501E12C8E010F5F1F4F26E732E042E7C4
:1006100052E06EE672E08AE692E00F94841C8FEF5F
:10062000809324020F900F900F900F90DF91CF9145
:100630001F910F91EF90DF90CF90BF90AF900895F2
:100640000F931F930E946C3100919B0710919C07A0
:1006500020919D0730919E07DC01CB01801B910BFF
:10066000A20BB30BB7FD11C08091030181FB992749
:1006700090F981E089279091030192FF8260909127
:10068000000196FF84608093A1078091A10781708B
:100690009091A10791FD826090917007891741F1B7
:1006A0008130A9F028F0823041F0833059F01EC02B
:1006B000913089F09230A9F019C0992361F09330FC
:1006C00081F014C0913069F0923081F404C0992314
:1006D00041F0933059F4909194079150909394077E
:1006E00005C0909194079F5F909394078093700743
:1006F0001F910F910895CF93DF930E94BF4DE4E0C7
:10070000F1E080818D7F8083C5E0D1E08881809594
:10071000827043E051E0DA018C9380818B7F80838B
:100720008881809584708C9321E031E0D9018C918F
:100730008F7B8C938091020180958074809300015F
:1007400080818E7F8083888180958170FA0180838B
:1007500082E08093A00774DF10929407DF91CF911D
:100760000C94F9B181E09091A307911101C080E050
:100770000895CF93DF932091BA0721111EC0FC0189
:1007800001900020E9F73197EF01C81BD90BC73161
:10079000D10534F031972081207C2038D9F3F4CF73
:1007A000BC01DD27AE0183EA97E00F949774CD5525
:1007B000D84F188283E080932302DF91CF91089570
:1007C000CF93DF93CDB7DEB78E819091BA078917AB
:1007D00080F08093BA079E01275F3F4F4F81588575
:1007E00066E170E083EA97E00F94E07483E0809321
:1007F0002302DF91CF9108950F931F93CF93DF933F
:100800008C0167FF03C01092BA0760E08091BA07BD
:1008100090E0262F062E000C330B281739070CF119
:100820006093BA07C8010F94F973F801E80FF91F34
:10083000EF01C01BD10BC731D10534F03197849142
:10084000807C8038D9F3F4CFDD27AE01B80183EA8C
:1008500097E00F941A74CD55D84F188283E0809397
:100860002302DF91CF911F910F9108954F925F92D4
:100870006F927F928F929F92AF92BF92CF92DF92B0
:10088000EF92FF920F931F93CF9376DED9DE809184
:10089000A10782FF15C080917B07811113C091E0F1
:1008A00090937B072091AF19211103C080913907E4
:1008B000892780938A071092AF1981E032DE02C047
:1008C00010927B078091030180958170C091A007F1
:1008D0008C17B9F08093A007882309F48EC164EFC8
:1008E00071E080E090E00E94CD9E0E94F48FC230C3
:1008F00009F07EC10E94C49083E0809323020E948D
:10090000BF4D0E946C316B017C0180917707909103
:100910007807A0917907B0917A07A7019601281B63
:10092000390B4A0B5B0B57FF05C080919A07882350
:1009300009F43DC2D701C6018C599F4FAF4FBF4F3D
:100940008093770790937807A0937907B0937A07FD
:1009500060919407062E000C770B77FF03C071950A
:1009600061957109062E000C770B880B990B0F947B
:10097000066D2B013C0120E030E040E050E40F9494
:10098000676E87FF05C080918A07811183C093C07D
:1009900080918F07882309F456C080908B07909030
:1009A0008C07A0908D07B0908E0781149104A1044C
:1009B000B104E1F120E030E040E05FE3C301B201C7
:1009C0000F94A26E2B013C01C701B6016819790989
:1009D0008A099B090F94046D9B01AC01C301B2010C
:1009E0000F946B6C20E030E04AE754E40F94A26E61
:1009F0004B015C0120E030E040EA52E40F94676E66
:100A000087FF0FC020E030E040EF51E4C501B401A2
:100A10000F94676E87FD0AC02AE030E040E050E0A6
:100A200009C024E630E040E050E004C021E030E0BE
:100A300040E050E0C0928B07D0928C07E0928D0787
:100A4000F0928E0704C021E030E040E050E0A09139
:100A500094070A2E000CBB0B0F940D7022E030E0BF
:100A600040E050E00F94D06F8091950790919607E9
:100A7000A0919707B0919807820F931FA41FB51FED
:100A80008093950790939607A0939707B093980744
:100A900010929407D701C6018856954CAF4FBF4FAF
:100AA0008093730790937407A0937507B0937607AC
:100AB00081E080932302209190073091910741E8D3
:100AC000283A340741F480912502882309F4A8C00C
:100AD0008150809325022554324571F4809193070B
:100AE00090919207891740F490912502992309F477
:100AF000A7C091509093250280916F0081FB22271F
:100B000020F981FF05C080916F008D7F80936F0079
:100B10008091510F9091520FA091530FB091540FAB
:100B2000222329F020916F00226020936F003AE089
:100B3000B695A795979587953A95D1F7009721E0B7
:100B4000A207B10520F08FEF9FEFA0E0B0E09695EF
:100B5000879520912302211105C030919A07311108
:100B600022C139C0009739F0409171075091720746
:100B70004817590780F580919A07811103C02230E8
:100B800008F076C0C1E08091900790919107885A53
:100B9000914809F0C0E08C2F0E948B49CC2309F4C6
:100BA00073C0D6DB10928A070E946C31DC01CB0146
:100BB0008C199D09AE09BF09009171071091720748
:100BC00020E030E0081719072A073B0720F490932C
:100BD0007207809371078091900790919107885ACE
:100BE000914809F4A3C080919F0781119FC0CAC09A
:100BF00060E085E394E300DE7FCEEDD5C23009F4FA
:100C00007BCE60E088E294E3F7DD809190079091DD
:100C10009107885A914809F46FCE0E94C3776CCE31
:100C20008CE0809325028091710790917207019763
:100C3000909372078093710781E0809323024BCFDA
:100C400096E09093250291E0909323028F5F80932A
:100C50009307D701C6018856954CAF4FBF4F80937D
:100C6000730790937407A0937507B093760744CFEA
:100C7000243030F0243009F085CF1092230282CF47
:100C800081E0809323027ECF80919A07811114C066
:100C900080911F06811107C081E080931F0686EEB8
:100CA00095E00E942C3686EE95E00E94633681E046
:100CB0008093990780939A0783E00E94D84C61E063
:100CC00086EE95E00E948536E0919007F0919107BD
:100CD00019951092990780919A07882309F462CF99
:100CE00086EE95E00E94673691E0811101C090E0A8
:100CF00090939A07992309F455CF0E946C31DC0137
:100D0000CB018C199D09AE09BF09C0907107D09025
:100D10007207E12CF12CC816D906EA06FB0608F08A
:100D200046C0909372078093710741C058E9C50E81
:100D30005AE3D51EE11CF11CC0927307D0927407D0
:100D4000E0927507F092760780919A0781112FC083
:100D500080912302813099F0833049F5CF911F9122
:100D60000F91FF90EF90DF90CF90BF90AF909F904A
:100D70008F907F906F905F904F900C94F24D1092F7
:100D8000230215C08091730790917407A091750795
:100D9000B0917607C81AD90AEA0AFB0AF7FCD4CF41
:100DA0000E94C377D1CF009709F4ECCEDDCECF916E
:100DB0001F910F91FF90EF90DF90CF90BF90AF9079
:100DC0009F908F907F906F905F904F90089561E01B
:100DD00013DD0C94C377CF93DF931F921F92CDB78F
:100DE000DEB789839A8387DC89819A81F0DF0F904F
:100DF0000F90DF91CF910C94C44D8091090A82FD30
:100E000005C08091A219823061F410C08091BA09A6
:100E1000811103C08CEF99E002C08AEB99E061E098
:100E2000A8CC813031F081E094E305C08BE194E3FC
:100E300002C08FE094E36FEFDFCC8091090A82FF5C
:100E400009C083FF04C080913908811106C020E0E9
:100E50002093A2078091A20708958091C4079091E2
:100E6000C507A091C607B091C7070097A105B105B6
:100E700071F3BC01CD016D597F4F8F4F9F4F24E619
:100E800030E040E050E00F94AE6F6091C007709189
:100E9000C1078091C2079091C3070F94AE6FD8CF5E
:100EA00088EA91E89093910780939007089561E014
:100EB000FC0180810E9491338FEF0C9457AACF934D
:100EC000DF93EC018A810E9418AA60E08881DF919B
:100ED000CF910C9491338F929F92AF92BF92EF92E9
:100EE000FF920F931F93CF93DF93EC018B017A0155
:100EF0000E946C314B015C012CE2820E21E0921EBB
:100F0000A11CB11C0E9431AA8B838F3F61F40E9407
:100F10006C31DC01CB0188199909AA09BB09B7FD1D
:100F2000F1CF81E10DC08E3F51F4B701C8010E949D
:100F300038AA0E9431AA0E9431AA11E003C08FE0B2
:100F4000898310E0CE01B3DF812FDF91CF911F9114
:100F50000F91FF90EF90BF90AF909F908F9008956A
:100F6000CF92DF92EF92FF926A017B010E946C3177
:100F7000C60ED71EE81EF91E0E9431AA8F3F61F0EF
:100F80000E946C31DC01CB018C199D09AE09BF09AF
:100F9000B7FDF2CF80E001C081E0FF90EF90DF90DD
:100FA000CF900895EF92FF921F93CF93DF9300D0DD
:100FB0001F92CDB7DEB77C01162F29833A834B836E
:100FC0005C837DDF48E552E060E070E0C701C8DF88
:100FD000812F80640E9457AA8C810E9457AA8B811E
:100FE0000E9457AA8A810E9457AA89810E9457AA03
:100FF000112311F087E801C085E90E9457AA1C302F
:1010000011F40E9431AA10E00E9431AAF7018383F3
:1010100087FF04C01F3F11F01F5FF6CF0F900F90A6
:101020000F900F90DF91CF911F91FF90EF90089557
:101030008F929F92AF92BF92CF92DF92EF92FF92E8
:101040000F931F93CF93DF93EC01162F1C8219820D
:1010500048830E946C316B017C0120EDC20E27E0B9
:10106000D21EE11CF11CA89561E088810E94913399
:1010700061E088810E9455330E9429AA85E08A8315
:101080000E9418AA0AE08FEF0E9457AA0150D9F7D0
:10109000A89520E030E0A90160E0CE0183DF8B83DA
:1010A000813061F00E946C31DC01CB018C199D090B
:1010B000AE09BF09B7FDEDCF81E055C0A8952AEA7A
:1010C00031E040E050E068E0CE016CDF853011F4A3
:1010D00081E009C004E00E9431AA8B830150D9F756
:1010E0008A3A51F482E08C83A8958C81823081F019
:1010F000812C912C540111C00E946C31DC01CB0178
:101100008C199D09AE09BF09B7FDD9CF82E02BC06C
:10111000812C912CA12C80E4B82E20E030E0A90194
:1011200067E3CE013FDFA501940169E2CE013ADF1A
:101130008B83882361F00E946C31DC01CB018C1918
:101140009D09AE09BF09B7FDE8CF8AE00CC08C81CC
:101150008230D1F420E030E0A9016AE3CE0122DF41
:10116000882329F088E08983CE01A1DE16C00E9481
:1011700031AA807C803C11F483E08C830E9431AAE8
:101180000E9431AA0E9431AACE0191DE173018F4D4
:101190001A8381E003C088E1898380E0DF91CF91E9
:1011A0001F910F91FF90EF90DF90CF90BF90AF9085
:1011B0009F908F9008950F931F93CF93DF93EC012F
:1011C00089018C81833039F089E0440F551F661FF7
:1011D000771F8A95D1F79A01AB0161E1CE01E2DE7A
:1011E000811109C040E052E0B801CE01DF91CF91FA
:1011F0001F910F9170CE84E08983CE0158DE80E08C
:10120000DF91CF911F910F910895CF93DF93EC0160
:10121000862FBA010E945CAA8FEF0E9457AA8FEF17
:101220000E9457AA0E9431AA8B83982F9F719530F4
:1012300031F083E18983CE013ADE80E001C081E0B4
:10124000DF91CF9108950F931F93CF93DF93EC011C
:1012500089018C81833039F089E0440F551F661F66
:10126000771F8A95D1F79A01AB0168E1CE019ADE2A
:1012700081111EC0A8016EEFCE01C7DF8823E1F007
:1012800048E552E060E070E0CE016ADE882371F04C
:1012900020E030E0A9016DE0CE0184DE81110AC0BA
:1012A0000E9431AA811106C011E007C087E103C086
:1012B00086E001C086E1898310E0CE01F8DD812F50
:1012C000DF91CF911F910F910895CF93DF931F92DC
:1012D000CDB7DEB72091B1193091B219CE01019688
:1012E0002115310519F0821B930B02C0875B9941D0
:1012F0000F90DF91CF910895FC01238121110C946F
:101300001C9A08958091090A847F8B7F8093090A33
:101310001092C0071092C1071092C2071092C30723
:101320001092C4071092C5071092C6071092C70703
:1013300010923508109274088EE091E0E5E7F8E02D
:10134000DF019C011D9221503040E1F78FEF809327
:10135000B9090895FC0120E03EE2DB014C914032E6
:1013600041F0283011F430833196DB014C914083F9
:1013700031962F5F6F5F7F4F2B3079F71082089582
:101380002F923F924F925F926F927F928F929F9295
:10139000AF92BF92CF92DF92EF92FF920F931F9383
:1013A000CF93DF93CDB7DEB7C356D1090FB6F8940C
:1013B000DEBF0FBECDBF8C015B014A014DB65EB6EC
:1013C000312C7E0187E5E80EF11C9BE1292E4AEBCA
:1013D00059E0BE016F5F7F4FC5010E948C981816BF
:1013E0000CF005C18C85282F2871203109F074C0BC
:1013F0009091BF079150923008F46EC06DB67EB6E2
:10140000BE016F5F7F4FC701A5DF0115110521F0F8
:10141000F8018081811173C021E081E090E0F70143
:1014200001900020E9F73197EE19FF09E80FF91F45
:1014300032968DB79EB78E1B9F0B0FB6F8949EBF4A
:101440000FBE8DBFEDB7FEB731966F01211102C0FF
:10145000B80102C060EC74E0C6010F948274B70159
:10146000C6010F946C7460EC74E0C6010F946C7448
:101470001CAE1FAE21E0A701B501CE01CC960E94A3
:10148000189C81110DC08091BF07811109C00E9475
:101490004FA381E396E30E9441A3C7010E94E8A8FD
:1014A000FE01FC96DE019196822D01900D928A95A7
:1014B000E1F740E050E0BE016F5D7F4FC60160DFA5
:1014C000CE01819619DFCE01CC9616DF0FB6F894C7
:1014D0007EBE0FBE6DBE7BCF9981992309F487C074
:1014E000953E09F474CF9E3209F471CF9091BA09F8
:1014F0009E3209F46CCF8A7009F069CF0AC0F801F6
:1015000001900020E9F73197CF01801B910B20E07B
:1015100086CF81E0203109F080E09091090A80FBBC
:1015200094F99093090A811108C08985873409F0DC
:101530004ECF8A858E3709F44ACF8091BF0781301C
:1015400021F068F08230B9F142CF8091BD079091CF
:10155000BE0701969093BE078093BD0738CFBE01AA
:101560006F5F7F4F8CEF99E0F5DE0115110511F0EB
:10157000680105C08CEFC82E89E0D82E08C0F6019E
:1015800081916F018823B1F30E9491A8F8CFF601F1
:1015900081916F01882319F00E9491A8F8CF80E211
:1015A0000E9491A86D8D7E8D8F8D98A14AE050E0AC
:1015B0000E94A4A90CCFBE016F5F7F4F8CEF99E012
:1015C000C9DE8114910441F06CEF79E0C4010F94FD
:1015D0005974892B51F40BC0832D90E02091BB07E7
:1015E0003091BC078217930711F03394F0CE0FB6F9
:1015F000F8945EBE0FBE4DBECD59DF4F0FB6F894C6
:10160000DEBF0FBECDBFDF91CF911F910F91FF9035
:10161000EF90DF90CF90BF90AF909F908F907F9092
:101620006F905F904F903F902F900895CF93DF93EE
:10163000CDB7DEB76B970FB6F894DEBF0FBECDBF48
:101640001092BF0740E050E0BA018EE999E00E9495
:101650003B998BE1EEE9F9E0DE01119601900D92E4
:101660008A95E1F740E050E0BE016F5F7F4F80E078
:1016700090E086DECE0101963FDE6B960FB6F894C1
:10168000DEBF0FBECDBFDF91CF9108950F931F93A3
:10169000CF93DF93CDB7DEB72D970FB6F894DEBFAB
:1016A0000FBECDBF80913908882391F0BE016F5FD6
:1016B0007F4F86E398E00E94AE968E010F5F1F4F2A
:1016C000F80181918F01882339F00E9491A8F8CF09
:1016D00087E296E30E9441A38AE00E9491A82D969A
:1016E0000FB6F894DEBF0FBECDBFDF91CF911F9133
:1016F0000F910895CF92DF92EF92FF920F931F9375
:10170000CF93DF93CDB7DEB7EDB6FEB6DC010D901B
:101710000020E9F79D01281B390B2C5F3F4F4DB787
:101720005EB7421B530B0FB6F8945EBF0FBE4DBFA2
:101730000DB71EB70F5F1F4F9F938F9381EE95E3F9
:101740009F938F931F930F930F94B174680154E08C
:10175000C50ED11C0F900F900F900F900F900F900F
:10176000F6018081882349F0082E000C990B0F9414
:10177000DD73F60181936F01F3CFC8010F941C5BF9
:101780008DED95E30F94175B0FB6F894FEBE0FBE78
:10179000EDBEDF91CF911F910F91FF90EF90DF9001
:1017A000CF9008958091090A83FF03C084608093DD
:1017B000090A08951092D60C8091090A8F7D8B7FBB
:1017C0008093090A0E94206B882321F086E398E029
:1017D0000C941C9A0895EEDF8091090A877F80930C
:1017E000090A08950F931F93CF93DF938B01EA01AA
:1017F000DB016D917C910E94AE96D801ED91FC9138
:101800009081888191110EC08936B0F48FE2808377
:10181000F8018081918101969183808388818F5F17
:1018200088830AC0893680F73196D801ED93FC93FE
:1018300088818F5F8883E1CFDF91CF911F910F91D6
:1018400008950F931F93CF93DF9300D0CDB7DEB7EA
:101850009C012F5F3F4F3B832A832FE2FC012083B3
:1018600081E0898310E00BE180917408181770F40F
:10187000019FC0011124AE014F5F5F4FBE016E5F3B
:101880007F4F8B58974FAEDF1F5FEECF89818B352F
:1018900070F4AE014F5F5F4FBE016E5F7F4F86E316
:1018A00098E0A0DF8A819B8101979B838A83EA81EC
:1018B000FB8110820F900F900F90DF91CF911F91BD
:1018C0000F9108958091090A82FF1FC085EA94E371
:1018D0000E9441A36091C0077091C1078091C20727
:1018E0009091C3074AE050E00E9493A98FE20E94C2
:1018F00091A86091C4077091C5078091C607909127
:10190000C7074AE050E00C94A4A984E994E30C943E
:1019100041A3EF92FF920F931F93CF93DF938C011C
:10192000FC0101900020E9F73197EF01C81BD90BAA
:10193000109236086EE470E00F9477747C01009783
:1019400029F4FE013197E00FF11F0EC060E270E054
:101950000F9477748C010F5F1F4F6AE270E0C7012C
:101960000F947774FC0131978DE081838AE0828344
:101970001382B80186E398E00E94AB9E80913608FE
:10198000882361F00E9452A38DE794E3DF91CF9109
:101990001F910F91FF90EF900C9441A3DF91CF9195
:1019A0001F910F91FF90EF90089586E398E00E94B9
:1019B000D19986E398E00E941C9A8091090A8D7F54
:1019C0008E7F8093090A1092C0071092C10710926F
:1019D000C2071092C30781E08093CF0C08950F9344
:1019E0001F93CF93DF93CDB7DEB76B970FB6F89405
:1019F000DEBF0FBECDBF8B0122E02093BF079093C7
:101A0000BC078093BB0740E050E0BA0183E899E04F
:101A10000E943B998BE1E3E8F9E0DE011196019029
:101A20000D928A95E1F7A801BE016F5F7F4F80E0BC
:101A300090E0A6DCCE0101965FDC6B960FB6F894C1
:101A4000DEBF0FBECDBFDF91CF911F910F910895E3
:101A5000CF93DF93CDB7DEB76B970FB6F894DEBFA9
:101A60000FBECDBF81E08093BF071092BE071092DA
:101A7000BD0740E050E0BA0183E899E00E943B993D
:101A80008BE1E3E8F9E0DE01119601900D928A9571
:101A9000E1F740E050E0BE016F5F7F4F80E090E0F3
:101AA0006FDCCE01019628DC8091BD079091BE07C6
:101AB0006B960FB6F894DEBF0FBECDBFDF91CF910E
:101AC00008952F923F924F925F926F927F928F92E2
:101AD0009F92AF92BF92CF92DF92EF92FF920F93BD
:101AE0001F93CF93DF93CDB7DEB76C970FB6F89403
:101AF000DEBF0FBECDBF5C014C8F2DB63EB6198246
:101B00001C82FB0180819E012F5F3F4F49018F3274
:101B100039F083E899E0F501918380838B0160C0FF
:101B20008EE999E0F501918380838B010F5F1F4F50
:101B30000115110509F454C04DB65EB66FE270E0B0
:101B4000C8010F9477743C010817190708F048C0C2
:101B50007C01E01AF10AFF24C70101962DB73EB7B8
:101B6000281B390B0FB6F8943EBF0FBE2DBF8DB7A3
:101B70009EB701966C01A701B8010F949774F60106
:101B8000EE0DFF1D10823C8D332319F0C6010E941B
:101B9000E8A8F5016081718121E0A601C4010E94DD
:101BA000189C811111C0B60180E694E30E9455A3F0
:101BB0008DE594E30E9441A30FB6F8945EBE0FBE7C
:101BC0004DBE00E010E00CC0F501918280828301DF
:101BD0000F5F1F4F0FB6F8945EBE0FBE4DBEA8CF6D
:101BE000C4018ADBC8010FB6F8943EBE0FBE2DBEFD
:101BF0006C960FB6F894DEBF0FBECDBFDF91CF91CC
:101C00001F910F91FF90EF90DF90CF90BF90AF901A
